:100000000C94A7040C94CF040C94CF040C94CF044C
:100010000C94CF040C94CF040C94CF040C94CF0414
:100020000C94CF040C94CF040C947D250C94CF0435
:100030000C94CF040C94CF040C94CF040C94CF04F4
:100040000C942B090C94CF040C94CF040C94CF0483
:100050000C94CF040C94CF040C94CF040C94CF04D4
:100060000C94CF040C94CF040C94CF040C94CF04C4
:100070000C94CF040C94CF040C94CF040C94CF04B4
:100080000C94C90F0C94CF040C94CF040C94CF049F
:100090000C94CF040C94CF040D0A416C6C206E6F4D
:1000A000646573202D20287229656164696E672C50
:1000B0002028702970696E673A000D0A50617573C7
:1000C00065642C2070726573732027502720746F2D
:1000D00020756E7061757365000D0A57616B652040
:1000E0007768696368206E6F64653A000D0A53741F
:1000F00061727475702C204920616D20636F6F727E
:1001000064696E61746F722E0D0A000D0A456E747B
:100110006572206E65772050414E4944000D0A45B6
:100120006E746572206E6577206368616E000D0ADB
:1001300053747265616D206D6F646520746F20610A
:100140006464723A000D0A456E7465722073686FBC
:10015000727420616464723A000D0A006E6F74203C
:100160007965742076616C6964000D0A49507636B1
:1001700020364C4F5750414E204946203D20006EBE
:100180006F74207965742076616C6964000D0A498A
:100190005076362045746865726E65742049462035
:1001A0003D2000506172743D524600556E6B6E6F7B
:1001B000776E3F00425553595F52585F4141434B60
:1001C0005F4E4F434C4B0052585F4141434B5F4F92
:1001D0004E5F4E4F434C4B0052585F4F4E5F4E4F59
:1001E000434C4B0054585F415245545F4F4E0052B0
:1001F000585F4141434B5F4F4E00425553595F5446
:10020000585F4152455400425553595F52585F411F
:1002100041434B00504C4C5F4F4E005452585F4F7F
:1002200046460052585F4F4E00425553595F54584E
:1002300000425553595F525800505F4F4E00526173
:1002400064696F205374617465203D200050414EF5
:10025000204944203D203078000D0A723D726561CE
:1002600064696E67206E3D6E616D6520773D7761D4
:100270006B6520503D70617573653A20000D0A640E
:100280003D64756D7020743D7461626C6520693DDC
:10029000696E666F20703D70696E6720733D737480
:1002A0007265616D20633D6368616E000D0A50697F
:1002B0006E67696E67206E6F646520000D0A4E6F71
:1002C000726D616C206D6F6465000D0A537461720C
:1002D0007475702C204920616D20636F6F726469A2
:1002E0006E61746F72206F6E20636820002C20682E
:1002F0006F7073203D2000206F6E20636820000D1A
:100300000A4173736F63696174696E6720746F204B
:10031000000D0A000D0A0D0A5245472044554D5064
:100320000D0A0020525353493D00204C51493D00D5
:100330000D0A50696E6720726573706F6E73652069
:1003400066726F6D20000D0A50696E6720726571CC
:10035000756573742066726F6D206E6F6465200022
:100360002066726F6D20706172656E7420000D0AD8
:1003700044726F7070696E67206368696C642000F6
:100380000D0A0020202020202020202020202020B6
:10039000202020202020202020202020202020205D
:1003A00020000D0A0D0A2020204C6F6E672041644A
:1003B000647220202020202053686F7274204164D2
:1003C000647220202020202020495076362041646D
:1003D00064720D0A0020202020000D0A000D0A4E34
:1003E0006574776F726B20547265650D0A000D0A93
:1003F0005461626C6520446174613A0D0A000D0A13
:100400004261642064657374206E6F6465202852B5
:100410005029000D0A0020486F7073203D20000D08
:100420000A4173736F636961746564206E6F6465FC
:1004300020000D0A526F7574652064617461206636
:10044000726F6D20436F6F7264000D0A526F757486
:1004500065206461746120746F206368696C640056
:100460001201000202000040EB03182000100102FC
:100470000301090243000201008032090400000167
:1004800002020100052400100105240103010424D7
:1004900002060524060001070584032000FF090465
:1004A0000100020A00000007058502200000070580
:1004B000060220000012010002EF020140EB0322BD
:1004C00020001001020301090264000301008032D0
:1004D000080B00020202FF0009040000010202FFF3
:1004E0000005240010010524010001042402000578
:1004F0002406000107058303080010090401000217
:100500000A000000070581024000000705020240C2
:10051000000009040200010300000009211101008C
:10052000012235000705840320001006FFFF0901A2
:10053000A10109020903150026FF00750895208115
:100540000209040905150026FF007508952091028F
:1005500009060907150026FF0075089504B102C0B9
:10056000120100020202FF40EB03192000100102F9
:100570000301090243000201008032090400000166
:100580000202FF00052400100105240100010424DB
:100590000200052406000107058303080010090472
:1005A0000100020A00000007058102400000070563
:1005B000020240000012010002020C0740EB03227D
:1005C00020001001020301090239000201008032FB
:1005D0000904000002020C07000705810240000028
:1005E00007050202400000090401000103000000A9
:1005F00009211101000122350007058303200010A5
:100600000C03410054004D0045004C002403410000
:1006100056005200200055005300420020005200B6
:1006200055004D00200043004F004F005200440091
:10063000040309040D0A52657374617274696E676C
:10064000204D41432026204E574B0D0A000D0A52E3
:10065000657374617274204D41432E0D0A000D0ABA
:1006600052657374617274204D41432E0D0A00016E
:100670000101000201010003010100040101000663
:10068000010100070101000A0101000B0101000C3A
:100690000101000D0101000E010100110101001412
:1006A0000101001601010002020100010102000225
:1006B0000102000301020004010200050102001B07
:1006C0000201000101010102010101030101010414
:1006D0000101010501010101010201020102010301
:1006E000010201000101FD020101FD010101FD0600
:1006F0000101FD030101FD040101FD50414E49448A
:100700003A203078424141440041746D656C0000EC
:100710000000000D0A004E756D6265720909537480
:100720006174650909495020416464726573730DF1
:100730000A00736963736C6F7770616E20756E6306
:100740006F6D70726573735F6864723A2065727260
:100750006F7220756E737570706F7274656420555A
:10076000445020636F6D7072657373696F6E0D0A0C
:1007700000736963736C6F7770616E20756E636F61
:100780006D70726573735F6864723A206572726F20
:100790007220636F6E74657874206E6F7420666F5C
:1007A000756E640D0A00736963736C6F7770616EA8
:1007B00020756E636F6D70726573735F6864723AF3
:1007C000206572726F7220756E6B6E6F776E20632C
:1007D0006F6D70726573736564206D6361737420EF
:1007E000616464726573730D0A00736963736C6F7F
:1007F0007770616E20756E636F6D70726573735F75
:100800006864723A206572726F7220636F6E7465ED
:100810007874206E6F7420666F756E640D0A0073B5
:100820006963736C6F7770616E20756E636F6D7046
:10083000726573735F6864723A206572726F7220BA
:10084000636F6E74657874206E6F7420666F756E5A
:10085000640D0A00736963736C6F7770616E207545
:100860006E636F6D70726573735F6864723A206552
:1008700072726F7220636F6E74657874206E6F741D
:1008800020666F756E640D0A00736963736C6F7711
:1008900070616E20756E636F6D70726573735F68E3
:1008A00064723A206572726F7220756E6B6E6F772C
:1008B0006E20636F6D70726573736564206D636124
:1008C000737420616464726573730D0A00736963E5
:1008D000736C6F7770616E20756E636F6D7072658B
:1008E00073735F6864723A206572726F7220636F0F
:1008F0006E74657874206E6F7420666F756E640D0B
:100900000A00736963736C6F7770616E20756E6334
:100910006F6D70726573735F6864723A206572728E
:100920006F7220636F6E74657874206E6F742066CA
:100930006F756E640D0A0045464765666700202B9B
:100940002D2E3031323334353637383968001124A2
:100950001FBECFEFD0E2DEBFCDBF14BE88E10FB621
:10096000F89480936000109260000FBE15E0A0E044
:10097000B1E0E2E5F4E001E00BBF02C007900D92A8
:10098000A83EB107D9F71CE1A8EEB5E001C01D9261
:10099000AB3CB107E1F70E9426080C9458730C9405
:1009A000000080916A11089580E01C9981E008950B
:1009B0002D982C988DE090E00197F1F72D9A0895ED
:1009C00008950895089581E06FE140E00E94650A6E
:1009D00008950E94E304282F8151823058F022307C
:1009E00049F0213039F080E090E02E3129F481E0A7
:1009F00090E0089581E090E00895CF93DF93EC01BB
:100A00000E94E304863021F0813011F084E407C0B5
:100A100086E06FE140E00E94650A888380E4DF9110
:100A2000CF91089583E067E040E00E94650A089551
:100A300081E160E245E00E94650A882311F08BE4C1
:100A400008958AE4089581E160E144E00E94650A26
:100A5000089581E16FE040E00E94650A089589E011
:100A60006FE040E00E94650A089588E060E645E096
:100A70000E94650A089585E06FE040E00E94650AE3
:100A8000089588E06FE140E00E94650A089586E0DD
:100A90006FE140E00E94650A8093E905109205121B
:100AA00008951F93CF93DF93EC0114E26991812F96
:100AB0000E94000A1F5F1C32C9F7DF91CF911F917E
:100AC00008951F93682F192F80E20E94000A81E287
:100AD000612F0E94000A1F9108951F93682F192FFC
:100AE00082E20E94000A83E2612F0E94000A1F91A5
:100AF0000895282F8EE268E043E00E94460A089598
:100B00002C988DE090E00197F1F782E06FE140E0F2
:100B100023E00E94460A83E090E00197F1F70895F0
:100B20000E94D404882311F080E408950E94800577
:100B30008BE490E00197F1F70E94E304883011F014
:100B400083E408952C9A80E408951F93162F66304D
:100B500010F082E414C0882329F483E068E043E0C5
:100B600021E004C083E068E043E020E00E94460A00
:100B700083E067E040E0212F0E94460A80E41F9155
:100B800008950E94D404882379F02C9881EE96E091
:100B90000197F1F781E060E00E94A5050E94E3045F
:100BA000883011F083E4089580E408950F931F9333
:100BB000182F062F603110F082E41AC00E94D4046E
:100BC000882311F084E414C0112329F081E160E14D
:100BD00044E021E004C081E160E144E020E00E94C3
:100BE000460A81E16FE040E0202F0E94460A80E43F
:100BF0001F910F9108951F93182F803110F082E4F8
:100C00000DC00E94D404882311F084E407C085E05D
:100C10006FE040E0212F0E94460A80E41F91089572
:100C20001F93182F8B50803110F082E421C00E9456
:100C3000D404882311F084E41BC00E94410581176D
:100C4000B1F088E06FE140E0212F0E94460A0E9447
:100C5000E304863011F0893021F48DE291E00197B0
:100C6000F1F70E944105811711F083E401C080E48F
:100C70001F9108958091E805882329F48CE10E9452
:100C80002C0A8093E8058091E8050895FF920F9360
:100C90001F93082F0E94E304182F0E943A06833006
:100CA00021F00E943A068730B1F4163029F4F02E74
:100CB000F69410E000E00CC0163169F4F8CF86E03D
:100CC00060E645E00E94650A110F110F182B0F5FB7
:100CD0000F15A8F303C00E94BC7E182F812F1F910F
:100CE0000F91FF9008951F93182F0E943A068230AB
:100CF00031F485E060E847E0212F0E94460A0E9417
:100D00003A06833031F484E060E245E0212F0E940E
:100D1000460A1F9108950F931F93182F883051F0A2
:100D2000863041F0893031F0863121F0893111F07F
:100D300082E455C00E94D404882311F084E44FC09B
:100D40000E94E9048823E1F70E943A06823039F4D0
:100D50000E94B40C882319F0163109F416E00E94A1
:100D6000E304082F1817D1F1183019F40E948005F8
:100D70002FC0193159F48930E1F082E06FE140E091
:100D800029E00E94460A063181F40CC0163189F42C
:100D9000893079F082E06FE140E029E00E94460A64
:100DA000093119F483E090E002C089E691E00197EF
:100DB000F1F782E06FE140E0212F0E94460A0830FF
:100DC00019F489E691E002C083E090E00197F1F721
:100DD0000E94E304811711F083E401C080E41F91B5
:100DE0000F910895FF920F931F93DF93CF9300D03D
:100DF0000F92CDB7DEB7F82E8B01809107128230AB
:100E000011F484E430C0882389F0CB016F2D40E0D9
:100E100025E834E10E948324882341F08AE1898314
:100E20001B821A82CE0101960E94830BF7FE02C03C
:100E300082E419C00E94E9048823E1F789E10E9455
:100E40008B060E94E3048931C9F7F80185819681F8
:100E50009093041280930312F2E0FF0EC8016F2DED
:100E60000E94B30980E40F900F900F90CF91DF9113
:100E70001F910F91FF900895DF93CF9300D000D082
:100E80000F92CDB7DEB70E94E3048A838A81813155
:100E900051F08A81863039F08A81813021F08A814F
:100EA000863109F06EC080910712882331F41D82CB
:100EB0001C821B820E94C5091DC0813079F40E94EA
:100EC000C50981E090E09D838C838AE18B83CE010C
:100ED00003960E94830B1D821C820CC085E894E15E
:100EE0000E94DC24882309F47EC08AE18B831D8262
:100EF0001C8242C09091EC1080E02091EB10AC017C
:100F0000420F511D9A015093EC104093EB108091C9
:100F1000F0108F3F41F48091F1108F3F21F4842F26
:100F2000807F09F060C01B8258E821363507E1F068
:100F300088E82236380740F448E02330340761F06F
:100F400020503048C9F40AC088E82336380771F0C9
:100F50002356384C89F40EC085E10DC00E94B40CB4
:100F6000882351F084E107C080E105C08091F4102E
:100F7000813011F487E18B83CE0103960E94830BAD
:100F800032C08A81823049F08A81823131F08A818F
:100F9000893119F08A81893031F5109205121B824E
:100FA0001D821C8282E060EE45E00E94650A898312
:100FB0008981833051F0843018F4823050F403C0BA
:100FC000853039F404C081E103C083E101C082E1CE
:100FD0008B838B81882321F0CE0103960E94830BA3
:100FE00086E10E948B060F900F900F900F900F904C
:100FF000CF91DF9108950E943A06823011F486E184
:1010000008958091E90508950F931F930DEF13E064
:10101000C8010197F1F70E948F090E94D80482E06D
:101020006FE140E023E00E94460AC8010197F1F712
:101030008EE06CE00E94000A89E06FE040E027E06B
:101040000E94460A80E41F910F9108951092640057
:10105000109265000E947A0880E8809361001092E7
:1010600061008DB187608DB98EB183608EB98FEFCD
:1010700087B981B980E090E00E946F0B0E940D104B
:101080000E945D260E9478260E9414690E940C1816
:1010900078940E9478130E94CF0B0E945A260E94D7
:1010A000F3260E940634F4CF9C01F999FECF32BD9D
:1010B00021BDF89A80B508959C01F999FECF1FBA19
:1010C00032BD21BD60BD0FB6F894FA9AF99A0FBEF1
:1010D000089584B1866084B9299A209A289A80E577
:1010E0008CBD81E08DBD08958EBD0DB407FEFDCF92
:1010F0008EB5089508959C01CB01B9012CE538E027
:101100000E94587F0895DF93CF930F92CDB7DEB73B
:10111000FC01362FCA012FB72983F894BF01432F52
:1011200050E00E947B0889818FBF0F90CF91DF91A3
:10113000089524E538E00E943C7F0895DF93CF9323
:101140000F92CDB7DEB7FC01362FCA012FB7298326
:10115000F894BF01432F50E00E94990889818FBF06
:101160000F90CF91DF910895DF92EF92FF920F934E
:101170001F93DF93CF9300D0CDB7DEB78091EA0500
:10118000882311F011E05CC081E08093EA05D090E3
:101190006600F89461E00E94A505E090B100F0902F
:1011A0008100009180001092B10010928100109295
:1011B000800020E030E063E056E04FEF6093B10044
:1011C000509381001092B20010928500109284001A
:1011D00046BB47BBB89BFECF8091840090918500B1
:1011E0009A838983109281001092B10089819A813B
:1011F0008A5F934020F48091660081500AC0898103
:101200009A818650944010F411E00CC080916600E1
:101210008F5F809366002F5F3F4F83E0283E380743
:1012200069F610E081E060E00E94A505E092B1005F
:10123000F092810000938000112311F4D092660097
:10124000812F0F900F90CF91DF911F910F91FF9001
:10125000EF90DF9008951F920F920FB60F920BB68A
:101260000F9211240F931F932F933F934F935F93EC
:101270006F937F938F939F93AF93BF93EF93FF935E
:101280008FE00E942C0A082F182F83FF02C00E94B3
:101290003C0714FF02C00E94CF0C12FF10C0289818
:1012A00080E28EBD0DB407FEFDCF8EB51EBC0DB421
:1012B00007FEFDCF8EB5289A0E9447050AC007FF9A
:1012C00008C08EE00E942C0A682F6F778EE00E9483
:1012D000000AFF91EF91BF91AF919F918F917F9104
:1012E0006F915F914F913F912F911F910F910F90AF
:1012F0000BBE0F900FBE0F901F901895249A259A41
:101300000E948C09EFE6F0E080818062808383E4B4
:1013100080938100B59A08950E94690808950E94FB
:101320007E090E948C09EFE6F0E080818062808374
:1013300083E480938100B59A08951F93CF93DF9340
:10134000EC01162F289880E60E947408812F0E94D5
:10135000740889910E9474081150D9F7289ADF9176
:10136000CF911F910895DF93CF930F92CDB7DEB742
:101370002FB72983F8942C9A2C980E949D09898173
:101380008FBF0F90CF91DF910895EF92FF921F933F
:10139000DF93CF930F92CDB7DEB78FB78983F894E1
:1013A000289880E20E94740880E00E947408182F38
:1013B00083508D37A8F41093EA108BEEE82E80E16D
:1013C000F82E80E00E947408F70181937F0111508C
:1013D000C1F780E00E94740880936A11289A07C0C0
:1013E000289A1092EA1010926A1110926B1189815A
:1013F0008FBF0F90CF91DF911F91FF90EF900895D5
:101400000F931F93DF93CF930F92CDB7DEB7062FC5
:10141000182F106C8FB78983F8942898812F0E9419
:101420007408802F0E947408289A89818FBF1F73C7
:10143000123061F4602F6F71663011F0663121F463
:1014400081E08093C00F02C01092C00F0F90CF9127
:10145000DF911F910F9108951F93DF93CF930F9208
:10146000CDB7DEB7182F10688FB78983F894289806
:10147000812F0E947408812F0E947408289A9981F4
:101480009FBF0F90CF91DF911F910895DF92EF9250
:10149000FF920F931F93D82EF62EE42E022F0E9458
:1014A0002C0A6F2D6095682310E002C0000F111FF9
:1014B000EA94E2F7F0226F298D2D0E94000A1F9115
:1014C0000F91FF90EF90DF900895FF920F931F937D
:1014D000062FF42E0E942C0A082310E002C0159556
:1014E0000795FA94E2F7802F1F910F91FF900895CE
:1014F000FC011182818180830895DC0111969C9109
:101500001197FD01E90FF11D22818C91981711F4BB
:101510002FEF06C0892F8F5F87FD80E011968C9397
:10152000822F0895FC019081818120E0981321E0B1
:10153000822F0895FC018081282F30E08181281BB3
:10154000310937FF02C020583F4F822F0895089578
:1015500081EC9FE00E949A0A089581EC9FE00E942E
:101560009A0A089587E490E10E949A0A089587E410
:1015700090E10E947D0A089590E08091EB05882318
:1015800009F491E09093EB05089580E008950895A3
:1015900004C00E945A260E94F32681EC9FE00E941C
:1015A0009A0A8823B1F381EC9FE00E947D0A089596
:1015B0000F931F93CF93DF93EC01062F18811F5FCA
:1015C00017FF12C010E010C08091C9108823A9F441
:1015D00080910A05813021F080910B05882369F004
:1015E0000E945A260E94F3268981181769F3888180
:1015F000FE01E80FF11D02831883DF91CF911F9147
:101600000F910895682F81E08093C91081EC9FE0CD
:101610000E94D80A1092C9100895682F8091EB0596
:10162000882329F4789487E490E10E94D80A0895E9
:10163000DF92EF92FF920F931F93CF93DF93EC0112
:10164000D42E00E0E62EFF240894E108F1080E9461
:10165000C80A182F802F90E08E159F0534F01D309A
:1016600021F01A3011F0183091F7DD2019F0812F98
:101670000E940D0B1A3029F01D3019F0183089F432
:101680000AC01882802FDF91CF911F910F91FF9098
:10169000EF90DF9008950023D1F201501882219736
:1016A000D6CF19930F5FD3CFCF93DF93EC0102C056
:1016B0000E940D0BFE01219684918823C9F7DF91CA
:1016C000CF910895CF93DF93EC0103C00E940D0BDF
:1016D000219688818823D1F7DF91CF91089581ECFD
:1016E0009FE00E94780A87E490E10E94780A0E94B5
:1016F0006C2708959091CA108091CB1020E0981328
:1017000021E0822F08950F931F93482F192F0091E6
:10171000CA10E02FF0E02091CB10CF0101966AE0D3
:1017200070E00E94728130E082179307B9F0DF0108
:10173000AA0FBB1FAE0FBF1FA453BF4E842F912F04
:101740009C01F90183E001900D928150E1F7802F17
:101750008F5F8A3008F080E08093CA101F910F914C
:101760000895DF93CF930F92CDB7DEB78091CB1062
:101770008983998189818F5F898389818A3008F083
:10178000198289818093CB1023E0929F90011124CC
:1017900024533F4EC9010F90CF91DF91089558C057
:1017A0000E94B10BFC0180818431D1F0853178F445
:1017B000813109F446C0823120F4803109F048C0FB
:1017C0001BC08231D9F1833109F042C034C0863167
:1017D00071F0863150F1873159F18A31C9F534C041
:1017E0008091F6118823A1F50E94BD0C31C00180C3
:1017F000F281E02D09952CC08091F611882341F1EA
:101800008BEE90E10E949A1B2091F4103091F5101C
:101810008091FB119091FC112817390719F40E944F
:10182000A51016C00E94AC2113C00E949F1110C0C9
:101830000E94C81F0DC00E94DE180AC00E94DB185B
:1018400007C00E94E11804C0818192810E94472351
:101850000E947A0B882309F0A3CF08958093021287
:101860000E94100608951F93DF93CF93CDB7DEB784
:1018700028970FB6F894DEBF0FBECDBF182F8FEF9D
:101880009FEF9093FA118093F9119093FC1180933C
:10189000FB111092F6119093FE118093FD1190931D
:1018A00000128093FF11109201121092051281E034
:1018B000809306120E940408109302121F3F19F031
:1018C000812F0E94100681E00E94730688E00E942A
:1018D0008B060E94E20487E164E042E021E00E947E
:1018E000460A86E10E948B0680E090E068E04EEEBA
:1018F00051E10E949E0881E00E9479058FEF9FEFE1
:101900000E9461058FEF9FEF0E946D058CE260EFF2
:1019100044E022E00E94460A8091EE118983809182
:10192000EF118A838091F0118B838091F1118C8368
:101930008091F2118D838091F3118E838091F41147
:101940008F838091F5118887CE0101960E94510501
:101950000E94EC1B28960FB6F894DEBF0FBECDBFD9
:10196000CF91DF911F9108958091EC0508958093A8
:10197000000108958091000108958091EC0588236D
:1019800069F0E091ED05F0E0EE0FFF1FE351FA4F33
:10199000838194818C509E4F94838383089587E044
:1019A0000E942C0AE091ED05F0E0EE0FFF1FE351DD
:1019B000FA4F23813481280F311D3483238387E03C
:1019C00060E00E94000A089583E098E090936E1111
:1019D00080936D118091F71180936F118F5F8093C9
:1019E000F7118FEF9FEF9093711180937011909387
:1019F00073118093721187E08093741188E06DE613
:101A000071E10E94F20608950F931F93DF93CF9325
:101A1000CDB7DEB76A970FB6F894DEBF0FBECDBF65
:101A20008091ED058A31D8F11092EC058EE00E948C
:101A30002C0A682F6F7E8EE00E94000AA6E0B6E0B6
:101A4000FD012FEF3FEF808191818217930708F40A
:101A50009C01329686E0E632F807A9F74BE060E099
:101A60008E010F5F1F4F8D919C91119782179307E5
:101A700029F4F801E60FF11D40836F5F4F5F129666
:101A80004B3189F76623F1F08091EF050E94668162
:101A9000FE01E90FF11D81810E94171813C08F5FAD
:101AA0008093ED050E9410060E94E40C87E060E040
:101AB0000E94000A84E190E064E07DE00E946E0FE5
:101AC0008093EE056A960FB6F894DEBF0FBECDBFC9
:101AD000CF91DF911F910F910895E0EFF5E0119202
:101AE000119286E0E632F807D1F78AE08093ED059F
:101AF0001092EE058FEF0E94330C86E00E948B0659
:101B000088E00E9446068093EF058BE00E94100655
:101B10008EE00E942C0A682F60618EE00E94000A0D
:101B200081E08093EC050E94040D08951F9310E05E
:101B3000809135128F3FE1F011E080913112909148
:101B400032129093FA118093F9112091331230914F
:101B500034123093FE112093FD110E946D05809187
:101B600035120E942E0C809139128F5F80930112E2
:101B7000812F0E9405121F910895909102129F3F9C
:101B8000A9F481E08093EC0586E1E0E3F2E1DF0176
:101B90001D928A95E9F7909335128BE0809302129B
:101BA00080910001803811F080930212409102125E
:101BB0004B3148F4242F30E08091000190E00196F1
:101BC0002817390741F41092EC058FEF8093021229
:101BD0000E94960D0895842F0E942E0C0E94E40C02
:101BE000809102128F5F8093021284E190E06DEB8E
:101BF0007DE00E946E0F0895DF93CF930F92CDB7D3
:101C0000DEB79C01009711F421E030E08FB78983A3
:101C1000F894309366122093651289818FBF0F90DC
:101C2000CF91DF910895DF93CF930F92CDB7DEB7B9
:101C30008FB78983F894209163123091641289815F
:101C40008FBFC9010F90CF91DF910895DF93CF939C
:101C50000F92CDB7DEB78FB78983F89420914612E3
:101C600030914712409148125091491289818FBF9B
:101C7000B901CA010F90CF91DF9108950F931F937F
:101C8000CF93DF938C010E94130EE801C80FD91F78
:101C9000012B29F00E94130EC817D907D9F7DF913D
:101CA000CF911F910F910895909126069F5F09F49F
:101CB00091E0E9E6F2E121E08081891709F420E072
:101CC000359682E1ED3CF807B9F7ECE4F2E180816A
:101CD000891709F420E0359682E1E536F807B9F76F
:101CE000222321F390932606892F0895982FE9E661
:101CF000F2E120E030E08081891751F4F901EE0F24
:101D0000FF1FEE0FFF1FE20FF31FE959FD4E16C034
:101D10002F5F3F4F35962431310569F7ECE4F2E14E
:101D200020E030E08081891769F4F901EE0FFF1F90
:101D3000EE0FFF1FE20FF31FE65BFD4E11821082D4
:101D4000128208952F5F3F4F35962530310551F7A8
:101D50000895DF92EF92FF920F931F93DF93CF933B
:101D600000D00F92CDB7DEB7809146129091471206
:101D7000A0914812B09149120196A11DB11D809306
:101D8000461290934712A0934812B0934912809143
:101D9000010190910201019790930201809301014A
:101DA000892B49F007E612E136E1D32E7E01089433
:101DB000E11CF11C27C088EE93E090930201809310
:101DC00001010AE412E126E1D22E7E010894E11C11
:101DD000F11CF80180819181009769F0019791834E
:101DE0008083892B41F4D982838194819B838A8368
:101DF000C7010E94830B0B5F1F4FF2E103361F07E1
:101E000041F7D0CFF80180819181009769F0019767
:101E100091838083892B41F4D982838194819B8330
:101E20008A83C7010E94830B0B5F1F4FF2E10B3CBB
:101E30001F0741F70F900F900F90CF91DF911F91E7
:101E40000F91FF90EF90DF900895EF92FF920F9324
:101E50001F93DF93CF930F92CDB7DEB7AC010097FE
:101E600019F4FB01099531C0EAE4F2E120E0808138
:101E70009181892B31F5E22EFF248701000F111F7C
:101E8000000F111F0E0D1F1D065B1D4EF801518323
:101E90004083748363830E94540EF80182838FB75A
:101EA0008983F8940E94BA0F89818FBFF701EE0FE2
:101EB000FF1FEE0FFF1FEE0DFF1DE65BFD4E828143
:101EC00005C02F5F3596253091F680E00F90CF91B9
:101ED000DF911F910F91FF90EF9008950F931F9343
:101EE000DF93CF930F92CDB7DEB7AC01009719F413
:101EF000FB01099538C08FB78983F894E7E6F2E1D2
:101F000000E080819181892B51F5202F30E0F9018B
:101F1000EE0FFF1FEE0FFF1FE20FF31FE959FD4EFB
:101F2000CA014115510511F481E090E0918380834D
:101F30008901000F111F000F111F020F131F0959F4
:101F40001D4EF801748363830E94540EF80182834E
:101F50000E94BA0F89818FBFF801828105C00F5F8F
:101F60003596043171F680E00F90CF91DF911F918B
:101F70000F91089580912706882351F410929500BF
:101F80001092940082E08093710081E08093270694
:101F900008951F920F920FB60F920BB60F92112455
:101FA0002F933F934F935F936F937F938F939F9361
:101FB000AF93BF93EF93FF9380916312909164125C
:101FC00001969093641280936312809146129091CF
:101FD0004712A0914812B09149120196A11DB11D5E
:101FE0008093461290934712A0934812B0934912DF
:101FF0000E94A90EFF91EF91BF91AF919F918F9198
:102000007F916F915F914F913F912F910F900BBEF8
:102010000F900FBE0F901F901895E1E9F0E08081BE
:102020008A60808388EE93E0909399008093980073
:1020300080919400909195000E94C17E089508952A
:1020400008950895282F8091FB119091FC11681735
:102050007907E9F08091F6118823C9F07093290679
:102060006093280620932A0610922B06CB010E942B
:102070005121882319F480E090E002C085E090E0CF
:1020800068E470E10E946E0F81E08093051208956C
:102090001F93DF93CF93CDB7DEB760970FB6F89459
:1020A000DEBF0FBECDBF81E698E89A838983809119
:1020B000F8118B838F5F8093F8118091F9119091C3
:1020C000FA119D838C838091FB119091FC1199876B
:1020D00088879D878C8780912806909129069B8709
:1020E0008A8780912A068E870E94FB078F870E942D
:1020F000D104888B80912806909129060E948C1A21
:10210000182F8E831F8290E00E942D1A882331F0B1
:10211000812F90E00E94491A882331F480E1BE01AA
:102120006F5F7F4F0E94F20660960FB6F894DEBF95
:102130000FBECDBFCF91DF911F91089580916C119B
:102140006DE671E10E94F20608958091F81090E02A
:102150008F7790708230910579F0833091051CF46F
:102160000197F9F406C08330910569F00597C9F429
:1021700011C00E94A51208958091F6109091F71059
:102180000E94C31208958091F6109091F7100E945A
:10219000E41808956091EA1060518BEE90E10E947E
:1021A0007D6C0895AF92BF92CF92DF92EF92FF9233
:1021B0000F931F93CF93DF937C01162F6A01B22EEA
:1021C000A02E2091FB113091FC118217930709F486
:1021D00087C08FEFE8168FEFF80609F481C0809171
:1021E000F611882309F47CC081E698E890936E117B
:1021F00080936D118091F81180936F118F5F8093A0
:10220000F8118091F9119091FA11909371118093C6
:1022100070113093751120937411F0927711E09240
:1022200076113093791120937811C7010E945121C2
:10223000082FC7010E94761AEC015E2D4F2D06C0B3
:10224000CE010E94761A5C2F4D2FEC012097C1F72A
:102250005093721140937311B0927A1190E009C0BB
:10226000E92FF0E0E359FE4ED6018D916D0186878E
:102270009F5F9117A8F32091721130917311809193
:10228000FB119091FC112817390751F12F5F3F4F37
:1022900039F1125F10936C1181E080930512C70130
:1022A0000E942D1A882319F0C7010E94491AAA20FA
:1022B00061F0002319F487E090E002C085E090E02F
:1022C0000E943E0E0E949E100BC0002319F487E06E
:1022D00090E002C085E090E06EE970E10E946E0F30
:1022E000DF91CF911F910F91FF90EF90DF90CF90F2
:1022F000BF90AF9008950F93022F25E00E94D21057
:102300000F9108950F93DF93CF9300D0CDB7DEB731
:102310007A83698362E0AE014F5F5F4F26E000E0A1
:102320000E94D2100F900F90CF91DF910F910895DE
:102330000F9321E000E00E94D2100F91089580E0F9
:1023400090E890936E1180936D118091F7118093B6
:102350006F118F5F8093F7118091F9119091FA11AD
:1023600090937111809370118091FB119091FC11E9
:1023700090937311809372118FEF90E49093751185
:102380008093741186E0809376118091011280937E
:1023900077118BE06DE671E10E94F20608950F93CC
:1023A0001F93CF93DF93EC018FEFCF3FD80761F4FA
:1023B00088E00E944606182F00E088E00E9446064A
:1023C000C82FD0E0C02BD12BCE010E946D05D09339
:1023D000FA11C093F91180E090E00E94610510921B
:1023E000FC111092FB11DF91CF911F910F91089575
:1023F00008955F9808955F9808955F9808950895E7
:102400000895089508950895089508958DE792E038
:102410000E94540B89E592E00E94540B08956F923C
:102420007F928F929F92AF92BF92CF92DF92EF9264
:10243000FF920F931F93DF93CF93CDB7DEB7A8978B
:102440000FB6F894DEBF0FBECDBF84E193E00E94CB
:10245000540B2BE8E22E24E0F22E9BEEC92E91E0E5
:10246000D92E4E010894811C911C83E0682E81E0D6
:10247000782ED7018C910E942C0A182FEDB7FEB749
:1024800038970FB6F894FEBF0FBEEDBF3196ADB7CB
:10249000BEB712969C928E92119773826282D582F9
:1024A000C482868317820E94A87FEDB7FEB7389654
:1024B0000FB6F894FEBF0FBEEDBFC4010E94620BC1
:1024C00007E0A12EBB24C501002E02C0959587957B
:1024D0000A94E2F780FD02C080E301C081E30E941C
:1024E0000D0B015080F781E191E00E94620B08948E
:1024F000E11CF11C80E190E0C80ED91E95EBE916B5
:1025000094E0F90609F0B5CF81E193E00E94540B05
:10251000A8960FB6F894DEBF0FBECDBFCF91DF9166
:102520001F910F91FF90EF90DF90CF90BF90AF90F1
:102530009F908F907F906F9008955F9A8AE090E0CF
:1025400069EF71E10E946E0F08958091F81081305B
:1025500091F45F9A8AE090E069EF71E10E946E0F5A
:10256000E091EA10E051F0E0E551FF4E168689EF68
:1025700090E10E94620B089588EE93E06CEB72E1AB
:102580000E946E0F0895EF92FF920F931F937C01AC
:102590005F9A81E090E069EF71E10E946E0F86E43E
:1025A00093E00E94540B00D000D000D0EDB7FEB7EE
:1025B000319608E012E1ADB7BEB712961C930E93A8
:1025C000119784E191E093838283F582E4820E94F3
:1025D000A87F8DB79EB706960FB6F8949EBF0FBE24
:1025E0008DBFC8010E94620B83E0B7010E942210D8
:1025F0001F910F91FF90EF9008955F9A81E090E016
:1026000069EF71E10E946E0F08955F9A89E190E091
:1026100069EF71E10E946E0F08950F931F93882355
:1026200049F080939A06709399066093980681E02A
:1026300080939B0680919A06882309F456C0809166
:102640009B0690E00E94291BFC018081882311F4E5
:1026500090E032C080919A06813069F58CEA92E070
:102660000E94540B00D000D000D0EDB7FEB73196D9
:1026700008E012E1ADB7BEB712961C930E93119706
:1026800084E191E09383828380919B068483158209
:102690000E94A87F8DB79EB706960FB6F8949EBF8E
:1026A0000FBE8DBFC8010E94620B60919B0682E045
:1026B00070E00E94221091E080919B068F5F8093D2
:1026C0009B068A3060F4992319F481E090E002C0FF
:1026D0008AEF90E06EE877E10E946E0F06C01092DC
:1026E00099061092980610929A061F910F910895DC
:1026F0009F92AF92BF92CF92DF92EF92FF920F9391
:102700001F93DF93CF93CDB7DEB7EC970FB6F89456
:10271000DEBF0FBECDBF109297060E94A80A882385
:1027200009F4EAC380910512882309F0E5C30E94E9
:10273000C80A082F843111F410922C0680912C06BF
:10274000882309F11092960680919606E82FF0E012
:10275000E25DF94F00838F5F80939606843640F4E4
:102760000E94A80A882321F00E94C80A082FECCFF3
:102770008091940690919506609196064EE256E0FF
:102780000E949811B9C380912D0687FD47C09927F3
:1027900087FD90958F779070892B09F43FC0802F2B
:1027A0000E940D0B0D3011F00A3081F480919606D5
:1027B000E82FF0E0E25DF94F10828F5F809396067C
:1027C00080912D06806880932D0628C08091960602
:1027D000083039F4E82FF0E0E25DF94F10828150C3
:1027E00006C0E82FF0E0E25DF94F00838F5F809331
:1027F000960680919606843640F080912D0680687A
:1028000080932D061092960677C30E94A80A88230B
:1028100009F472C30E94C80A082FC1CF10912D0677
:1028200017FF102F81E191E00E94620B193649F1E8
:102830001A3684F4103509F43BC3113524F41134ED
:1028400009F050C33CC3133609F4D8C2143609F05A
:1028500049C30FC0133709F4BBC2143724F410372F
:1028600009F040C39DC2143739F0173709F03AC355
:1028700004C30E940F1236C30E94821C0E947B1E5A
:1028800031C32DB73EB72A5030400FB6F8943EBF43
:102890000FBE2DBFEDB7FEB731960EE216E0ADB715
:1028A000BEB712961C930E93119787E191E0938324
:1028B00082838091FB119091FC1195838483809198
:1028C000FD119091FE11978386838091FF11909165
:1028D0000012918780870E94A87FEDB7FEB73A96D5
:1028E0000FB6F894FEBF0FBEEDBFC8010E94620B89
:1028F00000D000D000D0EDB7FEB73196ADB7BEB76F
:1029000012961C930E93119783E491E09383828334
:1029100080910212848315820E94A87FEDB7FEB7D2
:1029200036960FB6F894FEBF0FBEEDBFC8010E94E9
:10293000620B8DE492E00E94540B00D000D000D0D6
:10294000EDB7FEB7319608E012E1ADB7BEB712960B
:102950001C930E9311978FE491E09383828380916F
:10296000F9119091FA11958384830E94A87FEDB7A5
:10297000FEB736960FB6F894FEBF0FBEEDBFC80186
:102980000E94620B81E191E00E94620B0E94E304CD
:10299000082F10E08EE392E00E94540B0115110500
:1029A00019F489E392E04AC00130110519F481E37A
:1029B00092E044C00230110519F489E292E03EC071
:1029C0000630110519F483E292E038C00830110591
:1029D00019F48BE192E032C00930110519F484E159
:1029E00092E02CC00131110519F487E092E026C075
:1029F0000231110519F48AEF91E020C0063111056A
:102A000019F48FEE91E01AC00931110519F484EE22
:102A100091E014C00C31110519F488ED91E00EC05D
:102A20000D31110519F487EC91E008C00E31110544
:102A300019F484EB91E002C08BEA91E00E94540B00
:102A400081E191E00E94620B1091EE11B090EF11C4
:102A5000A090F0119090F1116091F2117091F3112A
:102A60008091F4119091F5112DB73EB72C50304064
:102A70000FB6F8943EBF0FBE2DBFEDB6FEB608945C
:102A8000E11CF11CEEE2CE2EE6E0DE2EADB7BEB7C5
:102A90001296DC92CE92119722E531E0F701338352
:102AA0002283212F3B2D4A2D592D00E20E94EC7DDF
:102AB000C901BA01D70114962C93149715969C93CB
:102AC000159716964C93169717967C93179718960A
:102AD0001C9318971996BC9219971A96AC921A974C
:102AE0001B969C920E94A87FEDB7FEB73C960FB64E
:102AF000F894FEBF0FBEEDBFC6010E94620B80912D
:102B0000F611882319F428E631E002C02EE631E000
:102B10008DB79EB708970FB6F8949EBF0FBE8DBFB6
:102B2000EDB7FEB731960EE216E0ADB7BEB712961E
:102B30001C930E93119783E791E0938382833583EF
:102B4000248380910112868317820E94A87FEDB7AB
:102B5000FEB738960FB6F894FEBF0FBEEDBFC801A2
:102B60000E94620B88E00E94460600D000D000D090
:102B7000EDB7FEB73196ADB7BEB712961C930E9364
:102B800011972DE831E033832283848315820E94DC
:102B9000A87FEDB7FEB736960FB6F894FEBF0FBE0E
:102BA000EDBFC8010E94620B0E943A06833059F0C3
:102BB000873069F0823021F466EEA62EB12C0AC06F
:102BC000A82EBB2407C057EEA52EB12C03C044EDA0
:102BD000A42EB12C83EA91E00E94540B8DE10E9457
:102BE0002C0A2DB73EB7285030400FB6F8943EBFA0
:102BF0000FBE2DBFEDB7FEB731960EE216E0ADB7B2
:102C0000BEB712961C930E9311972BE931E03383D4
:102C10002283B582A482868317820E94A87FEDB7A3
:102C2000FEB738960FB6F894FEBF0FBEEDBFC801D1
:102C30000E94620B00D000D000D0EDB7FEB73196F5
:102C4000ADB7BEB712961C930E93119788EA91E028
:102C50009383828335EBE32E31E0F32EF582E48219
:102C60000E94A87FEDB7FEB736960FB6F894FEBF68
:102C70000FBEEDBFC8010E94620B00D000D000D093
:102C8000EDB7FEB73196ADB7BEB712961C930E9353
:102C9000119789EB91E09383828388E090E095839C
:102CA00084830E94A87FEDB7FEB736960FB6F894DE
:102CB000FEBF0FBEEDBFC8010E94620B00D000D066
:102CC00000D0EDB7FEB73196ADB7BEB712961C93E4
:102CD0000E93119788EC91E093838283F582E482CE
:102CE0000E94A87FEDB7FEB736960FB6F894FEBFE8
:102CF0000FBEEDBFC8010E94620B00D000D000D013
:102D0000EDB7FEB73196ADB7BEB712961C930E93D2
:102D1000119787ED91E09383828388EE91E095830C
:102D200084830E94A87FEDB7FEB736960FB6F8945D
:102D3000FEBF0FBEEDBF8DE891E00E94540B809165
:102D4000D21B8F3F61F08E010F5F1F4FC80162ECF5
:102D50007BE10E945978C8010E94620B04C08FE792
:102D600091E00E94540B8AE691E00E94540B8091FE
:102D7000D21B8F3F61F08E010F5F1F4FC8016BE3C5
:102D80007CE10E945978C8010E94620B04C08CE566
:102D900091E00E94540B89E591E00E94540BA2C07F
:102DA00085E491E00E94540B8EE296E062E341E0FC
:102DB0000E94180B8EE296E00E94CC7E682F8093D2
:102DC00094069093950682E0792F0E9422108AC083
:102DD0008EE291E00E94540B8EE296E062E341E0C5
:102DE0000E94180B8EE296E00E94CC7E909395068E
:102DF0008093940681E080932C0674C08DE191E06D
:102E00000E94540B8EE296E062E341E00E94180BB0
:102E10008EE296E00E94CC7E182F8BE091E00E941B
:102E2000540B8EE296E062E341E00E94180B812F82
:102E30000E94330C8091F9119091FA110E94CF11E8
:102E40008CEE90E00E94540B81E08093F6118EE2AC
:102E500096E00E94CC7E909395068093940600970E
:102E600009F440C00E946D058091940690919506EA
:102E70009093FA118093F91135C089ED90E00E948A
:102E8000540B8EE296E062E341E00E94180B8EE262
:102E900096E00E94CC7E90939506809394060E94C3
:102EA000CF0B80919406909195060E94791B1AC0D1
:102EB0008AEB90E00E94540B0E94BC0A13C088E980
:102EC00090E00E94540B8EE296E062E341E00E94A3
:102ED000180B80912E06803729F481E060E070E0C5
:102EE0000E940D1380912D06882331F48AEF90E023
:102EF00066E072E10E946E0FEC960FB6F894DEBFAA
:102F00000FBECDBFCF91DF911F910F91FF90EF903A
:102F1000DF90CF90BF90AF909F90089580E060E0E9
:102F200070E00E940D1308958FE260E00E94000A95
:102F300082E060E070E00E94221084EF91E064E99A
:102F400077E10E946E0F80939C060895CF92DF92E6
:102F5000EF92FF920F931F93DF93CF93CDB7DEB71E
:102F600028970FB6F894DEBF0FBECDBF6E01089450
:102F7000C11CD11C80E090E068E0A6010E949E0880
:102F8000760186019E01275F3F4FF80180818F3FC8
:102F9000A9F40F5F1F4F02171307B9F727C088E086
:102FA0000E944606F70181937F01E017F107B9F708
:102FB00080E090E068E0A6010E94830880E190E054
:102FC00062E0A6010E949E08F601808191818F5FD8
:102FD0009F4F99F484E190E0F6019183808380E132
:102FE00090E062E0A6010E94830807C080E00E9492
:102FF000040886E00E948B06D2CF28960FB6F8947C
:10300000DEBF0FBECDBFCF91DF911F910F91FF901B
:10301000EF90DF90CF9008950E9405130E94A617AD
:103020000E946D0D8CEB92E00E94540B0895FF926C
:103030000F931F93F82E0E94330C8FEF9FEF0E9487
:10304000CF118AEC92E00E94540B00D000D000D047
:10305000EDB7FEB7319608E012E1ADB7BEB71296F4
:103060001C930E93119784E191E093838283F48201
:1030700015820E94A87F8DB79EB706960FB6F8946A
:103080009EBF0FBE8DBFC8010E94620B81E080937E
:10309000F6116091FB117091FC118091F9119091E2
:1030A000FA110E9475681F910F91FF900895EF9299
:1030B000FF920F931F938FEF92E00E94540B00D06A
:1030C00000D000D0EDB7FEB7319608E012E1ADB701
:1030D000BEB712961C930E9311978FE491E09383E1
:1030E00082838091331290913412958384830E945D
:1030F000A87F8DB79EB706960FB6F8949EBF0FBEF9
:103100008DBFC8010E94620B87EF92E00E94540BB2
:1031100000D000D000D0EDB7FEB73196ADB7BEB746
:1031200012961C930E931197A4E1EA2EA1E0FA2EB9
:10313000F382E28280913512848315820E94A87FF7
:103140008DB79EB706960FB6F8949EBF0FBE8DBF83
:10315000C8010E94620B8DEE92E00E94540B00D0D9
:1031600000D000D0EDB7FEB73196ADB7BEB712961E
:103170001C930E931197F382E2828091391284831B
:1031800015820E94A87F8DB79EB706960FB6F89459
:103190009EBF0FBE8DBFC8010E94620B809133128B
:1031A00090913412609135120E9468191F910F910D
:1031B000FF90EF9008950E94672208950E94672271
:1031C00008950E9464220895EF92FF920F931F9337
:1031D0007C0180E393E00E94540B00D000D000D02B
:1031E000EDB7FEB7319608E012E1ADB7BEB7129663
:1031F0001C930E9311978FE491E093838283F58261
:10320000E4820E94A87F8DB79EB706960FB6F89409
:103210009EBF0FBE8DBFC8010E94620B8AE293E081
:103220000E94540B0E94D10400D000D000D0EDB712
:10323000FEB73196ADB7BEB712961C930E93119799
:10324000B4E1EB2EB1E0FB2EF382E282848315829F
:103250000E94A87F8DB79EB706960FB6F8949EBFC2
:103260000FBE8DBFC8010E94620B83E293E00E94F3
:10327000540B0E94FB0700D000D000D0EDB7FEB782
:103280003196ADB7BEB712961C930E931197F38289
:10329000E282848315820E94A87F8DB79EB706962E
:1032A0000FB6F8949EBF0FBE8DBFC8010E94620B7F
:1032B00081E191E00E94620B5F9A8AE090E069EF01
:1032C00071E10E946E0F1F910F91FF90EF90089592
:1032D00008950895EF92FF920F931F93CF93DF937A
:1032E000E82EEB018A0181E08093A106F880B98184
:1032F000AA817B816C813D812E819F81E0EBF6E08C
:1033000041E050E080818F15A9F481818B1791F401
:1033100082818A1779F48381871761F48481861703
:1033200049F48581831731F48681821719F48781E6
:103330008917A1F04F5F5F4F3E964A30510511F754
:10334000EFEAF6E041E050E08081882351F04F5FE2
:103350005F4F3E964A305105B9F735C04A305105A6
:1033600090F5CA01880F991FBC0123E0660F771FF3
:103370002A95E1F7681B790B9B012F55394FF9010D
:10338000E1928881D90111968C931197898181836B
:103390008A8182838B8183838C8184838D818583E1
:1033A0008E8186838F8187831A961C930E9319973B
:1033B0001C961C921E921B97DB01A255B94F8C9153
:1033C0008E7F8C9302C04FEF5FEFCA01DF91CF91E8
:1033D0001F910F91FF90EF900895DC01EFEAF6E066
:1033E00021E030E08081882371F191818C919817E0
:1033F00051F5928111968C911197981721F593812F
:1034000012968C9112979817F1F4948113968C91DF
:1034100013979817C1F4958114968C911497981767
:1034200091F4968115968C911597981761F4978170
:1034300016968C911697981731F4908517968C9163
:103440001797981741F02F5F3F4F3E962A3031056E
:1034500049F62FEF3FEFC90108958A309105B0F486
:10346000880F991FFC0143E0EE0FFF1F4A95E1F71B
:10347000E81BF90BEF55F94F8081882339F020E0E4
:1034800081859285892B19F421E001C020E0822FEB
:1034900008958A30910510F080E00895880F991FF3
:1034A000FC0163E0EE0FFF1F6A95E1F7E81BF90BE3
:1034B000E255F94F80818695817009F081E0089589
:1034C00008958A30910588F4880F991FFC01A3E0C4
:1034D000EE0FFF1FAA95E1F7E81BF90BEF55F94F27
:1034E0001082128611861486138608958A309105FB
:1034F00018F020E030E00EC0880F991FFC0123E097
:10350000EE0FFF1F2A95E1F7E81BF90BEF55F94F76
:1035100021853285C90108950F931F93CF93DF93BF
:10352000EC018A309105D0F4CE01880F991F8C01EF
:1035300043E0000F111F4A95E1F7081B190B0F55C7
:10354000194FF8018081882349F0CE010E942D1A7D
:10355000882331F4F801C185D285E6CFC0E0D0E000
:10356000CE01DF91CF911F910F910895AC01EFEA49
:10357000F6E021E030E08081882329F08185928582
:103580008417950741F02F5F3F4F3E962A30310553
:1035900091F720E030E0C90108959C018A3091053F
:1035A00060F5880F991FFC01A3E0EE0FFF1FAA959D
:1035B000E1F7E81BF90BEF55F94F418552852F5F75
:1035C0003F4FC901880F991FFC0163E0EE0FFF1FF9
:1035D0006A95E1F7E81BF90BEF55F94F0BC08081B5
:1035E000882329F0818592858417950741F02F5F04
:1035F0003F4F3E962A30310591F720E030E0C90177
:1036000008958A30910518F020E030E00EC0880F50
:10361000991FFC0123E0EE0FFF1F2A95E1F7E81B3D
:10362000F90BEF55F94F23853485C90108958A3088
:10363000910570F4880F991FFC0143E0EE0FFF1F06
:103640004A95E1F7E81BF90BEF55F94F748763874B
:1036500008958A30910518F020E030E00CC0880F02
:10366000991F9C0163E0220F331F6A95E1F7281B25
:10367000390B2F55394FC9010895CF93DF93EC01D2
:103680000E942D1A882399F0CA30D10580F4CE010A
:10369000880F991FFC01A3E0EE0FFF1FAA95E1F729
:1036A000E81BF90BE255F94F80818E7F8083DF9113
:1036B000CF91089580E090E0089580E090E0089533
:1036C00021E0880F991FFC0133E0EE0FFF1F3A95B0
:1036D000E1F7E81BF90BEF55F94F8081882331F0B2
:1036E00081859285009719F02F5FEBCF20E0822F24
:1036F0000895CF93DF93EC010E94761A0097A1F40E
:10370000CA30D105A0F4CE01880F991FFC0153E007
:10371000EE0FFF1F5A95E1F7E81BF90BE255F94F41
:1037200080818160808303C0BE010E948211DF918D
:10373000CF910895EF92FF920F931F93CF93DF9352
:103740007C01DC011B960D911C911C97C8010E9405
:103750002D1A8823D1F10A301105B8F5C801880F58
:10376000991FFC01A3E0EE0FFF1FAA95E1F7E81BEC
:10377000F90BE255F94F90E0D7011D968C9187FD2A
:1037800091E0990F80818D7F892B8083C801880FFC
:10379000991FEC0173E0CC0FDD1F7A95E1F7C81B90
:1037A000D90BC255D94F888180FF08C0C80160E09D
:1037B00070E00E94821188818E7F8883C8010E94F8
:1037C0002110F70185858F778587DF91CF911F9134
:1037D0000F91FF90EF9008958CE8E1EAF6E0DF01A9
:1037E0001D928A95E9F7089590939E0680939D0611
:1037F0007093A00660939F0680EA90E066E07CE10B
:103800000E946E0F81E080930512089580919D06BD
:1038100090919E060E945121882319F480E090E047
:1038200002C085E090E06AED7DE10E946E0F089590
:10383000DF93CF930F92CDB7DEB79C01AB018A30F7
:10384000910508F05AC0880F991FFC01A3E0EE0F04
:10385000FF1FAA95E1F7E81BF90BEF55F94F80819F
:10386000882331F48EEF93E00E94540B80E046C031
:10387000232B09F442C02185328521153105E9F158
:1038800081E089836115710519F4A0E0B0E002C000
:10389000DB011A96C901880F991FFC0163E0EE0F46
:1038A000FF1F6A95E1F7E81BF90BEF55F94F80818F
:1038B000882321F189818F5F898381859285892B76
:1038C00041F44115510519F0FA01368325838981A8
:1038D00015C0109711F02D933D93C901880F991FC2
:1038E000FC0123E0EE0FFF1F2A95E1F7E81BF90B1F
:1038F000EF55F94F21853285CDCF81E00F90CF91E3
:10390000DF9108952F923F924F925F926F927F9234
:103910008F929F92AF92BF92CF92DF92EF92FF92DF
:103920000F931F93DF93CF93CDB7DEB7E6970FB614
:10393000F894DEBF0FBECDBF8091DF049091E0040C
:10394000A091E104B091E20489839A83AB83BC83A4
:103950008EEE93E00E94540B8FEA882E86E0982E1C
:1039600001E0602E712C15E0212E312C2C0E3D1E15
:103970002E010894411C511CF4012081222309F4DA
:1039800071C01181D280C380B480658176818781C6
:1039900090854DB75EB7465150400FB6F8945EBF64
:1039A0000FBE4DBFEDB6FEB60894E11CF11CEDB79D
:1039B000FEB73282218245EB54E0F7015383428304
:1039C000F201E20FF11D2081332727FD3095F70129
:1039D0003583248377826682F40121853285220F24
:1039E000331FF901A3E0EE0FFF1FAA95E1F7E21BD9
:1039F000F30BEF55F94F2081F201E20FF11D208109
:103A0000332727FD3095F70131872087F401218581
:103A10003285F70133872287F40123853485F70146
:103A200035872487212F3D2D4C2D5B2D00E20E94F0
:103A3000EC7DC901BA01F70126879787408B718B0E
:103A4000128BD38AC48AB58A0E94A87F4DB75EB70D
:103A50004A5E5F4F0FB6F8945EBF0FBE4DBFC10107
:103A60000E94620B8EE090E0880E991E0894611C03
:103A7000711C9DE2891697E0990609F07DCF8DEDC6
:103A800093E00E94540B00E010E0EE2455E0852EF8
:103A9000912C8C0E9D1E47EDA42E44E0B42E3E01C9
:103AA0000894611C711C01C08601EDB7FEB7389700
:103AB0000FB6F894FEBF0FBEEDBFADB7BEB71196FF
:103AC000928281821396BC92AE921297C801880F9F
:103AD000991FFC0123E0EE0FFF1F2A95E1F7E81B79
:103AE000F90BEF55F94F8081F301E80FF11D80814B
:103AF000992787FD909515969C938E93149717960A
:103B00001C930E9316970E94A87F4DB75EB7485F2F
:103B10005F4F0FB6F8945EBF0FBE4DBFC4010E9449
:103B2000620BC8010E94B61A009719F0E3948C0149
:103B3000BCCFC8010E94CD1A6C01009771F08AEDCC
:103B400093E00E94540B10E005C085ED93E00E94C5
:103B5000540B1F5F1E15C8F3A7CFC801880F991F0C
:103B6000FC0113E0EE0FFF1F1A95E1F7E81BF90BBC
:103B7000EF55F94F018512850115110511F0EA94F1
:103B8000D8CFE6960FB6F894DEBF0FBECDBFCF916B
:103B9000DF911F910F91FF90EF90DF90CF90BF903A
:103BA000AF909F908F907F906F905F904F903F90DD
:103BB0002F900895EF92FF920F931F93DF93CF936F
:103BC000CDB7DEB760970FB6F894DEBF0FBECDBF9E
:103BD0008EE693E00E94540B00D000D000D0EDB7E9
:103BE000FEB7319608E012E1ADB7BEB712961C934E
:103BF0000E93119794EEE92E94E0F92EF382E2826F
:103C000080919F069091A006958384830E94A87F4F
:103C10008DB79EB706960FB6F8949EBF0FBE8DBFA8
:103C2000C8010E94620B80E693E00E94540B00D012
:103C300000D000D0EDB7FEB73196ADB7BEB7129643
:103C40001C930E931197F382E28280919D069091CE
:103C50009E06958384830E94A87F8DB79EB70696A3
:103C60000FB6F8949EBF0FBE8DBFC8010E94620BB5
:103C700081E698E89A8389838091F8118B838F5F1E
:103C80008093F8118091F9119091FA119D838C83A2
:103C900000919D0610919E06C8010E948C1AAC01ED
:103CA00020919F063091A006009791F0388B2F87C6
:103CB00084E08E871D861C861B870A8719861886D6
:103CC0005F834E8380E1BE016F5F7F4F0E94F206EB
:103CD00060960FB6F894DEBF0FBECDBFCF91DF91D7
:103CE0001F910F91FF90EF90089586E16DE671E1CD
:103CF0000E94F20608953F924F925F926F927F92D8
:103D00008F929F92AF92BF92CF92DF92EF92FF92EB
:103D10000F931F93DF93CF93CDB7DEB7C255D0403B
:103D20000FB6F894DEBF0FBECDBF80911B1C882359
:103D3000C9F180911D1C8823A9F18091301C8F3F0F
:103D400011F4AA240DC0DE011196E0E2FCE180E14D
:103D500001900D928150E1F71F86188AAA24A3943E
:103D600080914B1C8F3F09F468C02A2D30E0C901B7
:103D7000A4E0880F991FAA95E1F7FE013196E80F9C
:103D8000F91FABE3BCE180E10D9001928150E1F7B6
:103D9000F4E0220F331FFA95E1F7FE013196E20FAE
:103DA000F31F48C04091A71C4D7F5091A81C8091E3
:103DB000B71B8F3F11F4AA2415C0DE011196E7EA64
:103DC000FBE180E101900D928150E1F749875A872C
:103DD0001B868FEF8C878EEF8D871E861F86188A35
:103DE000AA24A3948091D21B8F3F39F12A2D30E071
:103DF000C901E4E0880F991FEA95E1F7FE013196C9
:103E0000E80FF91FA2ECBBE180E10D900192815017
:103E1000E1F774E0220F331F7A95E1F7FE01319646
:103E2000E20FF31F4087518712868FEF83878EEF53
:103E30008487158616861786A39482EA93E00E94EB
:103E4000540B6FEA862E66E0962E51E0652E712C9B
:103E500041E2442E512C4C0E5D1E362CF401808123
:103E6000882309F46FC01181D280C380B48065813A
:103E70007681878190852DB73EB72E5030400FB6A2
:103E8000F8943EBF0FBE2DBFEDB6FEB60894E11C00
:103E9000F11CEDB7FEB75282418227EE34E0F70104
:103EA00033832283212F3D2D4C2D5B2D00E20E9478
:103EB000EC7DC901BA01F70124839583468377839A
:103EC0001087D186C286B386758664860E94A87FD5
:103ED0002DB73EB7225F3F4F0FB6F8943EBF0FBEDF
:103EE0002DBFC2010E94620B30E1C32ED12CCC0E3B
:103EF000DD1E00E010E024C0F6013082B80124E0AD
:103F0000660F771F2A95E1F721E030E02C0F3D1F67
:103F1000620F731FC2010E945978002321F083E8C9
:103F200093E00E94540BC2010E94620B80E893E070
:103F30000E94540B0F5F1F4F80E190E0C80ED91E06
:103F40000A15D0F2EEE0F0E08E0E9F1E0894611C80
:103F5000711CFDE28F16F7E09F0609F07ECFCE5A66
:103F6000DF4F0FB6F894DEBF0FBECDBFCF91DF910C
:103F70001F910F91FF90EF90DF90CF90BF90AF9087
:103F80009F908F907F906F905F904F903F9008959B
:103F9000EF92FF920F931F93CF93DF939091EC10CA
:103FA00080E02091EB10820F911D28E88336920764
:103FB00009F0A4C087EF90E10E94ED19BC018FEFDA
:103FC0006F3F780719F1CB01880F991FFC0123E09F
:103FD000EE0FFF1F2A95E1F7E81BF90BEF55F94F9C
:103FE0008081882399F0218532852115310521F4BE
:103FF000CB010E94611A0AC08091F5109091F610D1
:104000008217930719F0C9010E94F41B8091F510E3
:104010009091F6100E945121182F4091F510509167
:10402000F6108091FF1067EF70E10E946A19EC01B1
:10403000909382118093811183E698E890936E119A
:1040400080936D118091F81180936F118F5F809331
:10405000F8118091F9119091FA1190937111809358
:1040600070118091F2109091F310909373118093DE
:1040700072118091FB119091FC11909375118093B6
:10408000741182E0809376118091F5109091F61072
:1040900090937811809377118091F7108093791124
:1040A0008091F81080937A118091F91080937B11A0
:1040B0008091FA1080937C118091FB1080937D1188
:1040C0008091FC1080937E118091FD1080937F1170
:1040D0008091FE1080938011112319F480E090E00C
:1040E00002C085E090E065E77EE10E946E0F81E00E
:1040F00080930512CE010E949D1277C08356984C82
:1041000019F0C0E0D0E071C082EF90E10E94ED199B
:10411000BC01BFEF8F3F9B07B1F0880F991FFC01D7
:1041200013E0EE0FFF1F1A95E1F7E81BF90BEF55AF
:10413000F94F81859285009721F4CB010E94611A85
:1041400002C00E94F41B8091FD1062EF70E140E01C
:1041500050E00E946A19EC0183E69CE890936E118E
:1041600080936D118091F81180936F118F5F809310
:10417000F8118091F9119091FA1190937111809337
:1041800070118091F210809372118091F3108093DE
:1041900073118091F410809374118091F5108093C5
:1041A00075118091F610809376118091F7108093AD
:1041B00077118091F810809378118091F910809395
:1041C00079118091FB119091FC1190937B11809358
:1041D0007A1182E080937C11D0937E11C0937D117F
:1041E00082E16DE671E10E94F2068FE194E00E94A7
:1041F000540B00D000D000D0EDB7FEB7319608E0E8
:1042000012E1ADB7BEB712961C930E931197B3E0AF
:10421000EB2EB5E0FB2EF382E282D583C4830E94AD
:10422000A87F8DB79EB706960FB6F8949EBF0FBEB7
:104230008DBFC8010E94620B86E194E00E94540B7E
:10424000CE010E94601B00D000D000D0EDB7FEB7B9
:104250003196ADB7BEB712961C930E931197F382A9
:10426000E282848315820E94A87F8DB79EB706964E
:104270000FB6F8949EBF0FBE8DBFC8010E94620B9F
:1042800083E194E00E94540BCE010E940312DF915F
:10429000CF911F910F91FF90EF9008950895089589
:1042A0000895FF920F931F93DF93CF93CDB7DEB79F
:1042B000C258D0400FB6F894DEBF0FBECDBF8E01FE
:1042C0000D5F1F4FB8010E94181CF82E82E08F1559
:1042D00078F583E698E89C838B838091F811F80148
:1042E00082838F5F8093F8118091F9119091FA1178
:1042F00094838383108617828BEB818785819681D7
:104300009A83898389819A810E94011BF8016285C1
:1043100073858617970761F089819A810E94171B20
:10432000FF0C8F2D8A5FB8010E94F20681E001C068
:1043300080E0CE57DF4F0FB6F894DEBF0FBECDBF83
:10434000CF91DF911F910F91FF9008958FE76DE658
:1043500071E10E94F2060895ACE6B1E1EAEEF0E107
:1043600082E801900D928150E1F75F9A8AE090E037
:1043700069EF71E10E946E0F809176119091771133
:104380000E942D1A2091761130917711882309F11E
:104390008091F81180936F118F5F8093F8113093A3
:1043A0007311209372118091FB119091FC119093E5
:1043B0007511809374118AE494E00E94540B8091EB
:1043C0007611909177110E94491A882351F141E0AA
:1043D00029C08091F81180936F118F5F8093F8113D
:1043E000C9010E948C1A90937311809372111092DC
:1043F00075111092741182E394E00E94540B809125
:104400007611909177110E945121882351F085E017
:1044100090E066EA71E20E946E0F81E080930512DF
:10442000089540E0209172113091731180917611BE
:1044300090917711442341F040916C1142506DE608
:1044400071E10E94201008952F5F3F4F39F0809155
:104450006C1182506DE671E10E94F2060895089594
:10446000089580E090E0089508950895CF93DF9334
:10447000EC0181E080932D07CA30D10510F5CE0103
:10448000880F991FDC01E3E0AA0FBB1FEA95E1F753
:10449000A80FB91FA353BD4EFB0180E101900D92FF
:1044A0008150E1F7FE01EE0FFF1FCF0123E0880FDF
:1044B000991F2A95E1F7E80FF91FE353FD4E518B41
:1044C000408BDF91CF91089510922D070895809130
:1044D0002D07882331F080910312909104120E94DD
:1044E000791B10922D070895DF93CF9300D0CDB79D
:1044F000DEB79A838983482F5A81FA01EE0FFF1F96
:10450000CF0123E0880F991F2A95E1F7E80FF91FE3
:10451000E353FD4E208931892115310509F46BC023
:104520001092C4151092C31580E680934016109225
:1045300043161092421689E0809344161092451655
:1045400080E48093471681E180934616CA01880F64
:10455000991FFC01A3E0EE0FFF1FAA95E1F7E80FFA
:10456000F91FA8E4B6E1E353FD4E80E101900D92FE
:104570008150E1F7A8E5B6E1EBE3FCE180E10190D1
:104580000D928150E1F78A8180936616898180932C
:10459000671680EF92EB90936B1680936A163093B8
:1045A00068162093691680E099E090936D168093C9
:1045B0006C1687E78093701610926F1610926E1625
:1045C0000E94F73C8095909590936F1680936E169D
:1045D000892B31F48FEF9FEF90936F1680936E16B7
:1045E00081E390E09093C4158093C31581E080939C
:1045F000CA1C0E9459730F900F90CF91DF910895BC
:104600000F931F93182F092FE82FF92FEE0FFF1F7D
:10461000CF01A3E0880F991FAA95E1F7E80FF91FD2
:10462000E353FD4E208931892115310569F19091BF
:104630006A1680916B168217930731F5612F702FE0
:10464000660F771FCB01E3E0880F991FEA95E1F72A
:10465000680F791F63537D4E88E596E140E150E095
:104660000E940D7F009781F4E12FF02FEE0FFF1FC6
:10467000CF0143E0880F991F4A95E1F7E80FF91F32
:10468000E353FD4E118A108A1F910F9108950F93E5
:104690001F93DF93CF930F92CDB7DEB78C0180913C
:1046A0000712823041F50115110569F48BEE90E196
:1046B000BE016F5F7F4F45E854E10E94182480934C
:1046C000EA1001E010E080910D058823A1F08091AF
:1046D000EB10813681F48091EC10883861F4809180
:1046E000F8108F77853039F46091EA1060518BEEC5
:1046F00090E10E947D6C80914205809340168091EC
:104700004305809341168091440580934216809121
:104710004505809343168091460580934416809109
:10472000470580934516EBECF5E1A6E4B6E18191EF
:104730008D9385E1E13DF807D1F780E880934C1631
:104740008AE980934D168EE090E09093C415809393
:10475000C315012B61F48EE496E1BE016F5F7F4FBC
:1047600045E854E10E94182490E00E9613C02EE410
:1047700036E14091EA10EBEEF0E1C901BF0150E0F3
:104780000E941A7F2091EA108091C3159091C41560
:10479000820F911D9093C4158093C3156091C3152A
:1047A0007091C41580E496E141E00E94EF331092CD
:1047B000C4151092C3150F90CF91DF911F910F91E7
:1047C00008951F93182F8093071285E893E160E006
:1047D00071E045E854E10E94F623123011F486E0BE
:1047E00001C086E10E948B061F910895FA01918312
:1047F00080837583648397838683918780876150E4
:104800007040860F971F938382830895FC01408533
:104810005185868197814817590728F0481B590B05
:104820002481358101C09C01241B350BC9010895E9
:10483000CF93DF93EC01DA011696ED91FC91179777
:10484000508157FD02C0452F23C08D919C91119737
:1048500017969C938E93169719969C938E93189700
:1048600080E04EC0019617969C938E93169728175A
:10487000390738F48D919C91119717969C938E93DC
:1048800016971696ED91FC91179780818993415068
:1048900016968D919C91179712962D913C91139796
:1048A000442301F7019617969C938E931697281729
:1048B000390738F48D919C91119717969C938E939C
:1048C00016971696ED91FC9117978081FB018083D6
:1048D00016968D919C911797019617969C938E939F
:1048E000169712962D913C9113972817390738F493
:1048F0008D919C91119717969C938E931697852F67
:10490000DF91CF910895EF92FF920F931F93CF9372
:10491000DF938C01F62EE42EE901C9010E940624E2
:104920002F2D30E02E5F3F4F8217930710F460E089
:104930003BC0E885F985F08288859985019699873D
:1049400088872A813B812817390720F4888199813B
:10495000998788874F2D14C0D8018C9180838885D2
:1049600099850196998788872A813B81281739077D
:1049700020F488819981998788870F5F1F4F415064
:10498000E885F985442341F7E08288859985019679
:10499000998788872A813B812817390720F48881E5
:1049A0009981998788876F2D862FDF91CF911F91ED
:1049B0000F91FF90EF900895FF920F931F93CF9365
:1049C000DF93EC01289880E20E94740880E00E9446
:1049D0007408F82E83508D3708F04BC0CE010E942A
:1049E00006242F2D30E02E5F3F4F8217930708F4E7
:1049F00040C0E885F985F082888599850196998778
:104A000088872A813B812817390720F4888199817A
:104A1000998788870F2D80E00E947408E885F985C2
:104A20008083888599850196998788872A813B812B
:104A30002817390720F48881998199878887015040
:104A400051F70885198580E00E947408F801808379
:104A5000888599850196998788872A813B812817BF
:104A6000390720F48881998199878887289A8F2D22
:104A700002C0289A80E0DF91CF911F910F91FF90A3
:104A80000895089582E102C00E94E30481518230BA
:104A9000D8F30E9490058AB18F758AB98DB18F7352
:104AA0008DB980917A008F7780937A0080B7806883
:104AB00080BF8FEF809364008FE7809365007894C8
:104AC00083B7817F846083BF83B7816083BF88950C
:104AD00083B78E7F83BF10926400109265008AB105
:104AE000806A8AB98DB1806C8DB90E948C090E9450
:104AF000C10589E00E948B0608951F920F920FB6A0
:104B00000F920BB60F9211242F933F934F935F9305
:104B10006F937F938F939F93AF93BF93EF93FF9385
:104B20008091DA0080FF31C08091D80080FF2DC0D5
:104B30008EEF8093DA008091D90080FF19C081E068
:104B400080939A1480912E0790912F078260909302
:104B50002F0780932E078091E20088608093E20007
:104B60000E94F5278091E0008E7F8093E0000DC0C9
:104B700010929A1410929F1480912E0790912F07F3
:104B8000846090932F0780932E078091E10082FF2D
:104B900009C08091E20082FF05C08BEF8093E100A5
:104BA0000E9489268091E10080FF1FC08091E20071
:104BB00080FF1BC08EEF8093E1008091E200806156
:104BC0008093E2008FEE8093E1008091D8008062B4
:104BD0008093D80080912E0790912F078062909348
:104BE0002F0780932E070E9442258091E10084FFC9
:104BF0001AC08091E20084FF16C08091D8008F7D9A
:104C00008093D8008FEE8093E1008091E2008F7E48
:104C10008093E20080912E0790912F0780649093FB
:104C20002F0780932E078091E10085FF1AC08091A5
:104C3000E20085FF16C08091E2008F7E8093E20043
:104C40008FED8093E1008091E2008F7D8093E20000
:104C500080912E0790912F07806890932F07809363
:104C60002E078091E10083FF12C08091E20083FF54
:104C70000EC087EF8093E1000E94652B80912E0784
:104C800090912F07916090932F0780932E07FF91AB
:104C9000EF91BF91AF919F918F917F916F915F91B4
:104CA0004F913F912F910F900BBE0F900FBE0F9021
:104CB0001F9018950E9411280895E7EDF0E080817B
:104CC0008160808380818F7B808380818068808306
:104CD0000E94E42708959C01F999FECF1FBA32BDC6
:104CE00021BD60BD0FB6F894FA9AF99A0FBE0895E7
:104CF0008AB1806A8AB98DB1806C8DB95F985D9AEE
:104D00008EB1806C8EB9E2EEF0E0808184608083A9
:104D10000895809196148F5F8093961408957698E5
:104D200088EC8093971408950F931F9380910A0540
:104D3000882311F484E003C0833009F051C08093CC
:104D4000E9008091E80085FF4BC01091A314112366
:104D5000A9F0212F90E0E92FF0E0EC55FB4E808187
:104D60008093F1009F5F2150B1F71092A31403C00C
:104D70001092F1001F5F1032D8F321C00E94B20AD6
:104D8000882371F180910B05882331F181E08093B4
:104D9000F10000E00E94B20A882339F0002331F4C8
:104DA0000E94B70A8093F10003C001E01092F10065
:104DB0001F5F1F3179F7769888EC80939714809164
:104DC000E8008E7F8093E8008091E8008F778093E1
:104DD000E80006C00E94B70A0E94B20A8823D1F7F1
:104DE0001F910F9108950F931F938091971488231B
:104DF00021F081508093971401C0769A80919F147E
:104E00008823E9F180910A058130C9F580919614D3
:104E10008233C8F0809198148823A9F010929614D8
:104E20000E94BC2710C00093E9000E94B22788238B
:104E300009F44FC07698109397140E94B70A90E037
:104E40000E94C72702C005E018EC0E94B20A88231E
:104E500051F70E94AD0A8F3790F40E947127882382
:104E600049F40DC07698109397140E9493270E94DE
:104E7000020B01C018EC80919914882399F7809156
:104E80009F14882331F180910A05882311F58091C0
:104E900039078823E1F05F985D9A8EB1806C8EB9F6
:104EA0008091E00081608093E0008FE090E065E316
:104EB0000E946B262CE088E190E00FB6F894A8954C
:104EC000809360000FBE20936000F894FFCF0E9493
:104ED00094261F910F91089510929814109299148E
:104EE0000895809199148823C9F486E08093E9009D
:104EF0008091E80082FF12C08091F3008091F2005F
:104F000080939914882351F48091E8008B7F8093DB
:104F1000E8008091E8008F778093E80080919914F1
:104F2000811181E0089586E08093E90080919914D1
:104F3000882319F40E947127FBCF9091F100809192
:104F40009914815080939914882351F48091E8003A
:104F50008B7F8093E8008091E8008F778093E80052
:104F6000892F08958091E80090E025E09695879537
:104F70002A95E1F78170089585E08093E900E8EED5
:104F8000F0E080818F7780831092981408950F93BA
:104F90001F93182F092F85E08093E9000E94B22704
:104FA0008823E1F31093F100809198148F5F809330
:104FB00098148091E80085FD02C00E94BC27812FD3
:104FC000902F1F910F9108957894E8EDF0E0808183
:104FD0008F76808380818069808380818F7B8083CE
:104FE000808181608083789408958EE089BD09B4C2
:104FF00000FEFDCF8091D8008F7D8093D8008091F6
:10500000E20081608093E2008091E20088608093FA
:10501000E2000E94652B8091E0008E7F8093E0008B
:1050200008958091D90080FF09C080919A14882347
:1050300029F481E080939A140E94F52780912E072D
:1050400090912F0790FF10C080912E0790912F070D
:105050009E7F90932F0780932E0781E08093EA0034
:105060001092EA0010929F141092E9008091E800DB
:1050700083FF02C00E949D2A809151078823F9F086
:1050800083E08093E9008091E80085FF18C081E00B
:105090008093F1001092F1001092F1001092F10053
:1050A0001092F1001092F1001092F1001092F100B4
:1050B0008091E8008F778093E8001092510708955F
:1050C0009091E3008091F1008F779078892B809305
:1050D000E3008091E800877F8093E8008091E800FA
:1050E0008E7F8093E8008091E80080FFFCCF809164
:1050F000E30080688093E3000895DF93CF9300D0AE
:10510000CDB7DEB78091E800877F8093E80080917B
:105110009F148093F1008091E8008E7F8093E800D7
:105120008091E8008F778093E8008FEF9FEF03C0B6
:1051300089819A8101979A83898389819A81892BB0
:1051400021F08091E80082FFF3CF8091E8008B7F0F
:105150008093E8008091E8008F778093E8000F90BB
:105160000F90CF91DF910895DF93CF9300D0CDB70B
:10517000DEB78091F1008091F100E091F100809123
:105180003807813821F0823851F08038B1F48091AD
:10519000E800877F8093E8001092F10017C08091AB
:1051A000E800877F8093E800F0E0EF77F070EF5C35
:1051B000F84F80818093F10009C08091EB008062FC
:1051C0008093EB008091E800877F1FC01092F10070
:1051D0008091E8008E7F8093E8008FEF9FEF03C0FF
:1051E00089819A8101979A83898389819A81892B00
:1051F00021F08091E80082FFF3CF8091E8008B7F5F
:105200008093E8008091E8008F778093E8000F900A
:105210000F90CF91DF91089580913807813049F147
:105220008230E1F58091F1009091F100882361F5E1
:10523000E091F100EF77E9F0E093E9008091EB0075
:1052400080FF15C08091EB0080628093EB0010928C
:10525000E900F0E0EF5CF84F81E080838091E800A6
:10526000877F8093E8008091E8008E7F0AC01092CB
:10527000E9008091EB0080628093EB008091E80070
:10528000877F8093E80008958091EB00806280938F
:10529000EB008091E800877F8093E800089580917B
:1052A00038078823E9F18130D9F1823009F04DC007
:1052B0008091F1009091F1008823E9F5E091F100EF
:1052C000EF77E093E9008091EB0080FF27C0EE23A9
:1052D000B1F08091EB0080618093EB0081E090E081
:1052E0000E2E02C0880F991F0A94E2F78093EA00FD
:1052F0001092EA008091EB0088608093EB0010929E
:10530000E900F0E0EF5CF84F10828091E800877FC1
:105310008093E8008091E8008E7F0AC01092E90037
:105320008091EB0080628093EB008091E800877FA2
:105330008093E80008958091EB0080628093EB00F9
:105340008091E800877F8093E8000895EBEEF0E01D
:10535000808180628083E8EEF0E08081877F8083B7
:1053600008958091E800877F8093E8008091E800AD
:105370008E7F8093E8008091E80080FFFCCF089545
:10538000DF93CF9300D0CDB7DEB710923007609196
:10539000F1008091F1001092A2141092A1141092C9
:1053A0009C1410929B14813019F0823099F407C03C
:1053B0000E94922B8093A0140E947D2B06C00E9415
:1053C000A92B8093A0140E94942B9093A2148093F5
:1053D000A1140DC00E947C31882349F48091EB0018
:1053E00080628093EB008091E800877F80C080918D
:1053F000F1008091F1008091F10089838091F100AA
:105400008A838091E800877F8093E80029813A8130
:105410008091A01490E08217930758F48F739070D6
:10542000892B21F481E08093300737C01092300738
:1054300034C02093A01431C08091E80080FFFCCFDD
:1054400020E022C0203421F1E091A114F091A214B7
:10545000309749F03196F093A214E093A11431975C
:1054600084918093F100E0919B14F0919C1430970B
:1054700039F081918093F100F0939C14E0939B1498
:105480002F5F91509093A0149091A0149923D1F67E
:105490008091E8008E7F8093E8008091A01488239B
:1054A00021F08091E80082FFC7CF8091E80082FD63
:1054B00016C080913007813071F48091E80080FF40
:1054C000FCCF8091E8008E7F8093E80004C080913B
:1054D000E80083FD0EC08091E80082FFF8CF809144
:1054E000E8008B7F8093E8008091E8008F778093BD
:1054F000E8000F900F90CF91DF9108959091F10007
:10550000923080F48091E800877F8093E800909348
:105510009F148091E8008E7F8093E800892F0E947D
:10552000E83008958091EB0080628093EB008091D9
:10553000E800877F8093E80008959091F1009093B0
:1055400038076091F1006630D9F0673058F4613067
:10555000B9F1613008F444C06330D1F1653009F02D
:1055600058C01EC0693021F16A3020F4683009F05B
:1055700050C00EC06A30F1F16B3009F04AC044C02F
:10558000903819F40E94C0290895892F66E039C027
:10559000903819F40E947D280895892F68E031C061
:1055A000992319F40E9460280895892F65E029C085
:1055B000992319F40E947E2A0895892F69E021C059
:1055C000933018F40E944F290895892F61E019C083
:1055D000933018F40E940C290895892F63E011C0BC
:1055E000892F8058833018F40E94B4280895892F99
:1055F00060E007C0913819F40E94A6290895892F08
:105600006AE00E9413320895913091F40E94B1290A
:105610000895892F0E941332882351F48091EB0062
:1056200080628093EB008091E800877F8093E800A0
:1056300008959091EB0091609093EB008093EC00C3
:105640008091ED008270862B8093ED008091ED00BB
:1056500082608093ED008091EE00881F8827881F6C
:1056600008959091F40080E090FD06C08F5F873030
:1056700011F09695F9CF80E00895FB018093E90041
:1056800004C081918093F10041508091E80085FF32
:1056900002C04423B1F7842F0895FB018093E900F1
:1056A00004C08091F100819341508091E80085FF12
:1056B00002C04423B1F7842F08958093E900EBEEF4
:1056C000F0E080818062808308958091D8008F7B94
:1056D0008093D8008091D90081FF0DC01092E9001D
:1056E0008091EB0080FD07C01092E90082E060E34A
:1056F0000E94192B089580E0089580910A05813059
:1057000019F420E634E00CC0882319F425EB34E0CA
:1057100007C0833019F020E635E002C025EB35E004
:10572000C901089582E1089580910A05813019F434
:1057300022E734E00CC0882319F427EC34E007C0DA
:10574000833019F022E735E002C027EC35E0C901CB
:10575000089580910A05813041F0882311F484E690
:105760000895833011F489E3089583E408958091C6
:10577000E800877F8093E80080918F148093F10088
:10578000809190148093F100809191148093F100A6
:10579000809192148093F100809193148093F10092
:1057A000809194148093F100809195148093F1007E
:1057B0008091E8008E7F8093E8008091E80080FF70
:1057C000FCCF8091E80082FFFCCF8091E8008B7FC6
:1057D0008093E8008091E8008F778093E800089537
:1057E0008091E800877F8093E8008091E80082FF45
:1057F000FCCF8091F10080938F148091F100809311
:1058000090148091F100809391148091F100809325
:1058100092148091F100809393148091F100809311
:1058200094148091F100809395148091E8008B7F0F
:105830008093E8008091E8008F778093E800809162
:10584000E8008E7F8093E8008091E80080FFFCCF25
:1058500008958091E800877F8093E8008091E800B8
:105860008E7F8093E8008091E80080FFFCCF089550
:10587000DF93CF9300D0CDB7DEB785E38093A0143C
:105880008BE295E09093A2148093A1148091E8009C
:10589000877F8093E8006633710528F04091A0145B
:1058A0002BE235E01CC06093A014F8CF8091E80093
:1058B00080FFFCCFF90190E00AC0542F5150903482
:1058C00049F09F5F84918093F1003196452F9F01AD
:1058D000442399F78091E8008E7F8093E800442369
:1058E00059F08091E80082FFE1CF3093A214209319
:1058F000A1144093A01406C03093A2142093A114C5
:105900001092A0148091E80082FD10C08FEF9FEFED
:1059100003C089819A8101979A83898389819A81B9
:10592000892B21F08091E80082FFF3CF8091E8007D
:105930008B7F8093E8008091E8008F778093E80068
:105940000F900F90CF91DF9108958091E800877FAD
:105950008093E80060933A078091E8008E7F8093FF
:10596000E8008091E80080FFFCCF0895DF93CF939B
:1059700000D0CDB7DEB78091E800877F8093E80044
:10598000452B49F080913A078093F1008091E8001F
:105990008E7F8093E8008FEF9FEF03C089819A810B
:1059A00001979A83898389819A81892B21F080913B
:1059B000E80082FFF3CF8091E8008B7F8093E800BE
:1059C0008091E8008F778093E8000F900F90CF913F
:1059D000DF910895982F8091E800877F8093E800F9
:1059E000913011F490E205C0933011F494E001C0BD
:1059F00090E0452B91F0992381F080E01092F10026
:105A00008F5F8917D8F38091E8008E7F8093E8003C
:105A10008091E8008F778093E8000895DF93CF931B
:105A200000D0CDB7DEB789E08093A0148BE195E07C
:105A30009093A2148093A1148091E800877F8093B3
:105A4000E8006A30710528F04091A0142BE135E0A0
:105A50001CC06093A014F8CF8091E80080FFFCCFB9
:105A6000F90190E00AC0542F5150903449F09F5FE3
:105A700084918093F1003196452F9F01442399F73B
:105A80008091E8008E7F8093E800442359F0809154
:105A9000E80082FFE1CF3093A2142093A114409339
:105AA000A01406C03093A2142093A1141092A01445
:105AB0008091E80082FD10C08FEF9FEF03C08981C5
:105AC0009A8101979A83898389819A81892B21F010
:105AD0008091E80082FFF3CF8091E8008B7F809374
:105AE000E8008091E8008F778093E8000F900F9096
:105AF000CF91DF910895DC01FC0120E030E029C066
:105B0000109721F08091F100819302C08091F10003
:105B10004150504061502F5F3F4F6623D1F44115F3
:105B20005105B9F08091E8008B7F8093E800809167
:105B3000E8008F778093E8008091E80082FFFCCF37
:105B40006091F200662329F466277727621B730BA6
:105B500004C041155105A1F670E0CB0108952F92C4
:105B60003F924F925F926F927F928F929F92AF92ED
:105B7000BF92CF92DF92EF92FF920F931F93DF932A
:105B8000CF9300D0CDB7DEB77C01D62E83E0861749
:105B900008F066C2F7019081992309F461C291303F
:105BA000B9F480910B05882309F45AC2DA9487016D
:105BB000FF24F3940AC0F80181810F5F1F4F8823EF
:105BC00009F44EC20E94020BF394FD14A0F348C2E4
:105BD000903109F065C18091A314882309F040C277
:105BE0009093A41481E08093A31401E074E1372E14
:105BF00063E1262E52E1752E41E1642E30E1532EF1
:105C000027E0422E99E7A92EB12CCC24C3949924E5
:105C10009A9485E0882EF701E00FF11D908196306F
:105C200009F44EC0973038F4943089F0953070F50F
:105C3000992359F029C1983009F4C5C0983008F467
:105C400084C09B3008F020C1D6C00D2D1DC18091AD
:105C5000A3148F3108F018C1E82FF0E0EC55FB4E8B
:105C600090838F5F9091F611A82FB0E0E82FEF5F3F
:105C7000992331F0AC55BB4E809102128C9303C036
:105C8000AC55BB4E9C92E093A314FEC08091A3142C
:105C90008E3108F0F9C0E82FF0E0EC55FB4E808221
:105CA0008F5FE82FF0E0EC55FB4E9091F911908357
:105CB0008F5FE82FF0E0EC55FB4E9091FA117EC01B
:105CC0008091A3148F3108F0DFC0E82FF0E0EC558D
:105CD000FB4E9083982F9F5F80910712882381F459
:105CE00080910C05A92FB0E0E92FEF5F882321F008
:105CF000AC55BB4E5C92C7CFAC55BB4E6C92C3CF7C
:105D0000813051F480910C058823C1F4E92FF0E033
:105D1000EC55FB4E708217C0823081F480910D05E6
:105D2000A92FB0E0E92FEF5F882321F4AC55BB4EDB
:105D30002C92A9CFAC55BB4E3C92A5CFE92FF0E0F9
:105D4000EC55FB4E10829F5F9DC08091A3148A3159
:105D500008F09AC0E82FF0E0EC55FB4E40828F5FD0
:105D6000E82FF0E0EC55FB4E9091420590838F5F59
:105D7000E82FF0E0EC55FB4E9091430590838F5F48
:105D8000E82FF0E0EC55FB4E9091440590838F5F37
:105D9000E82FF0E0EC55FB4E9091450590838F5F26
:105DA000E82FF0E0EC55FB4E9091460590838F5F15
:105DB000E82FF0E0EC55FB4E9091470590838F5F04
:105DC0008093A31461C01091A3141F3108F05CC02C
:105DD000E12FF0E0EC55FB4E90831F5F1093A3146E
:105DE0000E94FB07E12FF0E0EC55FB4E80831F5F24
:105DF0001093A31449C08091A3148F3008F044C0BD
:105E0000E82FF0E0EC55FB4E9083482F4F5F409316
:105E1000A31420E030E0993011F421E030E02A9D15
:105E2000F0012B9DF00D3A9DF00D1124EE52F44E31
:105E30008081A42FB0E0E42FEF5F8F3F21F0AC55BD
:105E4000BB4ECC9203C0AC55BB4E1C92E093A31446
:105E50009091A3142A9DD0012B9DB00D3A9DB00DB9
:105E60001124AE53B44E20E030E0E92FE20FF0E011
:105E7000EC55FB4E8D9180832F5F3F4F20313105D4
:105E8000A1F7905F9093A3140F5F0D1508F4C3CE94
:105E90008091A314813009F0E3C01092A314E0C0F4
:105EA000913109F0D8C011E001E05E010894A11C15
:105EB000B11CF701E10FF11DE081E430E9F0E530BC
:105EC00040F4E13089F0E13068F0E23009F0B7C029
:105ED00009C0E63009F450C0E63030F1E73009F08F
:105EE000AEC093C01D2DABC01F5FF701E10FF11DC8
:105EF000808180930B05A3C01F5FF701E10FF11DA7
:105F000080810E94330C8091F9119091FA119A834B
:105F10008983809102120E94330C89819A810E94A8
:105F2000CF118EE596E023C0912F9F5FF701E90F17
:105F3000F11D8081F50180831E5FF701E10FF11DE6
:105F40008081F5018183809102120E94330C898146
:105F50009A810E94CF116091FB117091FC11809188
:105F6000F9119091FA110E9475688DE496E00E94F3
:105F7000540B0093F61163C01F5FF701E10FF11D91
:105F8000E081E33131F482E00E94E12310920D05BB
:105F900007C0E43141F482E00E94E12300930D0543
:105FA00010920C0511C0E23111F481E0F5CFE1311E
:105FB00011F480E0F1CFEE2339F080E00E94E1237C
:105FC00000930C0500930D058091F9119091FA1141
:105FD0009A838983809102120E94330C89819A816D
:105FE0000E94CF110E94146980E090E00E94B9687D
:105FF0006091FB117091FC118091F9119091FA114F
:106000000E94756884E396E0B2CF8091A3148A3130
:10601000B0F41F5FF701E10FF11D8081809342050D
:1060200080818093430580818093440580818093A3
:1060300045058081809346058081809347051F5FD9
:106040001D1508F436CF80910712823049F486E09E
:106050000E948B0605C0983A19F481E080933907B5
:106060000F900F90CF91DF911F910F91FF90EF90C4
:10607000DF90CF90BF90AF909F908F907F906F9068
:106080005F904F903F902F900895DF93CF9300D073
:1060900000D000D0CDB7DEB78091E800877F809335
:1060A000E8008091E8008E7F8093E8008FEF9FEFFB
:1060B00003C089819A8101979A83898389819A8112
:1060C000892B09F58091F1008B838091F1008C83FD
:1060D0008091F1008D838091F1008E838091E800A2
:1060E0008B7F8093E8008091E8008F778093E800B1
:1060F0008091E8008E7F8093E800CE01039664E0F3
:106100000E94AF2D05C08091E80082FFD2CFDACF88
:106110008091E80080FFFCCF26960FB6F894DEBF92
:106120000FBECDBFCF91DF910895DF93CF93CDB751
:10613000DEB7A2970FB6F894DEBF0FBECDBF809139
:10614000E800877F8093E8008091E8008E7F80934D
:10615000E8008FEF9FEF03C089819A8101979A83AE
:10616000898389819A81892B41F4FE013396CF017D
:106170004E2F9E012D5D3F4F05C08091E80082FFAC
:10618000EBCFF3CF8091F1008193E217F307D1F7C2
:106190008091E8008B7F8093E8008091E8008F7702
:1061A0008093E8008091E8008E7F8093E800842F40
:1061B00060E20E94AF2D8091E80080FFFCCFA296A4
:1061C0000FB6F894DEBF0FBECDBFCF91DF9108951B
:1061D000FF920F931F9380910A05823011F088235C
:1061E00019F583E08093E90081EC60E30E94192BAC
:1061F00081E08093E90081E864E30E94192B12E0BA
:106200001093E90080E864E30E94192B88E08093F2
:10621000EA001092EA001093EA001092EA0084E08B
:106220008093EA001092EA0080910A05882379F4AD
:1062300084E08093E90081EC64E20E94192B80E104
:106240008093EA001092EA0082E080933B078091FD
:106250000A05813021F584E08093E90081EC60E259
:106260000E94192B85E08093E90081E860E20E949A
:10627000192B86E08093E90080E864E20E94192BE4
:1062800080E18093EA001092EA0080E28093EA00C5
:106290001092EA0080E48093EA001092EA000091F4
:1062A0000A05033029F5FF24F394F092E90081E810
:1062B00064E30E94192B12E01093E90080E864E384
:1062C0000E94192B0093E90081EC60E20E94192BD7
:1062D0001093EA001092EA0084E08093EA001092A2
:1062E000EA0088E08093EA001092EA00F0923B070F
:1062F0001F910F91FF9008959F92AF92BF92CF92FE
:10630000DF92EF92FF920F931F93833009F080C0CA
:10631000613071F0613030F0623081F0633009F04B
:1063200077C016C084E08093A01480E396E00BC091
:106330008CE08093A01480E096E005C084E2809316
:10634000A0148CE096E09093A2148093A1145EC0F8
:106350001091EE11B090EF11A090F0119090F1110A
:106360006091F2117091F3118091F4119091F511F7
:106370002DB73EB72C5030400FB6F8943EBF0FBE3D
:106380002DBFEDB6FEB60894E11CF11CECE3CE2E59
:10639000E7E0DE2EEDB7FEB7D282C18225E335E01D
:1063A000F70133832283212F3B2D4A2D592D00E203
:1063B0000E94EC7DC901BA01F701248395834683CD
:1063C00077831087B186A28693860E94A87FF60104
:1063D000A1E1B5E02DB73EB7245F3F4F0FB6F8946B
:1063E0003EBF0FBE2DBF8191992787FD90958D935C
:1063F0009D9337E0EE34F307B1F786E28093A01463
:106400008FE095E090939C1480939B1481E001C0F1
:1064100080E01F910F91FF90EF90DF90CF90BF90A1
:10642000AF909F900895DF93CF9300D000D0CDB769
:10643000DEB7582FA091F1007091F1008091F1002A
:1064400089838091F1008A838091F1008B83809110
:10645000F1008C835A9A5A9840910A05442311F00E
:106460004230B9F4513211F0513A89F489819A815C
:10647000892B69F4662319F0613049F405C08B81DA
:106480009C810E94283A76C00E943A3573C044230A
:1064900019F0433009F05AC05138D9F429813A81B2
:1064A00080913B0790E02817390799F4663089F40A
:1064B000713219F0723269F406C06B817C81C901B6
:1064C0000E940E2D51C06B817C81C9010E94382C25
:1064D0004BC0442311F04330C9F5513211F0513A09
:1064E000A9F5E981FA8180913B0790E0E817F90767
:1064F00069F5623021F1633018F4613039F518C064
:10650000693019F06A3011F50BC0723019F0733030
:10651000E9F403C00E94953027C00E94453024C092
:106520002B813C818A2F672FAF010E94A52C1CC0B4
:106530004B815C81872FBF010E94EA2C15C04B81E3
:106540005C818A2FBF010E94B62C0EC0413089F4B5
:10655000613229F0623251F0603259F403C00E9476
:10656000B72B02C00E94F02B81E004C00E94292CAE
:10657000FBCF80E00F900F900F900F90CF91DF91A5
:1065800008955D988AE08093C514089577988AE00D
:106590008093C4140895FF920F931F93CF93DF93BA
:1065A0008C01EB01F42E8091B215823011F080E065
:1065B0009CC081E090E0A0E0B0E08093C61490938E
:1065C000C714A093C814B093C91484E290E0A0E06B
:1065D000B0E08093CE149093CF14A093D014B093D6
:1065E000D114CB01A0E0B0E08093D2149093D314E7
:1065F000A093D414B093D5141092DA141092DB1433
:106600001092DC141092DD141092D6141092D7144C
:106610001092D8141092D9141092DE141092DF1434
:106620001092E0141092E1141092E2141092E3140C
:106630001092E4141092E5141092E6141092E714EC
:106640001092E8141092E9141092EA141092EB14CC
:106650001092EC141092ED141092EE141092EF14AC
:106660001092F0141092F1148C96A11DB11D80931C
:10667000CA149093CB14A093CC14B093CD1481E0A2
:106680008093E9008091E8008F778093E800809103
:10669000E80085FFFCCFE6ECF4E181918093F10006
:1066A00084E1E23FF807C9F718C0F80180818093C0
:1066B000F1008091E80085FD09C08091E8008F77A6
:1066C0008093E8008091E80085FFFCCFFF2011F067
:1066D0000E94C6320F5F1F4F2197209731F780919C
:1066E000E8008F778093E80081E0DF91CF911F91E0
:1066F0000F91FF900895DF92EF92FF920F931F93F7
:10670000DF93CF9300D000D0CDB7DEB7FC01D42EFD
:1067100080919F14882309F456C09B012C5F3F4F42
:1067200081E08093E9008091E80085FFFCCF209311
:10673000F100832F8F738093F10012C081918093B9
:10674000F100615070408091E80085FD09C08091A2
:10675000E8008F778093E8008091E80085FFFCCF08
:106760006115710559F78EED89838DEA8A838EEB69
:106770008B838FEE8C838E010F5F1F4F85E0E82E99
:10678000F12CEC0EFD1EF80180818093F1008091C8
:10679000E80085FD09C08091E8008F778093E800CC
:1067A0008091E80085FFFCCFDD2011F00E94C63209
:1067B0000F5F1F4F0E151F0531F78091E8008F778F
:1067C0008093E80081E00F900F900F900F90CF9191
:1067D000DF911F910F91FF90EF90DF9008959C0142
:1067E00080910E05813081F080910A05833021F47B
:1067F000C9010E947B330895823011F0882321F46F
:10680000C9010E94CB32089580E008951F93CF9371
:10681000DF938091C514882321F081508093C514A3
:1068200001C05D9A8091C414882321F08150809327
:10683000C41401C0779A80919F14882309F46DC015
:1068400080910A05833009F068C080914E05882345
:1068500039F05F9A88E495E00E94B96810924E057D
:1068600082E08093E9008091E80082FF56C0809129
:10687000C3159091C415892B09F04FC08091071260
:10688000823009F44AC06091F200623068F02091D1
:10689000F1002093C6148091F1008093C714162F45
:1068A0001250882364F439C08091E8008B7F809374
:1068B000E8008091E8008F778093E800E8CF90E0CF
:1068C0008F739070D82FCC27822F90E0C82BD92BB4
:1068D000209719F10E94C13280E496E1612FAE0148
:1068E0000E947B2D8091E8008B7F8093E80080914F
:1068F000E8008F778093E800BE016450704080917B
:106900000E05882331F080E496E140E00E947B335D
:1069100004C080E496E10E946B798091B2158230C8
:1069200009F0A0C080910A05882319F0823009F08F
:1069300099C080914E05882339F05F9A88E495E0EC
:106940000E94B96810924E0582E08093E900809120
:10695000E80082FF75C08091C3159091C415892B02
:1069600009F06EC080910712823009F469C060910D
:10697000F2006C3210F020E00BC08091E8008B7FB9
:106980008093E8008091E8008F778093E80021E011
:10699000E6ECF4E18091F100819384E1E23FF807B5
:1069A000C9F7162F1C528091C6149091C714A0915C
:1069B000C814B091C9140197A105B10559F080918F
:1069C000E8008B7F8093E8008091E8008F778093C8
:1069D000E80022E08091D2149091D314A091D414B5
:1069E000B091D5140097A105B10551F1222341F5CD
:1069F0000E94C1324091CE145091CF144452504065
:106A000080E090E0612F0E947B2D4091D214509144
:106A1000D31480E496E1612F0E947B2D8091E800E1
:106A20008B7F8093E8008091E8008F778093E80067
:106A30006091D2147091D31480E496E10E946B7936
:106A400080910712823071F48091E80082FF0AC0C1
:106A50008091E8008B7F8093E8008091E8008F7739
:106A60008093E800DF91CF911F91089581E080939A
:106A700051070895DF93CF9300D0CDB7DEB7809153
:106A8000E800877F8093E80090915207392FE0E07B
:106A90001DC08091E80080FFFCCF2E2F5E2F505C40
:106AA0000DC0432F4150251759F0E22FF0E0EA5F67
:106AB000FA4E80818093F1002F5F342F332389F7C2
:106AC0008091E8008E7F8093E800E22F332339F035
:106AD0008091E80082FFDDCF3093520702C0109210
:106AE00052078091E80082FD1FC0892F90E08F73CC
:106AF0009070892B49F48091E80080FFFCCF809151
:106B0000E8008E7F8093E8008FEF9FEF03C08981BC
:106B10009A8101979A83898389819A81892B21F0AF
:106B20008091E80082FFF3CF8091E8008B7F809313
:106B3000E8008091E8008F778093E80081E00F9073
:106B40000F90CF91DF910895DF93CF9300D0CDB711
:106B5000DEB79B01AC018091E80080FF53C08091BB
:106B60005207882309F04EC087E090E0A0E0B0E033
:106B70008093061590930715A0930815B0930915F7
:106B800084E190E0A0E0B0E080930A1590930B15AB
:106B9000A0930C15B0930D1520930E1530930F157F
:106BA0004093101550931115E6E0F5E18191809323
:106BB000F10085E1EA31F807C9F78091E8008E7F9E
:106BC0008093E8008091E80080FFFCCF8FEF9FEF7B
:106BD00003C089819A8101979A83898389819A81E7
:106BE000892B21F08091E80082FFF3CF8091E800AB
:106BF0008B7F8093E8008091E8008F778093E80096
:106C000081E001C080E00F900F90CF91DF91089557
:106C10000895A0911A15B0911B15FD01E25FFA4E7F
:106C20002481358146815781233331054105510542
:106C300010F082E303C0822F01C082501816ECF3DB
:106C4000209112153091131540911415509115157E
:106C50002B3182E0380781E0480780E0580709F4CB
:106C600080C02C3182E0380781E0480780E0580777
:106C7000C0F42F3081E0380781E0480780E05807F2
:106C800009F46FC0223181E0380781E0480780E0D5
:106C9000580709F466C02E50314041405040D1F5AC
:106CA00017C0213081E0380781E048078DE05807A0
:106CB00041F1223081E0380781E048078DE0580734
:106CC00009F44FC0235031404140514019F549C0AB
:106CD000A25FBA4E8D919D910D90BC91A02D809395
:106CE000530790935407A0935507B0935607009706
:106CF000A105B10511F082E001C081E08093B215D9
:106D000030C0A25FBA4E8D919C91909358058093AC
:106D1000570527C085E090E0A0E0B0E88093061515
:106D200090930715A0930815B093091520E130E062
:106D300040E050E020930A1530930B1540930C155A
:106D400050930D1581E090E0A0E0B0EC8093121517
:106D500090931315A0931415B09315152093520713
:106D6000089585E090E0A0E0B0E880930615909348
:106D70000715A0930815B093091580E190E0A0E0F5
:106D8000B0E080930A1590930B15A0930C15B09367
:106D90000D151092121510921315109214151092D1
:106DA0001515809352070895E6E0F5E184E090E040
:106DB000A0E0B0E88093061590930715A0930815FE
:106DC000B093091584E090E0A0E0B0E08093161540
:106DD00090931715A0931815B093191580E190E0C2
:106DE000A0E0B0E080931A1590931B15A0931C159A
:106DF000B0931D158091121590911315A091141543
:106E0000B0911515853021E0920722E0A20720E01D
:106E1000B20709F4DCC2863021E0920722E0A20723
:106E200020E0B20708F0BFC08D3021E0920721E0DA
:106E3000A20720E0B20709F4C8C18E3021E0920712
:106E400021E0A20720E0B20708F049C0863021E027
:106E5000920721E0A20720E0B20709F4A2C187301F
:106E600021E0920721E0A20720E0B207F8F4823087
:106E700021E0920721E0A20720E0B20709F4A7C2AF
:106E8000833021E0920721E0A20720E0B20738F426
:106E900081509140A140B04009F0A2C269C1855023
:106EA0009140A140B04008F09BC291C28C3021E0DB
:106EB000920721E0A20720E0B20708F081C18A30E2
:106EC00021E0920721E0A20720E0B20708F073C199
:106ED00087509140A140B04009F082C267C186311D
:106EE00021E0920721E0A20720E0B20709F48EC159
:106EF000873121E0920721E0A20720E0B20710F5D8
:106F00008F3021E0920721E0A20720E0B20709F4C8
:106F100082C18F3021E0920721E0A20720E0B20772
:106F200008F466C1813121E0920721E0A20720E048
:106F3000B20709F466C184519140A140B04009F004
:106F40004FC245C2823021E0920722E0A20720E032
:106F5000B20709F4FDC1833021E0920722E0A207C5
:106F600020E0B20780F4823022E0920721E0A207FD
:106F700020E0B20709F42BC281509140A240B040FA
:106F800009F02EC2DCC1833021E0920722E0A20783
:106F900020E0B20709F4EEC184509140A240B04015
:106FA00009F01EC2DEC1883021E0920721E0A2076D
:106FB0002DE0B20709F4F0C0893021E0920721E00A
:106FC000A2072DE0B20708F06AC0853021E09207E1
:106FD00021E0A20721E0B20709F4F9C1863021E0DF
:106FE000920721E0A20721E0B20740F5823021E0BC
:106FF000920721E0A20721E0B20709F438C18330EB
:1070000021E0920721E0A20721E0B20738F4815085
:107010009140A140B14009F0E3C1FDC0833021E0BF
:10702000920721E0A20721E0B20709F441C1845090
:107030009140A140B14009F0D3C13FC1833021E06C
:10704000920722E0A20721E0B20709F4C0C1843010
:1070500021E0920722E0A20721E0B20780F481300C
:1070600021E0920722E0A20721E0B20709F4AFC1B4
:1070700082509140A240B14009F0B2C1A8C1813014
:1070800021E0920721E0A2072DE0B20709F41AC11E
:1070900082509140A140BD4009F0A2C136C18E305E
:1070A00022E0920721E0A2072DE0B20709F474C0A4
:1070B0008F3022E0920721E0A2072DE0B20740F5D1
:1070C0008B3121E0920721E0A2072DE0B20709F4FD
:1070D00063C08C3121E0920721E0A2072DE0B207C6
:1070E00038F488519140A140BD4009F079C154C0A5
:1070F000843022E0920721E0A2072DE0B20709F4D4
:1071000066C186509240A140BD4009F069C112C1DC
:10711000803021E0920721E0A2072DEFB20709F4A9
:107120003AC1813021E0920721E0A2072DEFB2079A
:1071300078F4813122E0920721E0A2072DE0B20726
:1071400059F187519240A140BD4009F049C124C086
:10715000823021E0920721E0A2072DEFB20709F467
:107160002DC186509140A140BD4F09F039C12FC1BA
:107170008CE890E0A0E0B0E080931615909317158E
:10718000A0931815B0931915CF0148966FE676E0D5
:107190004CE850E00E94EA7E80E090E0A0E0B0E0A1
:1071A0002BC180E095E0A0E0B0E0ECC084E690E088
:1071B000A0E0B0E0E7C086E690E0A0E0B0E0E2C08A
:1071C0008FEF9FEFAFEFB0E0DDC088E090E0A0E090
:1071D000B0E08093161590931715A0931815B093EF
:1071E0001915CF01489669E077E048E050E0D2CF2A
:1071F0008091530790915407A0915507B09156077D
:10720000C1C084E195E0A0E0B0E0BCC080E090E1C6
:10721000A0E0B0E0B7C01092221510922315109292
:107220002415109225158091540580931E15809188
:10723000530580931F1580915205809320158091EE
:1072400051058093211580915005809322158091DE
:107250004F05809323158091161590911715A091D5
:107260001815B09119150296A11DB11D45C01092B7
:107270002215109223151092241510922515809135
:10728000540580931E158091530580931F1580919E
:10729000520580932015809151058093211580918E
:1072A00050058093221580914F058093231520C0AF
:1072B00080E090E0A0E0BEE065C081E090E0A0E06A
:1072C000B0E060C08091570590915805A0E0B0E013
:1072D00080931E1590931F15A0932015B093211530
:1072E0001092221510922315109224151092251534
:1072F00086E090E0A0E0B0E080931615909317151B
:10730000A0931815B093191547CF8DE090E0A0E039
:10731000B0E080931E1590931F15A0932015B09395
:10732000211582E295E16BEF76E04DE050E00E949E
:10733000FE7E32CF8CEE9FEFAFEFBFEF23C0809188
:10734000B3159091B415A091B515B091B6151AC0AA
:107350008091B7159091B815A091B915B091BA1553
:1073600011C08091BF159091C015A091C115B09129
:10737000C21508C08091BB159091BC15A091BD1598
:10738000B091BE1580931E1590931F15A0932015E4
:10739000B093211501CF83E090E0A0E0B0E08093AE
:1073A000161590931715A0931815B0931915789684
:1073B00083E0DF011D928A95E9F7EECE1092161553
:1073C000109217151092181510921915E5CE1092FB
:1073D0001E1510921F151092201510922115DCCE4B
:1073E0001092161510921715109218151092191563
:1073F00081E090E0A0E0B0EC80931215909313151B
:10740000A0931415B093151580911615909117152A
:10741000A0911815B09119154896A11DB11D809322
:107420000A1590930B15A0930C15B0930D15489762
:10743000A109B10941F410921A1510921B1510926E
:107440001C1510921D1580910A15809352070895FE
:107450002091E800277F2093E8009C018D3A910558
:1074600010F02CEA30E0E0E021C08091E80082FFDB
:10747000FCCF9E2F4E2F405C8091F100E92FF0E071
:10748000EA5FFA4E80839F5F21503040941719F0D5
:107490002115310589F78091E8008B7F8093E80002
:1074A0008091E8008F778093E800E92F211531055E
:1074B000E1F68091E8008E7F8093E80080910615C8
:1074C00090910715A0910815B09109158430910588
:1074D000A105B10509F4A4C085309105A105B10548
:1074E00058F482309105A105B105C1F00397A105BB
:1074F000B10509F0EFC08AC086309105A105B1053C
:1075000009F494C086309105A105B10508F48BC03B
:107510000897A105B10509F0DDC0B9C082E090E08F
:10752000A0E0B0E88093061590930715A093081586
:10753000B093091524E330E040E050E020930A15B1
:1075400030930B1540930C1550930D1581E090E08E
:10755000A0E0B0E08093161590931715A09318152E
:10756000B093191580931A1590931B15A0931C15B1
:10757000B0931D1510921215109213151092141538
:107580001092151580931E1590931F15A09320152A
:10759000B0932115109222151092231510922415E4
:1075A000109225158093261590932715A0932815E2
:1075B000B09329158AE395E0A0E0B0E080932A1506
:1075C00090932B15A0932C15B0932D1583E090E08C
:1075D000A0E0B0E080932E1590932F15A093301566
:1075E000B093311510923215109233151092341554
:1075F00010923515109236151092371510923815D5
:107600001092391581E08093B2153EC05F9A5D9863
:10761000779876988091E8008E7F8093E800FFCF7E
:107620000E94D4365AC00E94093657C01092B21533
:1076300086E090E0A0E0B0E88093061590930715EF
:10764000A0930815B093091520E130E040E050E028
:1076500020930A1530930B1540930C1550930D157C
:1076600010920E1510920F15109210151092111500
:1076700081E090E0A0E0B0E08093121590931315A4
:10768000A0931415B09315152093520726C088E0D7
:1076900090E0A0E0B0E88093061590930715A093C2
:1076A0000815B093091580E190E0A0E0B0E0809368
:1076B0000A1590930B15A0930C15B0930D1510920D
:1076C000121510921315109214151092151580931F
:1076D000520703C0779880E008958091E80080FF0A
:1076E000FCCF8091E80082FF0AC08091E8008B7F88
:1076F0008093E8008091E8008F778093E8000E94F3
:10770000363581E00895FC015381560F5093CA1518
:10771000272F33274281420F4093C915A181A0939F
:10772000C815E081E093C715842F90E08217930776
:1077300048F48A2F8F5F8093C815882319F4EF5F70
:10774000E093C715852F90E070708617970790F427
:10775000842F8F5F8093C915882361F48091C815A9
:107760008F5F8093C815882329F48091C7158F5F98
:107770008093C71508959C0141505040460F571FF4
:10778000FB010EC0708160E08181DB01A80FB11D9B
:107790002A0F3B1F2A173B0710F42F5F3F4F3296EB
:1077A000E417F50778F3E417F50749F4908180E0D2
:1077B000280F391F2817390710F42F5F3F4FC901D1
:1077C0000895AC0110925A0720E013C0E22FF0E0B8
:1077D000322F3F5FEE0FFF1FE45CF94E80819181F5
:1077E0008417950729F420935A071182108208956F
:1077F000232F223058F320935A070895AC0110929A
:107800005A0720E012C0E22FF0E0322F3F5FEE0F68
:10781000FF1FE45CF94E80819181892B29F420932C
:107820005A07518340830895232F223060F3209319
:107830005A070895BC018091E2159091E315449692
:107840000E94833BE091E215F091E3158091C7150A
:10785000848B8091C815858B8091C915868B80910A
:10786000CA15878B0895282F892F922F0895AF92DC
:10787000BF92CF92DF92EF92FF920F931F93CF931D
:10788000DF93B82EA92E6B0100915B0710915C0766
:107890007CE2E72E0F5F1F4F8DE70030180710F0D6
:1078A00000E010E1FF2411C0FE9CE0011124CC5146
:1078B000DA4E8DA1882341F0C8010E94333C28890B
:1078C00039892817390731F3F39482E0F81661F704
:1078D00000935B0710935C0710925A07C0E0D0E05A
:1078E00020E03CE216C0239FF0011124EC51FA4E37
:1078F00085A1882321F420935A07EF010EC0873019
:1079000039F4209721F096A18EA1891708F4EF0190
:107910002F5F223040F320935A07209789F182E0AD
:107920008DA380915D07888F80915E07898F8091FC
:107930005F078A8F809160078B8F84EC94E09F8F24
:107940008E8F99A388A381E090E09D8F8C8F1FA2DA
:1079500081E08EA383E08CA31AA280E18BA3C801EF
:107960000E94333C998B888BDB8ACA8ADE012B2DDF
:107970003A2DC901FC0180E101900D928150E1F79F
:10798000CE01DF91CF911F910F91FF90EF90DF908B
:10799000CF90BF90AF9008950F931F93109144160E
:1079A00000E090915807091B110990914516090FA5
:1079B000111D9801280F311DC90168E476E140E2EC
:1079C00050E00E94BB3B6091580770E06859794EC7
:1079D000A8010E94BB3B009719F42FEF3FEF03C0B3
:1079E0000E94333C9C01C9011F910F91089581E1D0
:1079F0000E94CC3C089586E00E94CC3C08958AE326
:107A00000E94CC3C089580E090E060E476E148E29A
:107A100050E00E94BB3B009719F42FEF3FEF03C0EB
:107A20000E94333C9C01C90108959C01AB0180E098
:107A300090E0B9010E94BB3B0E94333C0895EF9255
:107A4000FF920F931F939C0144275527F22EE32E9C
:107A500000E010E0362F272F40E050E0A901332747
:107A60002227E22AF32A042B152BB701C8011F9104
:107A70000F91FF90EF900895FC014091C515509132
:107A8000C61520E43BE1241B350B621773070CF489
:107A90009B011216130664F42093421B3093431B80
:107AA000E417F50729F0CA01BF01A9010E941A7F56
:107AB000089582E080935907A09158072A2F30E05B
:107AC000F901E859F94E8181682F70E0B3E0660F43
:107AD000771FBA95E1F7695F7F4F42E0285D3F4F1E
:107AE0003CC0F901E80FF91FE05CF94E8081882362
:107AF00019F0813019F42EC04F5F2FC090E0807CC8
:107B000090708038910549F0803C910549F08034AF
:107B1000910501F54093590709C04093590708C0E2
:107B200040935907809158168F3F11F481E00895D2
:107B3000242F30E040E050E02A0F311D411D511D3F
:107B4000285D3F4F4F4F5F4F84E062E00E94C74780
:107B500082E0089581818E5F480F842F90E068173E
:107B600079070CF0BECF4093590780E008950F933A
:107B70001F93CF93DF93C091E215D091E31584302A
:107B800009F4F5C20CE716E11093E1150093E01536
:107B90001093C6150093C515833069F48DA18F70BD
:107BA000833011F00C948C468C8D9D8D892B11F0B7
:107BB0000C948C4694C0823009F095C01092C41584
:107BC0001092C3151092431B1092421B80916007C4
:107BD0008F5F80936007882399F480915F078F5FA0
:107BE00080935F07882361F480915E078F5F8093A5
:107BF0005E07882329F480915D078F5F80935D077E
:107C00002DA1273011F0253051F48EA18F5F8EA366
:107C1000883711F00C948C461DA20C948C462223BC
:107C200011F40C948C468C8D9D8D892B09F452C0D7
:107C30008EA181508EA38F5F11F00C948C463FA1D2
:107C4000383029F02150223048F4353039F41DA263
:107C500080E88093DB150E94D27900C7353010F0A0
:107C600080E307C083E090E002C0880F991F3A9537
:107C7000E2F78EA38FA18F5F8FA38DA190E08F700D
:107C800090708330910501F1843091054CF481307E
:107C9000910509F491C4029711F00C948C460DC023
:107CA0008630910509F4EEC68830910509F4EAC6DC
:107CB000049711F00C948C46E5C6E0915807F0E06B
:107CC000E859F94E15867FC484E08093DB150E9445
:107CD000D27906C72F70233011F00C948C4688E0BF
:107CE0008093DB15AFC6853021F5E091DE15F0916C
:107CF000DF1580899189892B11F40C948C461092A0
:107D0000E3151092E215C8010C979093E11580934A
:107D1000E0159093C6158093C5151092431B1092E1
:107D2000421B1092C4151092C31588E08093DB1596
:107D30001CC280914016807F803609F0EDC790917B
:107D4000441680E020914516AC01420F511D9A0166
:107D50008091C3159091C4158417950708F4DCC76A
:107D6000285D3F4F3093C4152093C315809148166A
:107D70008F3F09F4D1C7C801849760E840E00E94B2
:107D8000F25F892B09F067C0C80184970E94576091
:107D9000882309F060C0809158168F3F09F058C0C1
:107DA00080915916823009F053C080915A169091F3
:107DB0005B16892B09F04CC080915C1690915D1682
:107DC000892B01F580915E1690915F16892BD1F475
:107DD0008091601690916116892BA1F480916216B2
:107DE00090916316892B71F48091641690916516B9
:107DF000892B41F480916616882321F480916716BF
:107E0000813049F180915C1690915D16892B01F5C6
:107E100080915E1690915F16892BD1F48091601647
:107E200090916116892BA1F480916216909163164E
:107E3000892B71F48091641690916516892B41F419
:107E400080916616882321F480916716823019F09C
:107E50000E949B4669C786E496E19093DD15809366
:107E6000DC151092580710925707E091DC15F0913D
:107E7000DD1580818B3209F44BC08C3248F486309A
:107E800009F4E0C1813109F4B1C0882389F06BC0E5
:107E90008A3309F474C08B3320F48C3209F063C048
:107EA0003BC78B3309F438C78C3309F05CC006C07C
:107EB0008091570780FD57C0816009C080915707A6
:107EC00081FF04C086FD4FC0806401C08260809342
:107ED00057070E94593D813009F41EC7813018F0C0
:107EE000823019F621C720915807E22FF0E0CF0128
:107EF0008859994E9093DD158093DC15285FFC011D
:107F00008181880F880F880F280F20935807ADCFE5
:107F10008091570782FD27C0846080935707909116
:107F20005807E92FF0E0DF01A859B94E13968C915C
:107F30001397882349F0BA969F01442737FD40954F
:107F4000542F84E060E018C0B093DD15A093DC15D9
:107F5000985FE859F94E8181880F880F880F980F34
:107F60009093580782CFE054F6419F01442737FD94
:107F70004095542F84E061E00E94C747D5C60E9417
:107F8000FF3C8F5F9F4F09F0C7C6E0915807F0E0B4
:107F9000E859F94EE081E538A9F0E63818F4E03800
:107FA000C9F413C0E73829F0E73848F0E83891F40D
:107FB00003C00E94085812C00E94A4560FC00E941D
:107FC000D24F0CC00E94B15C09C00E94FD120E94F9
:107FD000A64804C01092C4151092C3158091C31511
:107FE0009091C415892B09F497C69EC68091C3153C
:107FF0009091C415C0979093C4158093C31580E7E2
:1080000096E19093E1158093E015E0915807F0E038
:10801000E859F94E86819781892B31F00E94F73C0F
:108020008F5F9F4F09F078C684E49BE19093DF1542
:108030008093DE154BC0288939892115310509F453
:1080400040C080915807E82FF0E0E859F94E82814E
:10805000938182179307A9F52A893B892115310558
:1080600029F0808191818217930759F58881998140
:10807000892BE9F48A819B81892BC9F48C819D81AC
:10808000892BA9F48E819F81892B89F48885998514
:10809000892B69F48A859B85892B49F48C859D857C
:1080A000892B29F48E859F85892B09F449C088E4A2
:1080B00096E1BE0140E150E00E940D7F009709F477
:1080C0003FC06996D093DF15C093DE15C091DE15D1
:1080D000D091DF15BBE1C637DB0708F4ACCFE091E8
:1080E0005807F0E0E859F94E82819381998B888B8B
:1080F000808191819B8B8A8B2091DE153091DF15D9
:10810000C901DC01E8E4F6E180E101900D928150C3
:10811000E1F782E08093DB1580E796E19093E1152B
:108120008093E0159093C6158093C5158091C31573
:108130009091C415C0979093431B8093421B15C028
:108140001092E3151092E21582E08093DB1580E730
:1081500096E19093E1158093E0159093C615809376
:10816000C5151092431B1092421B0E9498762091D5
:10817000421B3091431B2115310509F4CDC5C901BE
:10818000C0969093C4158093C315285F3F4F3093DA
:108190004416885280934516A091DE15B091DF15E4
:1081A00054968C9154978093471681E1809346169C
:1081B000E0915807F0E0E859F94E3483258317829F
:1081C000168250968D919C915197918380835296FF
:1081D0008D919C91539793838283A8E5B6E120917A
:1081E000DE153091DF15C901FC0180E101900D928F
:1081F0008150E1F788E496E168E576E10E94D35D7D
:108200008CE796E19093E1158093E01580915807F3
:10821000C82FD0E0C859D94E0E94F73C8095909560
:108220009F838E8380915807E82FF0E0E859F94E3C
:1082300086819781892B09F065C58FEF9FEF978322
:10824000868360C50E94FB3C8F5F9F4F09F064C529
:1082500080915807082F10E00859194EC4EED5E157
:108260008DA18823D9F0D80112962D913C911397B6
:10827000888999892817390789F42D913C918A8931
:108280009B892817390751F488E496E1BE0140E143
:1082900050E00E940D7F009709F4B2C1AC96B6E1A0
:1082A000C031DB07E9F2E0F2F80185858F73823097
:1082B00001F5828193819093630780936207109206
:1082C0005A0713C0E42FF0E0EE0FFF1FE45CF94EF5
:1082D00020916207309163078081918128173907C7
:1082E00009F489C04F5F40935A0740915A074230C2
:1082F00048F380915807E82FF0E0DF01A859B94E04
:108300001D968C911D9782FD07C584E11D968C9367
:108310001D978CE390E09093C4158093C315FD01E5
:1083200080E5848797811B968C911B9717968C9379
:108330001797938796811A968C911A9716968C9315
:1083400016979287958119968C91199715968C930B
:1083500015979187948190935A0718968C91189746
:1083600014968C93149790871B968C911B978F5F14
:108370001B968C931B978823C1F41A968C911A979D
:108380008F5F1A968C931A97882379F419968C919B
:1083900019978F5F19968C931997882331F4189643
:1083A0008C9118978F5F18968C93E0915807F0E0A6
:1083B000DF01A859B94E2D913C9111973093630775
:1083C00020936207FD0182819381918380831396BC
:1083D0003C932E931297E8E5F6E1DF01509780E198
:1083E0000D9001928150E1F788E496E168E576E12D
:1083F0000E94D35D54C410925A07C0E0D0E04CE212
:1084000050E03CE225C0822F90E0849FF001859FE0
:10841000F00D949FF00D1124EC51FA4E85A18823A4
:1084200039F48CE2289FE0011124CC51DA4E14C0BB
:10843000873059F4209721F096A18EA1891728F44E
:10844000239FE0011124CC51DA4E2F5F20935A076D
:1084500020915A072230B8F2209709F45DC4D093D6
:10846000E315C093E21583E08EA38CA31AA284E0E7
:108470008BA31FA2E0915807F0E0E859F94E8281E2
:108480009381998B888B808191819B8B8A8BDE0174
:10849000E8E4F6E180E101900D928150E1F781E09E
:1084A0008DA380915D07888F80915E07898F809171
:1084B0005F078A8F809160078B8F81E090E09D8FAE
:1084C0008C8FE0915807F0E0E859F94E87818F8B47
:1084D000E0915807F0E0E859F94E86818E8BE091E3
:1084E0005807F0E0E859F94E85818D8BE0915807E7
:1084F000F0E0E859F94E84818C8B81E090E00E9495
:108500001A3CE0915807F0E0E859F94E848590E074
:10851000807F9070813591050CF44EC010925A07FF
:1085200035C0F901E05CF94E84AD80936107882382
:1085300009F442C0813021F44F5F40935A0726C0AE
:108540008230C1F485AD8430A9F436AD20E087AD2A
:1085500090E0822B932B9093630780936207F4E063
:10856000853C9F0710F084EC94E09F8F8E8F99A339
:1085700088A322C080915A07E82FF0E0E358F94E13
:10858000E081EE23C9F0E80FE0935A0740915A07C3
:10859000242F30E0E0915807F0E0E859F94E848547
:1085A00082958F7090E00597880F991F880F991F0B
:1085B000281739070CF4B5CFE0915807F0E0E859D7
:1085C000F94E80E18587E0915807F0E0DF01A85976
:1085D000B94E1D968C911D9782601D968C931D97A8
:1085E000FD0182E0848B84E0858B868B84EC878B15
:1085F00080E490E09093C4158093C31580E60EC389
:10860000D093E315C093E2151092DB1580915807C3
:10861000A82FB0E0FD01E859F94E858582FF03C01F
:108620001DA280E293C2848582958F70880F880F87
:1086300080935A072091C3153091C41528523040B9
:10864000281B31093093C4152093C3158DA18F7059
:10865000823039F4A859B94E1D968C918F738231AE
:1086600039F1232B59F4E0915807F0E0E859F94E1D
:10867000858590E083709070892BD1F080915807A8
:10868000E82FF0E0E859F94E94818C89981709F0A9
:10869000B2C295818D89981709F0ADC296818E89F5
:1086A000981709F0A8C297818F89981709F0A3C27B
:1086B000E0915807F0E0E859F94E858584FF52C0F3
:1086C0006C8D7D8D6115710509F44CC0CE01489605
:1086D0000E94833B80915807E82FF0E0E859F94E5B
:1086E00020858091C7152817E9F591858091C815D7
:1086F0009817C1F592858091C915981799F59385BA
:108700008091CA15981771F5288F8091C815898FA7
:108710008091C9158A8F8091CA158B8F8FA188236C
:10872000D1F42AA19CA18EA1981B822F86958695B3
:108730008695981B392F320F3AA38BA1282F2695A7
:108740002695821B97FD9195890F8BA336953695BB
:108750003695830F8CA381E08093DB158CA18EA3CB
:108760001D8E1C8E8DA1282F30E0C9018F70907056
:108770008430910509F4EFC1853091055CF48230B5
:10878000910591F1833091050CF0CAC0019709F071
:10879000C3C210C08630910509F425C28630910508
:1087A0000CF4FDC18730910509F425C2089709F042
:1087B000B3C2C6C18091DB1580FFAEC283E08DA33A
:1087C00080E48093DB151D8E1C8E2091C3153091A3
:1087D000C4152115310509F431C182E48093DB15FC
:1087E000C9010E941A3C2AC18091DB1580FF8DC00F
:1087F00080915807E82FF0E0E859F94E85858F738E
:10880000823109F082C0848590E0807F907081354C
:1088100091050CF44EC010925A0735C0F901E05C86
:10882000F94E84AD80936107882309F442C08130FA
:1088300021F44F5F40935A0726C08230C1F485ADC2
:108840008430A9F436AD20E087AD90E0822B932BE5
:10885000909363078093620724E0853C920710F0B1
:1088600084EC94E09F8F8E8F99A388A322C080917F
:108870005A07E82FF0E0E358F94EE081EE23C9F003
:10888000E80FE0935A0740915A07242F30E0E09117
:108890005807F0E0E859F94E848582958F7090E092
:1088A0000597880F991F880F991F281739070CF40F
:1088B000B5CF83E08DA3E0915807F0E0E859F94E79
:1088C00084818C8BE0915807F0E0E859F94E85815E
:1088D0008D8BE0915807F0E0E859F94E86818E8B38
:1088E000E0915807F0E0E859F94E87818F8B81E0DD
:1088F00090E00E941A3C82E48093DB151D8E1C8E52
:108900001092C4151092C31599C080E28093DB15B4
:108910000E94D279E091E215F091E31515A2E9CC1D
:1089200080915807E82FF0E0E859F94E858580FFDF
:1089300025C024FD23C08C8D9D8D892B09F0ECC1B1
:108940008091C3159091C41501960E941A3C209104
:10895000DB15822F80618093DB158091C315909188
:10896000C415892B19F022612093DB150E94D2795E
:1089700081E090E09D8F8C8F88E082C085FF25C0CC
:10898000328920E0838990E0282B392B8091E015F3
:108990009091E115820F931F9093E1158093E0155C
:1089A000E0915807F0E0E859F94E328920E08389D8
:1089B00090E0282B392B8091C3159091C415821B10
:1089C000930B9093C4158093C3152091C3153091D8
:1089D000C4152115310559F08DA184FD08C0809181
:1089E000DB1582608093DB15C9010E941A3CE0917F
:1089F0005807F0E0E859F94E968580E02785820F08
:108A0000911D909363078093620728A139A12817CD
:108A1000390710F0892B21F4309363072093620704
:108A200080916207909163079F8F8E8F8091DB15F5
:108A300090E083709070892B09F46EC11092431BF3
:108A40001092421B0E94D2798091DB15282F85FF5E
:108A50000CC01092431B1092421B1DA2E0915807BC
:108A6000F0E0E859F94E84E1CCC084FF12C01092C6
:108A7000431B1092421B81E090E09D8F8C8F84E01D
:108A80008DA31FA2E0915807F0E0E859F94E81E16B
:108A9000B8C08091421B9091431B892B01F120FFAC
:108AA00002C01D8E1C8E8C8D9D8D0097A1F42E8D85
:108AB0003F8D8091421B9091431B2817390720F46A
:108AC0003093431B2093421B8091421B9091431B88
:108AD0009D8F8C8F04C09093431B8093421B1FA2D9
:108AE0008091C5159091C6159093E1158093E0157E
:108AF0008091421B9091431B892B81F08C8D9D8D21
:108B0000009761F0CC969093C4158093C315E091C3
:108B10005807F0E0E859F94E88E110C08091DB1564
:108B200081FFFAC08CE390E09093C4158093C31545
:108B3000E0915807F0E0E859F94E80E1858768C078
:108B40008091DB1580FFE8C01DA280E18093DB15DA
:108B50000E94D279E1C08091C3159091C41500970D
:108B600011F00E941A3CE0915807F0E0E859F94EE4
:108B700085859091DB1580FF0BC090FF06C087E0D4
:108B80008DA31EA21D8E1C8E1DC086E08DA31AC053
:108B900090FF22C085E08DA31D8E1C8EBDC08091EC
:108BA000C3159091C415009711F00E941A3CE091F2
:108BB0005807F0E0E859F94E858580FF0DC087E041
:108BC0008DA31EA281E090E00E941A3C80E1809378
:108BD000DB150E94D2790FC08091C3159091C41506
:108BE000892B49F499C08091DB1580FF95C087E0FF
:108BF0008DA31EA291C0E0915807F0E0E859F94E0C
:108C000080E185878CE390E09093C4158093C31531
:108C1000E0915807F0E0E859F94E80E58487E0914B
:108C20005807F0E0E859F94E8C8980878D89818753
:108C30008E8982878F898387888D8483898D8583B8
:108C40008A8D86838B8D878386E0809346168889FC
:108C50009989918380838A899B8993838283A8E5FC
:108C6000B6E1FE0180E101900D928150E1F788E4C8
:108C700096E168E576E10E94D35D8DA1E091580709
:108C800084FF06C0F0E0E859F94E1786168607C043
:108C9000F0E0E859F94E84E0868784EC878780917C
:108CA000CA1C90E029E730E0829FF001839FF00D1D
:108CB000929FF00D1124E157F44E84818093471662
:108CC0008091C3159091C415889790934416809114
:108CD000C315885280934516E0915807F0E08F0144
:108CE0000859194ED80153961C92539752961C92CC
:108CF000F801118A108A0E94FB3C80959095F8013A
:108D0000918B808B80E680934016109241161092D2
:108D100043161092421608C01092C4151092C31543
:108D200010925807109257071092DB15DF91CF91E0
:108D30001F910F9108951F931091CA1C212F30E0AD
:108D400089E790E0289FF001299FF00D389FF00DF2
:108D50001124E157F44E8389882399F180915816A4
:108D60008E3F29F480915916803819F42AC08F3F1C
:108D700041F11092CA1C0BC088E596E10E945B4D40
:108D80008823C1F48091CA1C8F5F8093CA1C809194
:108D9000CA1C823088F327C00E949249892B51F463
:108DA0008091CA1C8F5F8093CA1C8091CA1C82303C
:108DB00098F31CC0809147168150809347168823F2
:108DC00029F41092C4151092C31516C080E496E1E0
:108DD000489660E840E00E94F25F892B69F081E0EC
:108DE0000E94B73D09C01092CA1CDFCF1092C41573
:108DF0001092C3151093CA1C1F910895EF92FF9211
:108E00000F931F93CF93DF938C017B01C0915B077E
:108E1000D0915C0721968DE7C030D80710F0C0E0F4
:108E2000D0E1CE010E94333C9C018091541B909173
:108E3000551B8217930771F380916D1B90916E1BE8
:108E40008217930739F3C0935B07D0935C071092A6
:108E50005A0720E049E150E01CC0322F3F5F822FCB
:108E600090E0849FF001859FF00D949FF00D1124F8
:108E7000EC5BF44E80899189892B51F420935A0739
:108E800089E1289FD0011124AC5BB44E49F434C071
:108E9000232F223010F320935A07A0E0B0E02CC01B
:108EA0005096DC9350975196CC9351975396FC92E1
:108EB000EE9252970115110531F480E1ED011992FE
:108EC0008A95E9F707C0ED01F80180E10190099268
:108ED0008150E1F78091CA1C90E029E730E0829F41
:108EE000F001839FF00D929FF00D1124E157F44E95
:108EF000848154968C935497CD01DF91CF911F912B
:108F00000F91FF90EF9008950F930E94C2630E940B
:108F1000344F80E009C0E82FF0E0EE0FFF1FE45C63
:108F2000F94E118210828F5F8230A8F320E04CE26C
:108F300050E00DC0822F90E0849FF001859FF00DDE
:108F4000949FF00D1124EC51FA4E15A22F5F2230A0
:108F500088F380E094E090935C0780935B0720E0C7
:108F600049E150E00EC0822F90E0849FF001859F80
:108F7000F00D949FF00D1124EC5BF44E118A108AD1
:108F80002F5F223080F320935A070F910895CF92DC
:108F9000DF92EF92FF920F931F93CF93DF93D82E20
:108FA000C62E79018A0110925807A4E6B7E0E8E5D9
:108FB000F6E180E101900D928150E1F78091C315B7
:108FC0009091C415C0969093C4158093C315815099
:108FD000954030F080E095E09093C4158093C315E0
:108FE00060E476E14091C3155091C4154053504060
:108FF000CB01C0960E94237F80E68093401610929A
:10900000411610924316109242168AE38093461638
:109010008091CA1C90E029E730E0829FF001839F95
:10902000F00D929FF00D1124E157F44E848180934E
:1090300047168091481690914916892B51F58091D9
:109040004A1690914B16892B21F580914C169091E0
:109050004D16892BF1F480914E1690914F16892B65
:10906000C1F48091501690915116892B91F4809102
:10907000521690915316892B61F480915416909159
:109080005516892B31F48091561690915716892BDD
:10909000D1F0E8E5F6E1DF01509780E10D90019213
:1090A0008150E1F7809164078F3F91F484E0D816F6
:1090B00051F422E0C21639F488E496E164E677E0E0
:1090C0000E94D35D0EC01092C4151092C31535C016
:1090D000A8E4B6E1E4E6F7E080E101900D9281506A
:1090E000E1F7E0915807CE2FD0E0FE01E859F94EA4
:1090F000D082C182C801B7010E941F3DC459D94E18
:10910000688379838A839B838091C3159091C4156A
:10911000889790934416889688528093451680913C
:109120005807C82FD0E0C859D94E1B821A820E9416
:10913000FF3C809590959B838A83DF91CF911F910F
:109140000F91FF90EF90DF90CF90089540E456E1AB
:109150008091CA1C90E029E730E0829FF001839F54
:10916000F00D929FF00D1124E157F44E848180930D
:109170004716809158168F3F81F4DA015896FA010C
:10918000389680E101900D928150E1F788E496E1F4
:1091900068E576E10E94D35D1BC0A4E6B7E0FA0162
:1091A000389680E101900D928150E1F7E8E4F6E114
:1091B000DF01509680E10D9001928150E1F7A8E522
:1091C000B6E1E4E6F7E080E101900D928150E1F72D
:1091D00060915807662301F18AE38093461670E098
:1091E0004091C3155091C415461B570B5093C4159D
:1091F0004093C3154852504050934416485D5F4F0A
:10920000842F8852809345166459794E4C525040B1
:109210008CE696E10E94237F1092580781E88093A4
:1092200068161092691610926B1610926A160E94B8
:10923000FF3C8095909590936B1680936A160895E5
:109240002091CA1C30E040E0ABE0B0E086E190E065
:10925000289FB001299F700D389F700D11240FC0F9
:10926000842F90E08A9FF0018B9FF00D9A9FF00D64
:109270001124E60FF71FE458F74F12864F5F423074
:1092800078F3409330090895CF93DF93DC01109277
:10929000360910923509109230095091CA1C252FB9
:1092A00030E040E0CBE0D0E086E190E0289FB001E4
:1092B000299F700D389F700D112429C0842F90E0D4
:1092C0008C9FF0018D9FF00D9C9FF00D1124E60FF7
:1092D000F71FE458F74F82858823C1F08081918180
:1092E0008A179B0799F4409330098BE0489FC0018F
:1092F000112426E1529F90011124820F931F84585C
:10930000974F909336098093350905C04F5F4230DF
:10931000A8F2409330098091350990913609DF9188
:10932000CF9108950F931F93CF93DF931092360937
:1093300010923509109230099091CA1C292F30E003
:1093400086E1989FD001112440E050E060E00BE0FE
:1093500010E086E190E0289FE001299FD00D389F22
:10936000D00D11242BE035C0862F90E0809FF001B6
:10937000819FF00D909FF00D1124EC0FFD1FE4581C
:10938000F74F8285882321F10190F081E02D3097FD
:10939000F9F0818D882311F0853059F4411551057C
:1093A000B9F4629FA00111244A0F5B1F4458574F24
:1093B0000FC0609330098BE0689FC00111248A0FB1
:1093C0009B1F8458974F909336098093350909C0A5
:1093D0006F5F623048F250933609409335096093CD
:1093E00030098091350990913609DF91CF911F9115
:1093F0000F910895FC0112860190F081E02D818D7E
:10940000853009F413A60895FC0181A18D7F81A305
:1094100008952091CA1C84E4289F900111242855A6
:10942000374FC90108956F927F928F929F92AF92AA
:10943000BF92CF92DF92EF92FF920F931F93CF9341
:10944000DF9310923609109235099091CA1C292F8A
:1094500030E086E1989FE001112440E050E060E0B8
:109460000BE010E086E190E0289FD001299FB00D2D
:10947000389FB00D11242BE018C0862F90E0809FFC
:10948000F001819FF00D909FF00D1124EA0FFB1F5A
:10949000E458F74F8285813039F4629FA00111248E
:1094A0004C0F5D1F4458574F6F5F623030F350933D
:1094B00036094093350910923409109233091092FD
:1094C00030098CE2A82EB12C04E8C02ED12C1CE26D
:1094D000712EB4E86B2EA2E08A2EF9E7EF2EF12C64
:1094E000E4E09E2EBEC05091CA1C252F30E0842F90
:1094F00090E08A9DF0018B9DF00D9A9DF00D112456
:109500002C9DC0012D9D900D3C9D900D1124E80FC8
:10951000F91FEC58F84F83A5813009F09DC0479D95
:10952000E0011124569DC0011124C80FD91FCC5849
:10953000D84FD0933409C0933309898D8130E9F035
:10954000813030F0833039F1843009F085C035C086
:109550008AA5833010F013A67FC0CE0182960E94A8
:109560009065892B09F478C04091330950913409F2
:1095700080E090E060E070E03EC0CE014A960E943C
:109580009065892B09F468C0E0913309F0913409A2
:10959000818E12A661C0CE014A960E949065892BE9
:1095A00009F45AC0E0913309F0913409918E12A662
:1095B00080E090E0BF01AF011EC08AA5833070F04B
:1095C0001AA6CE010E94444990933609809335092A
:1095D000009711F00E94FA491BA63EC0CE01829668
:1095E0000E949065892BC1F1409133095091340953
:1095F00080E090E0BA010E949B55009133091091E0
:1096000034098091CA1C90E08E9DF0018F9DF00D71
:109610009E9DF00D1124E157F44E65857685878572
:10962000908928EE33E040E050E00E948581CA0135
:10963000B90128EE33E040E050E00E944781AB01E1
:10964000BC01C80182960E94AA65E0913309F0919D
:10965000340982A58F5F82A7809130098F5F809344
:10966000300940913009433008F43DCF109232095F
:109670001092310981E080933009C4E4D0E002E225
:1096800014E440C05091CA1C252F30E0842F90E094
:10969000FC0175E0EE0FFF1F7A95E1F7880F991F27
:1096A000E80FF91F2C9FC0012D9F900D3C9F900D3E
:1096B0001124E80FF91FE753F74F808181FF1DC088
:1096C000409FF0011124519FC0011124E80FF91FA0
:1096D000E855F74FF0933209E093310981A180FDFD
:1096E0000CC0CF0141960E949065892B31F080918A
:1096F0003109909132090E94044A809130098F5FAC
:109700008093300940913009423008F4BBCFDF919B
:10971000CF911F910F91FF90EF90DF90CF90BF906E
:10972000AF909F908F907F906F900895AF92BF926F
:10973000CF92DF92EF92FF920F931F93CF93DF931D
:10974000182FB92EA62E69017A01109232091092B3
:10975000310981E0809330098091CA1C90E041E09A
:1097600024E430E0829FB001839F700D929F700DC2
:10977000112419C0242F2F5F842F90E0FC0155E0A5
:10978000EE0FFF1F5A95E1F7880F991FE80FF91F99
:10979000E60FF71FE753F74F808181FD03C0409329
:1097A00030090CC0422F423028F340933009423038
:1097B00029F40E94BC7E81E08093300990913009A9
:1097C00082E2989FF00111248091CA1C24E4829FB8
:1097D000C0011124E80FF91FE855F74FF093320943
:1097E000E0933109EF01212F3B2DC901DC0180E11C
:1097F0000D9009928150E1F7A08AC114D104E104CF
:10980000F10469F0CF014196B701A6010E94AA6553
:10981000E0913109F091320981A18E7F02C081A1CE
:10982000816081A32091CA1C30E060913009862FAD
:1098300090E0FC01B5E0EE0FFF1FBA95E1F7880F4D
:10984000991FE80FF91F84E490E0289FA001299F49
:10985000500D389F500D1124E40FF51FE753F74FBB
:1098600080818260808300FF13C0862F90E0FC011E
:1098700075E0EE0FFF1F7A95E1F7880F991FE80F4B
:10988000F91FE40FF51FE753F74F8081846012C082
:10989000862F90E0FC0135E0EE0FFF1F3A95E1F7CF
:1098A000880F991FE80FF91FE40FF51FE753F74FD3
:1098B00080818B7F80838091310990913209DF9183
:1098C000CF911F910F91FF90EF90DF90CF90BF90BD
:1098D000AF900895EF92FF920F931F93CF93DF9372
:1098E000EC017A018B011092360910923509109221
:1098F00030092091CA1C30E040E0ABE0B0E086E1E6
:1099000090E0289FB001299F700D389F700D1124A1
:1099100016C0242F2F5F842F90E08A9FF0018B9F29
:10992000F00D9A9FF00D1124E60FF71FE458F74F42
:109930008285882319F4409330090FC0422F4230AA
:1099400040F340933009423041F40E94BC7E62E013
:1099500070E00E94728180933009E09130098BE0C1
:10996000E89FF00111248091CA1C26E1829FC0016A
:109970001124E80FF91FE458F74FF0933609E093EC
:109980003509C193D193CF01B801A7010E94AA65FF
:109990002091300930E04091CA1C50E08BE090E00B
:1099A000289FF001299FF00D389FF00D112486E1CA
:1099B00090E09C01429FC001439F900D529F900DEB
:1099C0001124E80FF91FE458F74F81E08287809156
:1099D000350990913609DF91CF911F910F91FF903A
:1099E000EF900895EF92FF920F931F93CF93DF9321
:1099F0007C011092320910923109109230090091C5
:109A0000CA1C202F30E084E490E0289FE001299FC9
:109A1000D00D389FD00D11243EC0812F90E0FC0165
:109A2000B5E0EE0FFF1FBA95E1F7880F991FE80F19
:109A3000F91FEC0FFD1FE753F74F808181FF28C00E
:109A4000212F30E0C90175E0880F991F7A95E1F761
:109A5000220F331F820F931F8C0F9D1F8855974F26
:109A6000B70140E150E00E940D7F009789F482E247
:109A7000189FC001112424E4029F90011124820F39
:109A8000931F8855974F909332098093310908C0EE
:109A90001F5F1093300910913009123008F4BDCFC8
:109AA0008091310990913209DF91CF911F910F91EF
:109AB000FF90EF900895EF92FF921F93CF93DF9363
:109AC0007C01109230098091CA1C90E024E430E0BF
:109AD000829FE001839FD00D929FD00D112442C040
:109AE000812F90E0FC01B5E0EE0FFF1FBA95E1F782
:109AF000880F991FE80FF91FEC0FFD1FE753F74F71
:109B0000808181FF2CC0212F30E0C90175E0880FD2
:109B1000991F7A95E1F7220F331F820F931F8C0F45
:109B20009D1F212F30E0F90155E0EE0FFF1F5A95E0
:109B3000E1F7220F331FE20FF31FEC0FFD1FE85573
:109B4000F74F40894695469546958855974FB701FA
:109B500050E00E940D7F009711F481E009C01F5F63
:109B60001093300910913009123008F4B9CF80E019
:109B7000DF91CF911F91FF90EF900895AF92BF9228
:109B8000CF92DF92EF92FF920F931F93CF93DF93C9
:109B90006C0110923409109233091092300900912F
:109BA000CA1C202F30E01CE2A12EB12C84E890E0EA
:109BB000289F7001299FF00C389FF00C1124E901B7
:109BC000CF51DA4F2FC0812F90E08A9D90018B9D5D
:109BD000300D9A9D300D11242E0D3F1DF901EC58CA
:109BE000F84F83A58823D9F04881C9018C57984F35
:109BF000B60150E00E940D7F009789F48CE2189F17
:109C0000C001112424E8029F90011124820F931FA8
:109C10008C58984F909334098093330907C01F5F85
:109C20001093300910913009133068F28091330994
:109C300090913409DF91CF911F910F91FF90EF9098
:109C4000DF90CF90BF90AF900895CF92DF92EF92C8
:109C5000FF920F931F93CF93DF937C0110923409EF
:109C600010923309109230090091CA1C202F30E065
:109C70008CE2C82ED12C84E890E0289FE001299F37
:109C8000D00D389FD00D11242CC0812F90E08C9DD9
:109C9000F0018D9DF00D9C9DF00D1124EC0FFD1F2A
:109CA000EC58F84F83A58823C9F0CF01B70140E1F4
:109CB00050E00E940D7F009789F48CE2189FC0014C
:109CC000112424E8029F90011124820F931F8C58C5
:109CD000984F909334098093330907C01F5F109306
:109CE000300910913009133080F28091330990913E
:109CF0003409DF91CF911F910F91FF90EF90DF908A
:109D0000CF900895EF92FF920F931F93CF93DF931D
:109D1000182F092FEB01F42EE22E10923409109225
:109D20003309109230092091CA1C30E040E0ACE2C7
:109D3000B0E084E890E0289FB001299F700D389F23
:109D4000700D112416C0242F2F5F842F90E08A9F5E
:109D5000F0018B9FF00D9A9FF00D1124E60FF71F75
:109D6000EC58F84F83A5882319F4409330090FC0AD
:109D7000422F433040F340933009433041F40E9476
:109D8000BC7E63E070E00E94728180933009409154
:109D9000CA1C909130098CE2989FB001112484E88C
:109DA000489FC0011124680F791F6C58784F709339
:109DB000340960933309DB01212F302FC901FC01E5
:109DC00080E101900D928150E1F7E42FF0E02097BF
:109DD000B9F010923009EF51FA4F408190E00BC07A
:109DE000E92FF0E0DB01AE0FBF1FEC0FFD1F8081FC
:109DF00050968C939F5F941798F3909330090CC002
:109E0000EF51FA4F40819B01205F3F4FC90160E055
:109E100070E050E00E94357FE0913309F091340901
:109E2000F08EE18ECF014A9640E050E060E070E0B5
:109E30000E94AA658091330990913409829640E08E
:109E400050E060E070E00E94AA65E0913309F09173
:109E5000340912A681E083A7CF01DF91CF911F9132
:109E60000F91FF90EF9008953091CA1C432F50E05E
:109E700020E0ACE2B0E084E890E0489FB001499F68
:109E8000700D589F700D11240FC0822F90E08A9F93
:109E9000F0018B9FF00D9A9FF00D1124E60FF71F34
:109EA000EC58F84F13A62F5F233078F320E0ABE097
:109EB000B0E086E190E0489FB001499F700D589F47
:109EC000700D11240FC0822F90E08A9FF0018B9FAC
:109ED000F00D9A9FF00D1124E60FF71FE458F74F8D
:109EE00012862F5F223078F320E084E490E0489FD0
:109EF000B001499F700D589F700D112414C0822F1E
:109F000090E0FC01B5E0EE0FFF1FBA95E1F7880F76
:109F1000991FE80FF91FE60FF71FE753F74F8081EE
:109F20008D7F80832F5F223050F32093300989E7A3
:109F300090E0489FF001499FF00D589FF00D1124CB
:109F4000E157F44E8589882361F184E490E0489FCD
:109F5000D001499FB00D589FB00D1124FD01E85567
:109F6000F74F8EEF90E891838083138212821582DF
:109F70001482178216821186108613861286158621
:109F800014861786168680E4808BA753B74F8C9172
:109F900083608C93832F44E650E060E070E00E9481
:109FA00043670895AF92BF92CF92DF92EF92FF92F4
:109FB0000F931F93CF93DF93809147168F3F09F044
:109FC000A5C4809148168E3F09F0A0C4809149161F
:109FD000803809F09BC480915807A82FB0E0FD019C
:109FE000E859F94E8181882309F090C4A459B94EEB
:109FF0004C91442379F08091CA1C90E029E730E02D
:10A00000829FF001839FF00D929FF00D1124E15784
:10A01000F44E4483E0915807F0E0E459F94EA480EF
:10A02000B580C680D780A114B104C104D10409F45D
:10A0300048C02091CA1C30E04D2D55276627772750
:10A04000BA2DAA2799278827482B592B6A2B7B2BB7
:10A05000D601C50180709070B070892F9A2FAB2FF8
:10A06000BB27482B592B6A2B7B2BC501A0E0B0E006
:10A070008070A070B070BA2FA92F982F8827482B16
:10A08000592B6A2B7B2B89E790E0289FE001299FC1
:10A09000D00D389FD00D1124C157D44E8D819E8193
:10A0A000AF81B88584179507A607B70751F04D8390
:10A0B0005E836F8378870E947D5E69877A878B874E
:10A0C0009C87E0915807F0E0E459F94EA084B184F0
:10A0D000C284D384A114B104C104D104C9F1809114
:10A0E000CA1C90E029E730E0829FF001839FF00DC9
:10A0F000929FF00D1124E157F44E2D2D3327442764
:10A100005527BA2DAA2799278827282B392B4A2B80
:10A110005B2BD601C50180709070B070892F9A2F8B
:10A12000AB2FBB27282B392B4A2B5B2BC501A0E07B
:10A13000B0E08070A070B070BA2FA92F982F882738
:10A14000282B392B4A2B5B2B258736874787508B4B
:10A15000109239091092380910923B0910923A096D
:10A1600040E009C0E42FF0E0EE0FFF1FE45CF64F83
:10A17000118210824F5F4230A8F3409348098CE06F
:10A18000809337096091C3157091C41539C0F901E6
:10A19000E05CF94E8181882309F4B6C38081833065
:10A1A00071F0853039F08130D9F4F0933909E093BA
:10A1B000380916C0F0933B09E0933A0911C0809129
:10A1C0003C0990913D09892B19F4E0E040E0AFC3D0
:10A1D00080913E0990913F09892B09F4A6C342E082
:10A1E00080913709E0915807F0E0E05CF94EE80F04
:10A1F000F11D95A5990F990F990F980F9093370915
:10A200009091580780913709282F30E0290F311D90
:10A21000245D3F4F2617370708F4B9CF409348090C
:10A22000E0913A09F0913B09309709F441C0E4808C
:10A23000F580068117818091CA1C90E029E730E003
:10A24000829FF001839FF00D929FF00D1124E15742
:10A25000F44E212F332744275527BE2DAA279927AF
:10A260008827282B392B4A2B5B2BD801C7018070FC
:10A270009070B070892F9A2FAB2FBB27282B392BCA
:10A280004A2B5B2B00E010E080E09FEFA0E0B0E005
:10A29000E822F9220A231B23102F0F2DFE2CEE2477
:10A2A0002E293F29402B512B208331834283538316
:10A2B0001092480962C22481358146815781E08429
:10A2C000F18402851385A52EBB24CC24DD24B22F76
:10A2D000AA2799278827A82AB92ACA2ADB2ADA01B5
:10A2E000C90180709070B070892F9A2FAB2FBB2757
:10A2F000A82AB92ACA2ADB2A40E050E02070407020
:10A300005070542F432F322F2227A22AB32AC42A57
:10A31000D52A212F332744275527BE2DAA27992731
:10A320008827282B392B4A2B5B2BD801C70180703B
:10A330009070B070892F9A2FAB2FBB27282B392B09
:10A340004A2B5B2B00E010E080E09FEFA0E0B0E044
:10A35000E822F9220A231B23102F0F2DFE2CEE24B6
:10A360002E293F29402B512BA216B306C406D50631
:10A3700008F4FEC180898E3F21F48189803809F478
:10A38000F7C1838187FFC7C0CF0140960E94F24C7E
:10A39000EC019093430980934209E09148090097AA
:10A3A00009F05DC0F0E0EE0FFF1FE45CF64FC081E6
:10A3B000D181AC80BD80CE80DF80A114B104C10406
:10A3C000D10409F4A8C08E01005F1F4F9FEFA916AA
:10A3D0009FEFB9069FEFC9069FEFD90691F16D2D4A
:10A3E0007727882799275A2D442733272227622B3E
:10A3F000732B842B952BA601950120703070507023
:10A40000232F342F452F5527622B732B842B952B0D
:10A41000950140E050E0207040705070542F432F61
:10A42000322F2227622B732B842B952B28EE33E0BF
:10A4300040E050E00E9447819B01AC01C8016A8165
:10A4400006C0C8016A8120E030E040E050E000E052
:10A450000E94964B90934309809342095CC0F0E0C0
:10A46000EE0FFF1FE45CF64F0190F081E02DA48019
:10A47000B580C680D780A114B104C104D10451F0C5
:10A48000AFEFAA16AFEFBA06AFEFCA06AFEFDA0624
:10A4900041F403C00E94044A3EC089A1816089A39F
:10A4A0003AC06D2D7727882799275A2D44273327BF
:10A4B0002227622B732B842B952BA60195012070EC
:10A4C00030705070232F342F452F5527622B732B5C
:10A4D000842B952B950140E050E020704070507027
:10A4E000542F432F322F2227622B732B842B952B33
:10A4F00028EE33E040E050E00E944781AB01BC0110
:10A50000CE0141960E94AA65E0914209F09143096B
:10A5100081A18E7F81A3E0914809F0E0EE0FFF1F3B
:10A52000E45CF64F0190F081E02D838186FF20C12D
:10A5300084819581A681B7810097A105B10509F4B1
:10A5400017C1CF014096628141E00E94F25FEC01A9
:10A550009093470980934609E0914809009709F4D0
:10A56000B5C0F0E0EE0FFF1FE45CF64F0190F08104
:10A57000E02D24813581468157812F3FBFEF3B0776
:10A58000BFEF4B07BFEF5B0709F49DC0A52EBB24AF
:10A59000CC24DD24B22FAA2799278827A82AB92AF4
:10A5A000CA2ADB2ADA01C90180709070B070892F45
:10A5B0009A2FAB2FBB27A82AB92ACA2ADB2AC9019E
:10A5C000A0E0B0E08070A070B070BA2FA92F982FD3
:10A5D0008827A82AB92ACA2ADB2A21E2A2162CE156
:10A5E000B20620E0C20620E0D206A0F4CE014196D9
:10A5F0000E947A657B018C01C601B50128EE33E02B
:10A6000040E050E00E944781E616F7060807190768
:10A6100008F048C0E0914809F0E0EE0FFF1FE45C4D
:10A62000F64F0190F081E02DE480F58006811781DE
:10A63000C0904609D0904709612F7727882799272E
:10A640005E2D442733272227622B732B842B952BD7
:10A65000A8019701207030705070232F342F452FA0
:10A660005527622B732B842B952B00E010E020E004
:10A670003FEF40E050E0E222F32204231523102FA5
:10A680000F2DFE2CEE246E297F29802B912B28EE96
:10A6900033E040E050E00E944781AB01BC01C601BD
:10A6A000419609C08091460990914709419640E042
:10A6B0005DED6DE670E00E94AA65E0914609F091BB
:10A6C0004709118E55C081E0898F52C0F0E0EE0F2E
:10A6D000FF1FE45CF64FC081D181AC80BD80CE808D
:10A6E000DF808E01005F1F4F3FEFA3163FEFB306E1
:10A6F0003FEFC3063FEFD30691F16D2D77278827F3
:10A7000099275A2D442733272227622B732B842B1A
:10A71000952BA6019501207030705070232F342F97
:10A72000452F5527622B732B842B952B950140E0E9
:10A7300050E0207040705070542F432F322F22274A
:10A74000622B732B842B952B28EE33E040E050E0F6
:10A750000E9447819B01AC01C8016A8106C0C80103
:10A760006A8120E030E040E050E001E00E94C461F6
:10A77000809148098F5F80934809E0914809E23051
:10A7800058F4F0E0EE0FFF1FE45CF64F0190F0810B
:10A79000E02D309709F08FCD88E496E10E94254E98
:10A7A000FC019093410980934009609138097091B0
:10A7B00039096115710509F43FC0009769F46E5FAE
:10A7C0007F4F88E496E141E022E00E94824E909320
:10A7D00041098093400930C0818D882311F482E0C3
:10A7E000818F00913809109139090E5F1F4FC09178
:10A7F0004009D09141096096E091CA1CF0E0EF5108
:10A80000FA4FE080C801BE014E2D50E00E940D7F3E
:10A81000009761F0CE01B8014E2D50E00E941A7FE2
:10A82000E0914009F091410982E0818FE091400977
:10A83000F091410981E0808FE0915807F0E0E45900
:10A84000F94E82819381E0914009F0914109892B71
:10A8500009F44CC0309769F488E496E160E070E058
:10A8600041E025E00E94824E909341098093400987
:10A8700002C081E0808F80914009909141090E943F
:10A880004449DC019093450980934409E0915807BD
:10A890000097B9F4F0E0E459F94E9281838128EEF3
:10A8A00033E0829FA001839F500D929F500D112491
:10A8B00060E070E080914009909141090E946A4CEB
:10A8C00025C0F0E0E459F94E9281838128EE33E00F
:10A8D000829FA001839F500D929F500D112460E034
:10A8E00070E0CD0102960E94AA6510C0309771F009
:10A8F000CF010E94444990934509809344090097F1
:10A9000029F00E94FA4902C0409348091092C415E8
:10A910001092C315DF91CF911F910F91FF90EF908F
:10A92000DF90CF90BF90AF900895E1E041E0F0E07C
:10A93000EE0FFF1FE45CF64F205C394E318320831D
:10A940004FCCEF92FF920F931F93DF93CF9300D0E2
:10A95000CDB7DEB7E091CA1CF0E0EF51FA4F20818D
:10A96000822F90E00296022F0E5F87709070081B76
:10A97000892B09F0085F80E496E120E620934016D9
:10A980001092411610924316109242162AE3209319
:10A9900046162FEF20934716FC0178962FEF32E0F2
:10A9A00030935916209358161382128215821482FE
:10A9B00017821682118610861386128615861486D3
:10A9C00020E032E0378726870896BF010E94D35DDA
:10A9D00020915807A22FB0E0FD01E859F94E85E813
:10A9E00080831182FD01E459F94E10821182128296
:10A9F0001382109244168091481690914916892B23
:10AA000099F580914A1690914B16892B69F58091A2
:10AA10004C1690914D16892B39F580914E169091D8
:10AA20004F16892B09F58091501690915116892B5C
:10AA3000D9F48091521690915316892BA9F48091E4
:10AA4000541690915516892B79F480915616909151
:10AA50005716892B49F488E080934516D096B09319
:10AA6000C415A093C3154EC0E02EFF24822F90E0A2
:10AA7000C0968E0D9F1D9093C4158093C315085FDB
:10AA8000009345160850A059B94EB0933909A093C8
:10AA9000380981E08C9306950695069511960C93DE
:10AAA00011972091CA1C129630E0F901EF51FA4F2C
:10AAB000408153E0220F331F5A95E1F725533A4E58
:10AAC000CD01B90150E00E941A7FE091CA1CF0E06C
:10AAD000EF51FA4F808190E09701281B390B2250EB
:10AAE00030403A83298320913809309139092E5F0B
:10AAF0003F4F280F391FC90160E070E049815A813A
:10AB00000E94357F80915807082F10E00859194E90
:10AB1000F801138212820E94FF3C80959095F80103
:10AB2000938382830F900F90CF91DF911F910F91AC
:10AB3000FF90EF900895FF920F931F93CF93DF93B1
:10AB40008C01EA01E091CA1CF0E0EF51FA4F20813C
:10AB5000822F90E00296E2E0FE2EF20E8770907057
:10AB6000F81A892B11F088E0F80E1092580780E649
:10AB7000809340161092411610924316109242167E
:10AB80008AE3809346169FEF90934716E8E5F6E137
:10AB900061157105B9F49093581682E08183138290
:10ABA00012821582148217821682118610861286EE
:10ABB00081E0838794878D8585878E859F8597879C
:10ABC000868707C0DF01FB0180E101900D92815073
:10ABD000E1F787E8809368161092691610926C1658
:10ABE00010926D1610926E1610926F16A0E7B6E1D5
:10ABF000FE0180E101900D928150E1F71092441620
:10AC0000CE0160E840E00E94F25F892B09F05FC04E
:10AC10000115110549F0A8E4B6E1F80180E10190C1
:10AC20000D928150E1F706C088E496E168E576E18F
:10AC30000E94D35D88E1F80EF092451688EEF80E7A
:10AC40000F2D10E0005C1F4F1093C4150093C31527
:10AC500000541040E0915807F0E0E058F94EF093AE
:10AC60003909E093380981E08083F694F694F694EC
:10AC7000F1822091CA1C329630E0D901AF51BA4F0F
:10AC80004C9163E0220F331F6A95E1F725533A4E4A
:10AC9000CF01B90150E00E941A7FE091CA1CF0E098
:10ACA000EF51FA4F808190E0081B190B02501040C1
:10ACB00020913809309139092E5F3F4F280F391FF5
:10ACC000C90160E070E0A8010E94357F29C01092A0
:10ACD00049161092481610924B1610924A1610926E
:10ACE0004D1610924C1610924F1610924E1610924E
:10ACF000511610925016109253161092521610922E
:10AD0000551610925416109257161092561688E146
:10AD10008093451680E490E09093C4158093C3150A
:10AD200080915807C82FD0E0C859D94E1B821A828B
:10AD30000E94FF3C809590959B838A83DF91CF9101
:10AD40001F910F91FF900895CF92DF92EF92FF92A3
:10AD50000F931F93CF93DF9390915807E92FF0E063
:10AD6000DF01A459B94EEC90809147168F3F09F04E
:10AD700042C1E859F94E8181882309F03CC11496FB
:10AD80008C9114978F3F09F436C110E4C12ECE2068
:10AD9000E6FE05C0809158168F3F09F42CC184E16E
:10ADA000809337091092390910923809C091C31560
:10ADB000D091C41540E050E064E1292F30E0245DDB
:10ADC0003F4F0FC0FC01E05CF94E9181992309F4DB
:10ADD0000CC18081823009F4AF01990F990F990F4E
:10ADE000690FC901860F911D8C179D0758F3509369
:10ADF00039094093380960933709CD01049660E81A
:10AE000040E00E94F25FFC0190934709809346095D
:10AE1000009761F08089882309F0EDC08091580780
:10AE200090E08059994E0E946960E5C08091580772
:10AE300090E08059994E0E94254EEC019093410973
:10AE400080934009009709F4D6C000913809109109
:10AE500039090115110511F4FF240FC0BC01605F11
:10AE60007F4FE091CA1CF0E0EF51FA4F4081C801DA
:10AE7000029650E00E940D7FF82EF0E8DF2EDE20D3
:10AE8000898D882309F041C00115110509F4B3C06B
:10AE9000BE01605F7F4FE091CA1CF0E0EF51FA4FB6
:10AEA000408198012E5F3F4FCB01B90150E00E94D5
:10AEB0001A7FC0914009D0914109CC2019F181E05D
:10AEC000898F8091CA1C90E029E730E0829FF001D1
:10AED000839FF00D929FF00D1124E157F44E618590
:10AEE00072858385948528EE33E040E050E00E942F
:10AEF00047810E948581CE014A96BA01A9010E942C
:10AF0000AA656DC082E0898F6AC0E5FC08C0FF2099
:10AF100031F0813009F06FC082E0898F6CC001157B
:10AF2000110589F0BE01605F7F4FE091CA1CF0E01F
:10AF3000EF51FA4F408198012E5F3F4FCB01B9018D
:10AF400050E00E941A7FCC2041F1009140091091FD
:10AF5000410981E0F801818F8091CA1C90E029E7C6
:10AF600030E0829FF001839FF00D929FF00D11243D
:10AF7000E157F44E618572858385948528EE33E030
:10AF800040E050E00E9447810E948581C8014A96B6
:10AF9000BA01A9010E94AA650EC08091380990915A
:10AFA0003909892B41F0FF2031F0E0914009F091FF
:10AFB000410982E0818FE0914009F0914109808D43
:10AFC000882369F0DD2059F4CF010E944449909311
:10AFD000450980934409009711F00E94FA49E091D5
:10AFE0004009F0914109D08E06C050933909409331
:10AFF0003809609337091092C4151092C315DF9178
:10B00000CF911F910F91FF90EF90DF90CF90089517
:10B01000DF92EF92FF920F931F93CF93DF93809174
:10B0200047168F3F09F02DC280915807482F50E0F6
:10B03000FA01E459F94E84818F3F09F422C2FA01E2
:10B04000E859F94E8181882309F01BC21092390911
:10B050001092380984E180933709C091C315D091CB
:10B06000C41520E030E064E1FA01BC9611C0DC01B7
:10B07000A05CB94E11969C911197992309F4FBC1DC
:10B080008C91813009F49D01990F990F990F690FE7
:10B09000CF01860F911D8C179D0748F32093380927
:10B0A0003093390960933709232B09F46FC08091DD
:10B0B000481690914916892B59F580914A1690911E
:10B0C0004B16892B29F580914C1690914D16892BA2
:10B0D000F9F480914E1690914F16892BC9F4809106
:10B0E000501690915116892B99F480915216909197
:10B0F0005316892B69F48091541690915516892B1B
:10B1000039F48091561690915716892B09F4B9C1DC
:10B1100088E496E10E94254E8C019093410980932A
:10B1200040096091380970913909009749F46E5FC0
:10B130007F4F88E496E140E022E00E94824E26C0E4
:10B1400092E0E92EF12CE60EF71EE8016096E09100
:10B15000CA1CF0E0EF51FA4FD080C701BE014D2D5F
:10B1600050E00E940D7F009759F0CE01B7014D2DA0
:10B1700050E00E941A7FE0914009F091410904C01B
:10B18000F801818D882311F482E0818F8091580726
:10B1900090E08059994E60E840E00E94F25F909301
:10B1A000470980934609892B09F46BC180914816A1
:10B1B00090914916892B09F073C080914A1690919D
:10B1C0004B16892B09F06CC080914C1690914D164E
:10B1D000892B09F065C080914E1690914F16892BEE
:10B1E00009F05EC08091501690915116892B09F09C
:10B1F00057C08091521690915316892B09F050C078
:10B200008091541690915516892B09F049C0809170
:10B21000561690915716892B09F042C088E596E1A1
:10B220000E945760882309F42CC1E0914609F091EF
:10B2300047098089882361F18FEF92E09093591636
:10B240008093581610925B1610925A1610925D1643
:10B2500010925C1610925F1610925E161092611694
:10B260001092601610926316109262161092651674
:10B270001092641680E091E09093671680936616B2
:10B2800088E496E168E576E10E94D35D30E253C040
:10B290008091580790E08059994E0E946960F1C0F2
:10B2A00088E496E160E840E00E94F25F892B09F0B3
:10B2B000E8C088E596E10E9457608823B9F0E8E588
:10B2C000F6E1DF01509780E10D9001928150E1F7A6
:10B2D00080915807E82FF0E0A8E4B6E1E059F94E74
:10B2E00080E101900D928150E1F724C088E596E15C
:10B2F00060E840E00E94F25F2091460930914709E2
:10B300002817390709F0BDC0E8E5F6E1DF015097DD
:10B3100080E10D9001928150E1F780915807E82F6C
:10B32000F0E0A8E4B6E1E059F94E80E101900D9219
:10B330008150E1F730E6109258078091CA1CA82F7F
:10B34000B0E089E790E0A89FF001A99FF00DB89FB9
:10B35000F00D1124E157F44E838981113068AF510B
:10B36000BA4F2C91822F90E00296422F4E5F877049
:10B370009070481B892B09F0485F80E68093401647
:10B3800010924116109243161092421610924416D3
:10B39000485E4093451648518AE3809346168FEFE6
:10B3A0008093471688E88093681610926916309348
:10B3B0006C16A0E7B6E12091460930914709C90112
:10B3C000FC0180E101900D928150E1F7042F10E023
:10B3D000005C1F4F1093C4150093C3150054104018
:10B3E000E0915807F0E0E058F94EF0933909E09306
:10B3F000380982E0808346954695469541832091A1
:10B40000CA1C329630E0D901AF51BA4F4C9183E05B
:10B41000220F331F8A95E1F725533A4ECF01B90128
:10B4200050E00E941A7FE091CA1CF0E0EF51FA4F01
:10B43000808190E0081B190B0250104020913809C0
:10B44000309139092E5F3F4F280F391FC90160E045
:10B4500070E0A8010E94357F80915807C82FD0E086
:10B46000C859D94E1B821A820E94FF3C8095909544
:10B470009B838A830AC030933909209338096093EB
:10B4800037091092C4151092C315DF91CF911F9107
:10B490000F91FF90EF90DF9008952F923F924F927F
:10B4A0005F926F927F928F929F92AF92BF92CF9254
:10B4B000DF92EF92FF920F931F93DF93CF9300D011
:10B4C0000F92CDB7DEB7AC01E091CA1CF0E0EF51AE
:10B4D000FA4F2081822F90E0029602E0902E920E89
:10B4E00087709070981A892B11F088E0980E61157A
:10B4F000710529F58FEF92E09093591680935816B5
:10B5000010925B1610925A1610925D1610925C16ED
:10B5100010925F1610925E161092611610926016CD
:10B5200010926316109262161092651610926416AD
:10B5300080E091E0909367168093661608C0A8E5B6
:10B54000B6E1FB0180E101900D928150E1F74115D8
:10B55000510549F0A8E4B6E1FA0180E101900D92AD
:10B560008150E1F706C088E496E168E576E10E9443
:10B57000D35D1092580760E476E180E68093401630
:10B580001092411610924316109242168AE380934D
:10B5900046168FEF8093471686E880936816DB0186
:10B5A00099961C921CE2C12ED12CC60ED71EE0919A
:10B5B000CA1CAE2EBB2489E790E0A89EF001A99E8C
:10B5C000F00DB89EF00D1124E157F44E8481809364
:10B5D0006C1691898289D60112968C9312971396D4
:10B5E0009C932581368147815085E52EFF240027D5
:10B5F0001127B22FAA2799278827E82AF92A0A2B88
:10B600001B2BDA01C90180709070B070892F9A2FBE
:10B61000AB2FBB27E82AF92A0A2B1B2B40E050E06E
:10B62000207040705070542F432F322F2227E22A6F
:10B63000F32A042B152BD6011496ED92FD920D934F
:10B640001C9317972585368547855089E52EFF245D
:10B6500000271127B22FAA2799278827E82AF92A35
:10B660000A2B1B2BDA01C90180709070B070892FF2
:10B670009A2FAB2FBB27E82AF92A0A2B1B2B40E075
:10B6800050E0207040705070542F432F322F2227EB
:10B69000E22AF32A042B152BF601E086F1860287B5
:10B6A0001387092D10E0085C1F4F1093C4150093F9
:10B6B000C31508531040FB01F896F0933909E09345
:10B6C000380981E080937816892D86958695869530
:10B6D0008183665C7F4FF501EF51FA4F4081F501A0
:10B6E00053E0EE0FFF1F5A95E1F7E553FA4ECB01F9
:10B6F000BF0150E00E941A7FE091CA1CF0E0EF51B8
:10B70000FA4F808190E0081B190B025010402091E5
:10B710003809309139092E5F3F4F280F391FC90171
:10B7200060E070E0A8010E94357FFCE09F0E9092DF
:10B7300037090E94094A1C01809158078B83682EA3
:10B7400077248090C3159090C415409037095524F4
:10B75000ACE2B0E06A0E7B1EC5C0B2E25B9E500157
:10B760001124A20CB31CF50181A181FFBAC082FF94
:10B77000B8C080818E3F21F48181803809F4B1C046
:10B780006301C40CD11C80E496E1C80ED91EE3E02D
:10B79000D601EC93F0EC1396FC93139784E011968A
:10B7A0008C93D50150968C915097F6018283919697
:10B7B0008C9180FF0DC08FEF9FEFAFEFBFEF8483C1
:10B7C0009583A683B78380879187A287B38774C048
:10B7D000D50155966D917D918D919C91589728EE4C
:10B7E00033E040E050E00E948581C901DA01EB2E90
:10B7F000FF2400271127582F442733272227E22A26
:10B80000F32A042B152B9C01AD0120703070507071
:10B81000232F342F452F5527E22AF32A042B152BEB
:10B82000A0E0B0E08070A070B070BA2FA92F982F60
:10B830008827E82AF92A0A2B1B2BF601E482F582D5
:10B8400006831783D5015D966D917D918D919C91B5
:10B85000909728EE33E040E050E00E948581C901D6
:10B86000DA01EB2EFF2400271127582F4427332716
:10B870002227E22AF32A042B152B9C01AD0120700C
:10B8800030705070232F342F452F5527E22AF32A8A
:10B89000042B152BA0E0B0E08070A070B070BA2F20
:10B8A000A92F982F8827E82AF92A0A2B1B2BF601A3
:10B8B000E086F18602871387D6011C961D921D92A1
:10B8C0001D921C921F97F6017096D50180E10D9094
:10B8D00001928150E1F7B0E24B0EE0E2F0E08E0E13
:10B8E0009F1E5394F1E0F51508F037CF8092C315F1
:10B8F0009092C415409237095092480988ED9FEF05
:10B90000880E991E9A8289828A8180934416898141
:10B91000809345169B81092F10E00859194ED801D4
:10B9200013961C921E9212970E94FF3C8095909550
:10B93000F801938382830F900F900F90CF91DF9146
:10B940001F910F91FF90EF90DF90CF90BF90AF903D
:10B950009F908F907F906F905F904F903F902F902F
:10B960000895BF92CF92DF92EF92FF920F931F93B1
:10B97000DF93CF93CDB7DEB760970FB6F894DEBFF5
:10B980000FBECDBF8091CA1C90E029E730E0829FB6
:10B99000F001839FF00D929FF00D1124E157F44EBA
:10B9A0008389882309F4CCC0809147168F3F09F022
:10B9B000C7C080915807682F70E0FB01E859F94E25
:10B9C0008181882309F0BCC010923909109238098E
:10B9D00084E0809337090091C3151091C41520E0CD
:10B9E00030E044E0FB01BC9611C0DC01A05CB94E24
:10B9F00011969C911197992309F49CC08C918130E8
:10BA000009F49D01990F990F990F490FCF01840FE8
:10BA1000911D8017910748F3209338093093390915
:10BA200040933709232B09F470C0809148169091F8
:10BA30004916892B59F580914A1690914B16892BFE
:10BA400029F580914C1690914D16892BF9F480912F
:10BA50004E1690914F16892BC9F4809150169091F3
:10BA60005116892B99F48091521690915316892B77
:10BA700069F48091541690915516892B39F4809170
:10BA8000561690915716892B09F45AC088E496E10E
:10BA90000E94254E7C01909341098093400960915A
:10BAA000380970913909009749F46E5F7F4F88E437
:10BAB00096E140E022E00E94824E27C082E0C82E3C
:10BAC000D12CC60ED71E8701005F1F4FE091CA1C04
:10BAD000F0E0EF51FA4FB080C601B8014B2D50E0B5
:10BAE0000E940D7F009759F0C801B6014B2D50E020
:10BAF0000E941A7FE0914009F091410904C0F701CA
:10BB0000818D882311F482E0818F1092C4151092E8
:10BB1000C315DE011196E8E4F6E180E101900D9293
:10BB20008150E1F780E090E0BE016F5F7F4F0E949F
:10BB3000EA5E0AC0309339092093380940933709E7
:10BB40001092C4151092C31560960FB6F894DEBF1C
:10BB50000FBECDBFCF91DF911F910F91FF90EF905E
:10BB6000DF90CF90BF90089540E020E030E0FC01EE
:10BB7000E20FF31F5081FB01E20FF31FE0815E171C
:10BB800031F4485F2F5F3F4F403889F70AC0E527FF
:10BB9000842F885FE7FD05C04F5F481711F0EE0F57
:10BBA000F9CF842F08959F92AF92BF92CF92DF92E8
:10BBB000EF92FF920F931F93CF93DF93E82E992E6E
:10BBC000EB0188818E3F21F48981803819F437C0D8
:10BBD0008F3FA9F100E0FF2411E09BE1A92EB12CD9
:10BBE00089E7C82ED12C26C08091CA1C90E0212F55
:10BBF00030E02A9DB0012B9D700D3A9D700D1124EF
:10BC00009C012C9DC0012D9D900D3C9D900D1124FB
:10BC1000680F791FFB01E157F44E80A5813049F48C
:10BC20006955744ECE010E94B45D8F1510F0012F3E
:10BC3000F82E1F5F1330C0F21093530901C000E0CB
:10BC4000402F50E02091CA1C30E08BE190E0489FEB
:10BC5000F001499FF00D589FF00D112489E790E005
:10BC6000AC01249FC001259F900D349F900D11249D
:10BC7000E80FF91F2E2D392DC901DC01E955F44ECD
:10BC800080E101900D928150E1F7DF91CF911F91FA
:10BC90000F91FF90EF90DF90CF90BF90AF909F906B
:10BCA0000895E091CA1CF0E0DF01AC5AB64F1C9237
:10BCB000EE0FFF1FDF01A65AB64F6D917C91EA5A35
:10BCC000F64F808191810E944D5A08950E94BC7E5A
:10BCD000AA2797FDA095BA2FBC01CD0120E532E23D
:10BCE00046E050E00E9485819B01AC0120593A4F0B
:10BCF0004C4F5F4FB901CA0108954F925F926F9206
:10BD00007F928F929F92BF92CF92DF92EF92FF929B
:10BD10000F931F938091CA1C90E04FE8C42E4BE113
:10BD2000D42E39E7432E512C849DF001859DF00DD2
:10BD3000949DF00D1124EC0DFD1D658176818781A8
:10BD400090850E94568020E030E040E05FE30E9452
:10BD5000BC800E942A803B014C010E94BC7EB82E10
:10BD60000E94BC7EFB2CEE24E80EF91E00E010E0E1
:10BD70008091CA1C90E09C01249DC001259D900DDE
:10BD8000349D900D1124C80ED91EF601658176816F
:10BD9000878190850E9456800E942A809B01AC0179
:10BDA000C801B7010E9485819B01AC01260D371D9A
:10BDB000481D591DB901CA011F910F91FF90EF90C5
:10BDC000DF90CF90BF909F908F907F906F905F900B
:10BDD0004F9008951F93CF93DF939C011091CA1C3D
:10BDE000A12FB0E0FD01EC5AF64F8081882309F0C5
:10BDF0004AC02115310591F0CEE5D9E0F90180E185
:10BE0000019009928150E1F7FD01EE0FFF1FEA5A00
:10BE1000F64F8EE599E09183808307C0FD01EE0F18
:10BE2000FF1FEA5AF64F118210826115710591F0D9
:10BE3000CEE6D9E0FB0180E1019009928150E1F763
:10BE4000FD01EE0FFF1FE65AF64F8EE699E0918353
:10BE5000808307C0FD01EE0FFF1FE65AF64F1182E7
:10BE60001082AC5AB64F81E08C930E94BC7E64EF86
:10BE700071E00E947281AC01662757FD6095762FB4
:10BE8000812F0E94ED65DF91CF911F910895EF9270
:10BE9000FF920F931F930E94665E7B018C01E091DD
:10BEA000CA1CF0E0EF5AF64F8081833078F481E8C5
:10BEB000E8168EE3F80680E0080780E0180730F007
:10BEC00020E8E22E2EE3F22E012D112D80E090E0ED
:10BED00060E070E00E944D5A8091CA1CE82FF0E0AB
:10BEE000EF5AF64F90819F5F9083B801A7010E949F
:10BEF00030661F910F91FF90EF9008958091CA1CBA
:10BF0000A82FB0E089E790E0A89FF001A99FF00D6D
:10BF1000B89FF00D1124E157F44E84898823E1F095
:10BF2000AF5AB64F8C918823B9F40E94665EAC017B
:10BF3000CB01DA01AC01BD0141388EE3580780E046
:10BF4000680780E0780720F040E85EE360E070E09A
:10BF50008091CA1C0E94306608951F931091CA1CDC
:10BF6000E12FF0E0E15BF64F8081882371F40E94BD
:10BF7000BC7E60ED77E00E947281AC01662757FDC0
:10BF80006095762F812F0E947C661F9108950E94F4
:10BF90009249892BD1F4E091CA1CF0E0E15BF64FA5
:10BFA0008081843090F40E94A1548091CA1CE82FB3
:10BFB000F0E0E15BF64F90819F5F908348E853E1AA
:10BFC00060E070E00E947C6608958091CA1C0E9427
:10BFD000CA65E091CA1CF0E0E15BF64F10820E9456
:10BFE000D6750895BF92CF92DF92EF92FF920F9392
:10BFF0001F93CF93DF937C01062FB42E1092530929
:10C000002091CA1C30E00695069506954BE1C42E9A
:10C01000D12C89E790E0289FE001299FD00D389F1F
:10C02000D00D112433C0212F30E02C9DF0012D9D27
:10C03000F00D3C9DF00D1124EC0FFD1FE157F44E67
:10C0400080A58F3F01F182A98B1511F0BB20D9F497
:10C050002C9DC0012D9D900D3C9D900D11248C0FA9
:10C060009D1F8955944EB701402F50E00E940D7FCF
:10C07000009749F48BE1189F900111242C0F3D1F6C
:10C080002955344E09C01F5F10935309109153096D
:10C09000133048F220E030E0C901DF91CF911F91C9
:10C0A0000F91FF90EF90DF90CF90BF900895609137
:10C0B000CA1C29E7629FB00111246850744E40E108
:10C0C00050E00E940D7F9C0180E0232B09F481E069
:10C0D00008951F93CF93DF93BC011091CA1CE12FE9
:10C0E000F0E0EE0FFF1FE75BF64F8081918140E1AA
:10C0F00050E00E940D7F0097A9F4812F0E94D46523
:10C10000A091CA1CB0E0FD01EE0FFF1FE75BF64FE8
:10C11000808191812FEFEC01288B11821082A35B2B
:10C12000B64F1C928FEF9FEF0E9458731F93DC0154
:10C1300050968C9150978823E1F41091CA1CE12FFE
:10C14000F0E0EE0FFF1FE75BF64F80819181892BB6
:10C1500081F4B183A0830E94BC7E60ED77E00E94F1
:10C160007281AC01662757FD6095762F812F0E9462
:10C1700008671F9108951F93CF93DF932091CA1CE6
:10C18000A22FB0E0FD01EE0FFF1FE75BF64F4081ED
:10C1900051814115510509F489C0C9E7D0E0AC9F30
:10C1A000F001AD9FF00DBC9FF00D1124E157F44E4E
:10C1B000A35BB64F9C918789981788F580E090E043
:10C1C00060E070E00E949B551091CA1C212F30E066
:10C1D000F901E35BF64F80818F5F80832C9FF00134
:10C1E0002D9FF00D3C9FF00D1124E157F44E658515
:10C1F00076858785908928EE33E040E050E00E9404
:10C200008581CA01B90128EE33E040E050E00E9488
:10C210004781AB01BC01812F0E94086747C0822F74
:10C220000E94D4652091CA1C30E0F901EE0FFF1F77
:10C23000E75BF64FA081B18181E050968C9311822B
:10C240001082F901E35BF64F10821092530940E02F
:10C25000ABE1B0E02C9FB0012D9F700D3C9F700DA5
:10C26000112420C0242F2F5F842F90E08A9FF0019B
:10C270008B9FF00D9A9FF00D1124E60FF71FE157E9
:10C28000F44E80A5882369F4409353098BE1489FBD
:10C29000C0011124860F971F8955944E0E94966005
:10C2A00005C0422F4330F0F240935309DF91CF9104
:10C2B0001F910895CF93DF93DC01EB01E091CA1C3D
:10C2C000F0E0EF51FA4FE081E83061F49C01285F23
:10C2D0003F4FFB0188E00190E90109929E018150E6
:10C2E000D1F723C0E63039F59C01285F3F4FAB0101
:10C2F00083E0FA010190AF01F90101929F018150A1
:10C30000C1F78FEF1B968C931B978EEF1C968C9327
:10C310001C979D01235F3F4FFE01339683E0019000
:10C32000E90109929E018150D1F718968C911897D6
:10C3300092E0892720C0E23019F589811F968C93FD
:10C340001F9788811E968C931E971D961C921D9791
:10C350008EEF1C968C931C978FEF1B968C931B97DC
:10C360001A961C921A978091A81C19968C9319976B
:10C370008091A71C8D7F18968C93DF91CF910895A3
:10C380008FEF9FEF0E9458739F92AF92BF92CF9210
:10C39000DF92EF92FF920F931F93CF93DF93A82E1C
:10C3A000992E69017A01B02E21E0021719F4603448
:10C3B00009F0BDC0109253095091CA1CC52FD0E09E
:10C3C00040E00BE110E089E790E0C89FD001C99FF1
:10C3D000B00DD89FB00D1124A5C0642F70E0942F2C
:10C3E0009F5F609F9001619F300D709F300D112401
:10C3F0002A0F3B1FF901E157F44E80A58F3F09F04A
:10C4000090C040935309F901E955F44E8A2D992DB6
:10C410009C01D90180E10D9001928150E1F731E05A
:10C42000B31619F58BE190E09C01629FC001639FF8
:10C43000900D729F900D112429E730E0B901C69F3D
:10C440009001C79F300DD69F300D1124820F931F8E
:10C45000652F70E043E0660F771F4A95E1F765535B
:10C460007A4E8955944E0E945A618091CA1C90E080
:10C470002091530930E00BE110E0209FA001219FA3
:10C48000500D309F500D1124C9E7D0E09C012C9F26
:10C49000C0012D9F900D3C9F900D1124480F591FF6
:10C4A000FA01E157F44E10A6B2AAC114D104E10476
:10C4B000F10411F1CA018854944EB701A6010E94FB
:10C4C000AA652091530930E08091CA1C90E0209F1A
:10C4D000F001219FF00D309FF00D1124BC016C9FE5
:10C4E000C0016D9F900D7C9F900D1124E80FF91FE6
:10C4F000E157F44E11AA02C081E081AB809153094B
:10C500002BE1829FC00111242091CA1C49E7249F7E
:10C5100090011124820F931F8955944E0E949660BA
:10C5200006C0492F433008F458CF40935309DF9198
:10C53000CF911F910F91FF90EF90DF90CF90BF9020
:10C54000AF909F900895FF920F931F93CF93DF9327
:10C5500081E0809353090BE110E0C9E7D0E0FF24AC
:10C56000FA9444C08091CA1C90E030E0209FA00162
:10C57000219F500D309F500D11249C012C9FC00114
:10C580002D9F900D3C9F900D1124480F591FFA01CB
:10C59000E157F44E80A58F3F21F181A9813009F147
:10C5A000CA018854944E0E949065892BD1F0209145
:10C5B000530930E08091CA1C90E0209FF001219F38
:10C5C000F00D309FF00D11249C012C9FC0012D9F78
:10C5D000900D3C9F900D1124E80FF91FE157F44E88
:10C5E000F0A6809153098F5F8093530920915309DE
:10C5F000233008F4B7CFDF91CF911F910F91FF90B7
:10C6000008958F929F92AF92BF92CF92DF92EF9256
:10C61000FF920F931F93DF93CF93CDB7DEB7E297CF
:10C620000FB6F894DEBF0FBECDBF10925309FBE1E9
:10C63000CF2ED12CE9E7EE2EF12C8E010F5F1F4F8C
:10C6400079E5A72E75E0B72E6BE1862E59E7952E7A
:10C6500081C030E08091CA1C90E02C9DF0012D9D9E
:10C66000F00D3C9DF00D11249C012E9DC0012F9DCD
:10C67000900D3E9D900D1124E80FF91FE157F44EE7
:10C6800080A58F3F09F461C086E197E00E94540BBA
:10C690002091530930E08DB79EB708970FB6F894F4
:10C6A0009EBF0FBE8DBFADB7BEB71196EDB7FEB73B
:10C6B000128301831396BC92AE92129715963C9307
:10C6C0002E9314978091CA1C90E02C9DF0012D9D13
:10C6D000F00D3C9DF00D11249C012E9DC0012F9D5D
:10C6E000900D3E9D900D1124E80FF91FE157F44E77
:10C6F00080A5992787FD909517969C938E93169702
:10C700000E94A87F8DB79EB708960FB6F8949EBF7B
:10C710000FBE8DBFC8010E94620B60915309689DD6
:10C72000B00111248091CA1C899DC0011124680F99
:10C73000791F6955744EC8010E945978C8010E943A
:10C74000620B83E197E00E94540B809153098F5F45
:10C750008093530920915309233008F47ACFE2964D
:10C760000FB6F894DEBF0FBECDBFCF91DF911F9102
:10C770000F91FF90EF90DF90CF90BF90AF909F9080
:10C780008F9008957F928F929F92AF92BF92CF9297
:10C79000DF92EF92FF920F931F934B015C01142FD6
:10C7A000722E8091CA1C90E029E7C22ED12C8C9D5C
:10C7B00070018D9DF00C9C9DF00C11242FE83BE145
:10C7C000E20EF31E80E095E0A0E0B0E0F701808388
:10C7D0009183A283B38380E4848380E395E7A0E020
:10C7E000B0E085839683A783B0870E947D5EF701C2
:10C7F0006187728783879487F090CA1C6F2D70E0E1
:10C800006C9D90016D9D300D7C9D300D1124F901C2
:10C81000E157F44E88EE93E0A0E0B0E0858796877C
:10C82000A787B08B81E0878B928A818A138A148BC9
:10C83000758A068B40E0ABE1B0E05FEF0FC0842F5C
:10C8400090E08A9FF0018B9FF00D9A9FF00D1124CC
:10C85000E20FF31FE157F44E50A74F5F433078F3D8
:10C860004093530909E710E0609F9001619F300DEC
:10C87000709F300D1124D901A157B44EA759BF4F55
:10C880009FEF9D9382E08D931D921D921D921D92AC
:10C890001D921D921D921D921D92EE24E394ED9225
:10C8A0009D93FB01EF51FA4F8081FB0193E0EE0F66
:10C8B000FF1F9A95E1F7E553FA4EE80FF11D339704
:10C8C00081918D9381918D9380818C93A857B040F5
:10C8D000772009F45AC08EEF90E859969C938E9376
:10C8E00058975B961C921E925A975D961C921E92C8
:10C8F0005C975F961C921E925E9791961C921E9278
:10C90000909793961C921E92929795961C921E92C7
:10C91000949797961C921E9296976F2D70E0A3E0C5
:10C92000660F771FAA95E1F765537A4EC9018955BD
:10C93000944E0E945A618091CA1C90E09C01209FF5
:10C94000C001219F900D309F900D1124FC01E157F3
:10C95000F44E10A623E022ABE1AA8955944E0E9422
:10C9600096600E94AD5F81149104A104B10469F046
:10C970008091CA1C90E0809FF001819FF00D909FF4
:10C98000F00D1124E157F44EE38A8091CA1C48EE61
:10C9900053E060E070E00E94B7661F910F91FF9036
:10C9A000EF90DF90CF90BF90AF909F908F907F904F
:10C9B0000895FFCF08950F931F93DF93CF93CDB7C3
:10C9C000DEB728970FB6F894DEBF0FBECDBF8C013F
:10C9D0008091CA1C882309F055C00115110591F4F6
:10C9E00083E389838A83809164168B8380916516A3
:10C9F0008C83809166168D83809167168E838E015D
:10CA00000F5F1F4F6091C3157091C415FB01E15C6E
:10CA1000F94E03C080818687319726E1EF33F20714
:10CA2000C9F7D8018C91818311968C9111978283DB
:10CA300012968C911297838313968C91139784830B
:10CA400014968C911497858315968C918683ABEC04
:10CA5000B5E137968D91819325E1A13DB207D1F7DC
:10CA600086E880934C168DED80934D16625F7F4F64
:10CA70007093C4156093C31580E496E141E00E9471
:10CA8000EF3327C0813049F5809146168131F1F4AA
:10CA900088E596E1B8010E94A5718823B9F09091CC
:10CAA0006A1680916B16825B904F81F480917016AC
:10CAB000873761F450916816409169168091671626
:10CAC0009091661668E476E10E943622C8010E94C1
:10CAD000EF711092C4151092C31580E090E0289673
:10CAE0000FB6F894DEBF0FBECDBFCF91DF911F917F
:10CAF0000F910895EF92FF920F931F93FC01E08036
:10CB0000F180028113810E94260EE61AF70A080BB3
:10CB1000190BB701C8011F910F91FF90EF90089575
:10CB2000EF92FF920F931F93FC01E080F18002814E
:10CB300013810E94260E20E030E0E616F706080773
:10CB4000190710F421E030E0C9011F910F91FF9007
:10CB5000EF900895CF92DF92EF92FF920F931F9381
:10CB60006C017A018B01FC014483558366837783D2
:10CB70000E94260E6E0D7F1D801F911FF60160839F
:10CB80007183828393831F910F91FF90EF90DF90C9
:10CB9000CF900895E82FF0E0ED55F34E8081882383
:10CBA00011F00E94760E0895E82FF0E0EF55F34E55
:10CBB0008081882311F00E94760E0895CF93DF9331
:10CBC000C3E9DCE188810E94760E19928CE1CF39AD
:10CBD000D807C1F7DF91CF910895CF92DF92EF92FE
:10CBE000FF920F931F93C82ECB01BA0128EE33E0BA
:10CBF00040E050E00E948581C901DA017C018D018D
:10CC000081E0E81680E0F80681E0080780E0180778
:10CC100028F0E12CF12C81E0082F112D81E0C816BD
:10CC200021F4C7016CEE77E603C0C70165EE77E635
:10CC30000E94250FD82E882339F4E114F104010550
:10CC4000110511F00E94D964EC2DF0E0ED56F34E81
:10CC5000D2861F910F91FF90EF90DF90CF900895B3
:10CC6000CF92DF92EF92FF920F931F93C82E7A011B
:10CC70008B01413080E0580781E0680780E0780749
:10CC800068F481E0C81621F4CA016BEF77E603C0AF
:10CC9000CA0164EF77E60E946E0F18C0CB01BA019B
:10CCA00028EE33E040E050E00E948581C901DA01BE
:10CCB0007C018D0181E0C81621F4C7016BEF77E696
:10CCC00003C0C70164EF77E60E94250FD82E8823A2
:10CCD00039F4E114F1040105110511F00E94D96441
:10CCE000EC2DF0E0ED56F34ED0861F910F91FF90A2
:10CCF000EF90DF90CF900895CF92DF92EF92FF9266
:10CD00000F931F93C82ECA01DB017C018D0181E0C6
:10CD1000E81680E0F80681E0080780E0180728F0B0
:10CD2000E12CF12C91E0092F112D81E0C81621F49E
:10CD3000C7016AE078E603C0C70163E078E60E94B5
:10CD40006E0FD82E882339F4E114F1040105110582
:10CD500011F00E94D964EC2DF0E0ED55F34ED08235
:10CD60001F910F91FF90EF90DF90CF900895CF9299
:10CD7000DF92EF92FF920F931F93C82E7A018B01DF
:10CD8000413080E0580781E0680780E0780788F448
:10CD9000411551056105710589F4EC2DF0E0EE0FA8
:10CDA000FF1FE258F64F808191817C0100E010E086
:10CDB0000DC0E12CF12C31E0032F112DEC2DF0E012
:10CDC000EE0FFF1FE258F64FF182E08281E0C816B5
:10CDD00021F4C70160E278E603C0C70162E178E6AA
:10CDE0000E946E0FD82E882339F4E114F104010556
:10CDF000110511F00E94D964EC2DF0E0ED56F34ED0
:10CE0000D6821F910F91FF90EF90DF90CF90089501
:10CE1000CF92DF92EF92FF920F931F93C82ECA0119
:10CE2000DB017C018D0181E0E81680E0F80681E0FD
:10CE3000080780E0180728F0E12CF12C51E0052FBD
:10CE4000112D81E0C81621F4C70165E378E603C01F
:10CE5000C7016EE278E60E946E0FD82E882339F45F
:10CE6000E114F1040105110511F00E94D964EC2DC3
:10CE7000F0E0EF55F34ED0821F910F91FF90EF90AD
:10CE8000DF90CF900895CF92DF92EF92FF920F93B1
:10CE90001F93C82E7A018B01413080E0580781E052
:10CEA000680780E0780788F4411551056105710530
:10CEB00089F4EC2DF0E0EE0FFF1FEE57F64F808166
:10CEC00091817C0100E010E00DC0E12CF12C71E0BB
:10CED000072F112DEC2DF0E0EE0FFF1FEE57F64F50
:10CEE000F182E08281E0C81621F4C7016BE478E6A4
:10CEF00003C0C7016DE378E60E946E0FD82E882329
:10CF000039F4E114F1040105110511F00E94D9640E
:10CF1000EC2DF0E0ED56F34ED2821F910F91FF9071
:10CF2000EF90DF90CF900895CF92DF92EF92FF9233
:10CF30000F931F93C82E7A018B01413080E0580770
:10CF400081E0680780E0780788F4411551056105A4
:10CF5000710589F4EC2DF0E0EE0FFF1FEA57F64F54
:10CF6000808191817C0100E010E00DC0E12CF12C6A
:10CF700011E0012F112DEC2DF0E0EE0FFF1FEA570D
:10CF8000F64FF182E08281E0C81621F4C70167E61E
:10CF900078E603C0C70169E578E60E946E0FD82ED7
:10CFA000882339F4E114F1040105110511F00E9400
:10CFB000D964EC2DF0E0ED56F34ED0821F910F9125
:10CFC000FF90EF90DF90CF9008951092CA1C0E94BE
:10CFD000515E0E945973089581E08093CA1C0E949B
:10CFE000515E0E94597308951092CA1C0E94475FB7
:10CFF0000E945973089581E08093CA1C0E94475F84
:10D000000E94597308951092CA1C0E94C75F0E9423
:10D010005973089581E08093CA1C0E94C75F0E94E3
:10D02000597308951092CA1C80E040E050E060E01F
:10D0300070E00E94B7660E94A3620E94597308952F
:10D0400081E08093CA1C40E050E060E070E00E9404
:10D05000B7660E94A3620E94597308951092CA1C79
:10D060000E94BB600E945973089581E08093CA1C9E
:10D070000E94BB600E94597308951092CA1C80E000
:10D0800040E050E060E070E00E9443670E94134A75
:10D090000E945973089581E08093CA1C40E050E0DB
:10D0A00060E070E00E9443670E94134A0E94597337
:10D0B00008951092CA1C80E040E050E060E070E00B
:10D0C0000E9494670E9479760E945973089581E0C6
:10D0D0008093CA1C40E050E060E070E00E949467DA
:10D0E0000E9479760E94597308950F93DF93CF932E
:10D0F00000D000D0CDB7DEB79A8389837C836B8361
:10D1000081E08093CA1C8C818093D3158B8180939E
:10D11000D4158A818093A71C89818093A81C809153
:10D120000C05882341F460E070E080E090E040E08E
:10D1300020E001E00DC089E695E00E94387310926E
:10D14000CA1C68EE73E080E090E041E021E000E07E
:10D150000E94844781E044EF51E060E070E00E946B
:10D1600094670F900F900F900F90CF91DF910F91D8
:10D1700008950F93DF93CF93CDB7DEB760970FB6C7
:10D18000F894DEBF0FBECDBFAC011092CA1C009751
:10D1900079F020E030E0F901E553FA4EDA01A20F10
:10D1A000B31F8C9180832F5F3F4F2630310599F755
:10D1B00080910C05882341F460E070E080E090E00D
:10D1C00040E021E001E01DC0FE01319680E1DF0179
:10D1D0001D928A95E9F780E2898382E08A838DE057
:10D1E0008B8388EB8C8381E08D8381EE8E83CF01EE
:10D1F0000E94387368E077E080E090E041E021E051
:10D2000000E00E94844780E044EF51E060E070E07D
:10D210000E94946760960FB6F894DEBF0FBECDBF34
:10D22000CF91DF910F9108958AE899E09093861C41
:10D230008093851C0E94DE650E948D690895382FB9
:10D240001092360F20E02CC0822F90E0FC0173E09A
:10D25000EE0FFF1F7A95E1F7880F991FE80FF91F6E
:10D26000E25EF04F80818130D1F4822F90E0FC01AA
:10D2700053E0EE0FFF1F5A95E1F7880F991FE80F53
:10D28000F91FE25EF04F8181831749F42093360F36
:10D290008AE0289F90011124225E304F07C02F5F43
:10D2A000223090F22093360F20E030E0C90108953B
:10D2B000AC0181E08093360F21E02AC0322F3F5F1E
:10D2C000822F90E0FC01B3E0EE0FFF1FBA95E1F76B
:10D2D000880F991FE80FF91FE25EF04F80818823C5
:10D2E000B1F481E08093280F2093290F90E00AC0C9
:10D2F000E92FF0E0DA01AE0FBF1F8C91E25EF04F34
:10D3000084879F5F9830A0F39093360F0895232F62
:10D310002230A0F22093360F089581E080931E0FF3
:10D3200010921F0F8EEF8093200F80E88093210FC3
:10D3300021E010C0822F90E0FC0143E0EE0FFF1FC0
:10D340004A95E1F7880F991FE80FF91FE25EF04F49
:10D3500010822F5F223070F32093360F0895EF92E2
:10D36000FF920F931F93CF93DF937C01E091090A03
:10D37000F0910A0A80910B0A90E00396DF01A80F52
:10D38000B91F0397B093350FA093340FE80FF91F1F
:10D39000818186FD29C087FD12C0FD018191919197
:10D3A000A191B19180930E0A90930F0AA093100A55
:10D3B000B093110AF093350FE093340F31C080E63B
:10D3C00080930E0A8C918F7080930F0A11968D9125
:10D3D0009C9112979093110A8093100A1396B09320
:10D3E000350FA093340F1CC087FD11C08C9182951E
:10D3F0008F70806680930E0AFD0181918295807FF7
:10D4000080930F0AF093350FE093340F05C080E648
:10D4100080930E0A10920F0A1092110A1092100AAD
:10D4200080910B0AC091090AD0910A0AC80FD11D38
:10D43000898185FD0BC0E091340FF091350F81910A
:10D440008093140AF093350FE093340F898190E0B4
:10D45000887190708830910561F0893091051CF4D5
:10D46000892B79F019C08031910529F04897A1F4F2
:10D4700006C081E001C080E48093150A0DC08FEFE3
:10D48000FBCFE091340FF091350F81918093150A15
:10D49000F093350FE093340F8A8190E080739070A1
:10D4A00054E0959587955A95E1F70E941F69AC0164
:10D4B0009093330F8093320F8A81282F30E0207CA5
:10D4C00030702034310509F477C02134310524F45B
:10D4D000232B09F493C0A8C020383105D1F0203C9B
:10D4E000310509F0A1C04115510519F482E099E018
:10D4F0001CC0A6E1BAE0FA01329688E001900D92D4
:10D500008150E1F786E19AE061E87CE10E945A618E
:10D510008BC0A091340FB091350F8C9187FD27C03F
:10D520004115510529F48DEC98E00E94540BDEC1A1
:10D53000A6E1BAE0FA01329688E001900D9281509E
:10D54000E1F786E0EEE1FAE0DF011D928A95E9F766
:10D55000E091340FF091350F819191919093250ACC
:10D560008093240AF093350FE093340F5DC080FD63
:10D5700020C011968C91119781508230D0F48FEF9A
:10D580008093160A8C9186958F708093170A8DE090
:10D59000E8E1FAE0EF0119928A95E9F711968C918A
:10D5A00011978093250A1296B093350FA093340FEC
:10D5B0003BC089E898E0B9CF4115510519F484E5DD
:10D5C00098E0B3CFA6E1BAE0FA01329688E0019084
:10D5D0000D928150E1F7AEE1BAE08091340F909165
:10D5E000350F9C01F90188E001900D928150E1F71F
:10D5F0008091340F9091350F089612C0A6E1BAE0E1
:10D600008091340F9091350F9C01F90180E10190D8
:10D610000D928150E1F78091340F9091350F409633
:10D620009093350F8093340F80910B0A0091090A73
:10D6300010910A0A080F111DF801828183700E945F
:10D640001F69AC019093330F8093320FD80112966B
:10D650008C91282F30E02C7030702430310509F483
:10D6600075C02530310524F4232B09F491C0A6C0E0
:10D6700028303105D1F02C30310509F09FC041151B
:10D68000510519F48FE198E050CFA6E2BAE0FA0113
:10D69000329688E001900D928150E1F786E29AE09F
:10D6A00063E87CE10E945A6189C0A091340FB09177
:10D6B000350F8C9187FD25C04115510519F48AEE6F
:10D6C00097E033CFA6E2BAE0FA01329688E0019003
:10D6D0000D928150E1F786E0EEE2FAE0EF01199257
:10D6E0008A95E9F7E091340FF091350F819191918E
:10D6F0009093350A8093340AF093350FE093340FFA
:10D700005DC080FD20C011968C91119781508230B0
:10D71000D0F48FEF8093260A8C9186958F7080933A
:10D72000270A8DE0E8E2FAE0EF0119928A95E9F71D
:10D7300011968C9111978093350A1296B093350FFC
:10D74000A093340F3BC086EA97E0EFCE4115510518
:10D7500019F481E797E0E9CEA6E2BAE0FA01329641
:10D7600088E001900D928150E1F7AEE2BAE080913D
:10D77000340F9091350F9C01F90188E001900D92D2
:10D780008150E1F78091340F9091350F089612C0C7
:10D79000A6E2BAE08091340F9091350F9C01F90117
:10D7A00080E101900D928150E1F78091340F9091CA
:10D7B000350F40969093350F8093340F80910D0A6A
:10D7C000885D80930D0A80910B0AE091090AF0911F
:10D7D0000A0AE80FF11D818185FF5AC0A091340F1C
:10D7E000B091350F8C918C7F883F09F051C081E159
:10D7F0008093140A8C91883F29F18B3F09F045C032
:10D80000EEE0FAE0B89611968C91119782958F70A0
:10D8100090E080559F409093360A818311968C91B9
:10D82000119790E08F70907080559F409283838312
:10D8300012968D919C91139790933D0A80933C0A88
:10D84000149619C011968D919C9112979093370A56
:10D850008093360A13968D919C9114979093390A70
:10D860008093380A15968D919C91169790933D0A56
:10D8700080933C0A1796B093350FA093340F809194
:10D880000D0A885F80930D0A03C082E397E04DCEB6
:10D890002091340F8091090A281B20930B0AE11470
:10D8A000F10451F41092120A80910D0A885290915D
:10D8B000871C890F821B0CC0E8EDFFEFEE0EFF1EE8
:10D8C000F092120A88E290E0E80EF91E8E2D88523E
:10D8D0008093130A8091140A813141F48091120AD5
:10D8E0009091130A90933B0A80933A0ADF91CF916B
:10D8F0001F910F91FF90EF900895FF920F931F9348
:10D90000DF93CF93CDB7DEB764970FB6F894DEBF41
:10D910000FBECDBF8C01462F81E08093CA1C1092B0
:10D920000D0A10920B0A8091851C9091861C8093A1
:10D93000090A90930A0A6093871C1092881C980128
:10D94000225F3F4FB90150E00E941A7FD8011B9619
:10D950002D913C911C973A832983FE013196818158
:10D960008093811C89818093821C19968D919C9152
:10D970001A979A83898381818093831C89818093FC
:10D98000841CE091090AF0910A0A8081813021F417
:10D99000C9010E9474222DC186E19FE00E9490651A
:10D9A000892B41F010920F0F10920E0F1092110F51
:10D9B0001092100FE091090AF0910A0A308121813A
:10D9C000C9018070987F892F9927803C910549F083
:10D9D000803E910589F000E010E0FF2440E050E037
:10D9E00015C0890117705281438180910B0A8C5FA9
:10D9F00080930B0AFF240AC0F4805281438189017D
:10DA0000177080910B0A8B5F80930B0A8091100F27
:10DA10009091110F892B19F10115110509F4E9C035
:10DA200080910E0F90910F0F0817190709F0E1C0B0
:10DA30008091140F9091150F8417950709F0D9C0A4
:10DA40009091A51C8091811C981709F0D2C09091EB
:10DA5000A61C8091821C981709F0CBC01BC0011531
:10DA60001105C1F010930F0F00930E0F5093150F77
:10DA70004093140F86E19FE044EF51E060E070E0D6
:10DA80000E94AA658091811C8093A51C8091821CB4
:10DA90008093A61C80910B0A853049F12091090AD8
:10DAA00030910A0AF901E80FF11DE081E33021F01D
:10DAB000E13409F09EC004C0C8010E94AF6917C0DC
:10DAC0008F5F80930B0AAEE0BAE0F901E80FF11D19
:10DAD00088E201900D928150E1F780910B0A885DF8
:10DAE00080930B0A80910D0A885D80930D0A9091B6
:10DAF0000B0A4091871C491B40930C0A2F2D30E0E4
:10DB000063E0220F331F6A95E1F780910D0A280F19
:10DB1000311D225F354FE091090AF0910A0AE90FA1
:10DB2000F11DC901BF0150E00E941A7F012BC9F00D
:10DB30008091100F9091110F892B31F480910D0A73
:10DB40008093100F1092110F20910C0A8091100FEA
:10DB50009091110F820F911D9093110F8093100FD0
:10DB60000BC020910D0A80910C0A90E0820F911D4C
:10DB700090930F0F80930E0F2091100F3091110F83
:10DB80002115310539F080910E0F90910F0F281754
:10DB9000390779F500E416E12EE03AE040910E0FE6
:10DBA00050910F0FC801B9010E941A7F60910E0FAA
:10DBB00070910F0F10920F0F10920E0F1092110F05
:10DBC0001092100F1092C4151092C3151B829091E1
:10DBD000811C8091821C8C839D831C861E861D86E1
:10DBE000C801AE014D5F5F4F9E01245F3F4F0E9411
:10DBF000327964960FB6F894DEBF0FBECDBFCF91D9
:10DC0000DF911F910F91FF9008951F93CF93DF93A2
:10DC1000EC011092360F30C0812F90E0FC01B3E090
:10DC2000EE0FFF1FBA95E1F7880F991FE80FF91F54
:10DC3000E25EF04F80818130E1F4212F30E0C901B4
:10DC4000F3E0880F991FFA95E1F7220F331F820F37
:10DC5000931F805E904FBE0148E050E00E940D7F10
:10DC6000009739F48AE0189F90011124225E304F0A
:10DC700009C01F5F1093360F1091360F123060F2FB
:10DC800020E030E0C901DF91CF911F9108950F93FB
:10DC90001F93182F092FE091090AF0910A0A339671
:10DCA000F093350FE093340F339780910B0AE80F10
:10DCB000F11D1282118280910B0AE091090AF09104
:10DCC0000A0AE80FF11D83E0808380914116282F16
:10DCD00030E0C9018F709070892B09F03FC08091AE
:10DCE000421690914316892BC9F580910B0AE09159
:10DCF000090AF0910A0AE80FF11D8181806481838D
:10DD000080914016282F30E0C9018F709070892BC8
:10DD100081F480914116807F61F480910B0AE0913B
:10DD2000090AF0910A0AE80FF11D81818068818358
:10DD30005FC0E091340FF091350F94E0220F331F54
:10DD40009A95E1F78091411682958F70822B80839E
:10DD50008091340F9091350F019646C08091401606
:10DD600090E08F709070892B51F5822F807F39F56C
:10DD700080910B0AE091090AF0910A0AE80FF11D5F
:10DD8000818180688183E091340FF091350F90910B
:10DD900041169F7080914016807F982B9083E09170
:10DDA000340FF091350F8091421690914316928373
:10DDB00081838091340F9091350F039615C0E091C7
:10DDC000340FF091350F8091401690914116A0913B
:10DDD0004216B091431680839183A283B3838091CE
:10DDE000340F9091350F04969093350F8093340F34
:10DDF00080914616813161F480910B0AE091090A05
:10DE0000F0910A0AE80FF11D8181806281830EC0C2
:10DE1000E091340FF091350F80838091340F909111
:10DE2000350F01969093350F8093340F80914716EC
:10DE3000803479F08F3FC9F0813011F580910B0A61
:10DE4000E091090AF0910A0AE80FF11D81818860CA
:10DE50000AC080910B0AE091090AF0910A0AE80FC2
:10DE6000F11D81818061818319C080910B0AE0914D
:10DE7000090AF0910A0AE80FF11D81818861F3CF48
:10DE8000E091340FF091350F80838091340F9091A1
:10DE9000350F01969093350F8093340F88E496E107
:10DEA0000E94056EDC019093330F8093320F009730
:10DEB00009F49FC080910B0AE091090AF0910A0AC7
:10DEC000E80FF11D11968C918295807F9281892BAC
:10DED00082832091501630E08091A71C90E08D7FC6
:10DEE00028173907B9F5909151168091A81C9817F9
:10DEF00089F580915216882369F5809153168F3FDA
:10DF000049F5809154168E3F29F580915516882346
:10DF100009F58091CA1CE82FF0E083E0EE0FFF1FA7
:10DF20008A95E1F7E553FA4E90915616808198173D
:10DF300089F4909157168181981761F480910B0AAA
:10DF4000E091090AF0910A0AE80FF11D8281806CC4
:10DF5000828365C08091501690915116892B59F596
:10DF60008091521690915316892B29F58091541661
:10DF700090915516892BF9F48091561687FD1BC098
:10DF800080910B0AE091090AF0910A0AE80FF11D4D
:10DF9000828180688283E091340FF091350F809107
:10DFA000561690915716918380838091340F9091EB
:10DFB000350F029630C080910B0AE091090AF0916A
:10DFC0000A0AE80FF11D8281806482832091340F58
:10DFD0003091350FC901DC01E0E5F6E188E0019000
:10DFE0000D928150E1F78091340F9091350F089692
:10DFF00012C08091340F9091350F9C01D901E8E453
:10E00000F6E180E101900D928150E1F78091340FAB
:10E010009091350F40969093350F8093340F8091F7
:10E0200058168F3F09F065C080915A1690915B1683
:10E03000892B09F050C080915C1690915D16892B58
:10E0400009F049C080915E1690915F16892B09F006
:10E0500042C08091601690916116892BE1F5809104
:10E06000621690916316892BB1F580916416909198
:10E070006516892B81F580916616882361F580915C
:10E0800067168150823038F580910B0AE091090AB9
:10E09000F0910A0AE80FF11D828188608283E09185
:10E0A000340FF091350F80EA8083E091340FF091C6
:10E0B000350F8091591690E08F709070880F991FDE
:10E0C0002081282B2083E091340FF091350F80912F
:10E0D000671681838AC08091340F9091350F9C011F
:10E0E000D901E8E5F6E180E101900D928150E1F778
:10E0F000ADC088E596E10E94056EDC019093330F78
:10E100008093320F009709F494C080910B0AE0913C
:10E11000090AF0910A0AE80FF11D828111969C917B
:10E12000892B82832091601630E08091A71C90E0BB
:10E130008D7F2817390771F5909161168091A81C81
:10E14000981741F580916216882321F58091631616
:10E150008F3F01F5809164168E3FE1F48091651642
:10E160008823C1F4E12FF02F9091661680819817D3
:10E1700089F4909167168181981761F480910B0A58
:10E18000E091090AF0910A0AE80FF11D82818C6082
:10E19000828365C08091601690916116892B59F534
:10E1A0008091621690916316892B29F580916416EF
:10E1B00090916516892BF9F48091661687FD1BC036
:10E1C00080910B0AE091090AF0910A0AE80FF11D0B
:10E1D000828188608283E091340FF091350F8091C5
:10E1E000661690916716918380838091340F909189
:10E1F000350F029630C080910B0AE091090AF09128
:10E200000A0AE80FF11D8281846082832091340F15
:10E210003091350FC901DC01E0E6F6E188E00190BC
:10E220000D928150E1F78091340F9091350F08964F
:10E2300012C08091340F9091350F9C01D901E8E50F
:10E24000F6E180E101900D928150E1F78091340F69
:10E250009091350F40969093350F8093340F88E25C
:10E2600080930D0A80914616813109F064C0909127
:10E27000681680916916805B904F0F9770F59091AA
:10E280006A1680916B1620EF803B920730F18F5B0E
:10E29000904F18F5E091340FF091350F8BEF80839C
:10E2A000E091340FF091350F90916B16905B809157
:10E2B00069168295807F980F9183E091340FF091D9
:10E2C000350F80916E1690916F16938382838091A3
:10E2D000340F9091350F049625C0E091340FF091E2
:10E2E000350F88EF8083E091340FF091350F8091E6
:10E2F000681690916916A0916A16B0916B16818389
:10E300009283A383B483E091340FF091350F809111
:10E310006E1690916F16968385838091340F90913D
:10E32000350F07969093350F8093340F80910D0A27
:10E33000885F80930D0A8091340F9091090A891BA0
:10E3400080930B0A1F910F9108950F931F93CF9302
:10E35000DF93EC018B010E94056E892B31F128853A
:10E3600030E08091A71C90E08D7F28173907E9F4F1
:10E3700099858091A81C9817C1F48A858823A9F4EF
:10E380008B858F3F91F48C858E3F79F48D85882322
:10E3900061F49E85F8018081981739F420E09F850B
:10E3A0008181981719F421E001C020E0822FDF91CC
:10E3B000CF911F910F910895FC0190818181009769
:10E3C00069F04091851C5091861C6091871C21E06A
:10E3D0000E947B111092881C1092871C08950F9345
:10E3E0001F93DF93CF9300D0CDB7DEB7FC0110921F
:10E3F0000D0A10920B0A1092881C1092871C8091B3
:10E40000851C9091861C90930A0A8093090A309784
:10E4100009F5809146168A33D1F480915807282F48
:10E4200030E0F901E859F94E8081873881F4F9012B
:10E43000E459F94E8289898383898A83A8E5B6E104
:10E44000349680E101900D928150E1F707C0198266
:10E450001A8204C08081898381818A838E010F5F43
:10E460001F4FC8010E94476E80910D0A482F50E04F
:10E47000E091C315F091C415E41BF50BA0910B0AB4
:10E480002A2F30E08FE690E0821B930B6091090AFF
:10E4900070910A0A8E179F0708F0C6C0CB01049638
:10E4A0004A2F50E00E94237FE091090AF0910A0A66
:10E4B0002091C3153091C415C90180709F73906C71
:10E4C000892F9927322F2227822B932B91838083A8
:10E4D0009091120F8091130F8283938380910B0A86
:10E4E0008C5F80930B0A4FE6481B487F40930C0AD1
:10E4F000E80FF11D20910D0A30E0205C394ECF016C
:10E50000B90150E00E941A7F20910B0A80910C0AF9
:10E5100090E0820F911D9093881C8093871CC80106
:10E520000E94DC7120910D0A80910C0A90E0820F0C
:10E53000911D9093110F8093100F85E080930B0A2B
:10E540002091C3153091C415E091090AF0910A0A8F
:10E55000C90180709F71906E892F9927322F2227D1
:10E56000822B932B9183808388E680930C0A42C090
:10E57000A091090AB0910A0ACF0123E096958795E8
:10E580002A95E1F714968C9314979A012E1B3F0B52
:10E5900080910C0A90E02817390720F4842F8E1BF5
:10E5A00080930C0A80910B0A9D01280F311D409128
:10E5B0000C0AE05CF94EC901BF0150E00E941A7FCD
:10E5C00020910B0A80910C0A90E0820F911D90938C
:10E5D000881C8093871CC8010E94DC7120910C0A62
:10E5E0008091100F9091110F820F911D9093110F38
:10E5F0008093100FE091100FF091110F4091C3150F
:10E600005091C415E417F50708F4B2CF8091120FAA
:10E610009091130F01969093130F8093120F109205
:10E62000110F1092100F1CC0260F371F405C594E5F
:10E63000C901BA01AF010E941A7F20910B0A809193
:10E64000C3159091C415820F911D20910D0A821B54
:10E6500091099093881C8093871CC8010E94DC71EB
:10E6600081E00F900F90CF91DF911F910F9108954E
:10E67000CF93DF932091CA1CE22FF0E0DF0124E06A
:10E68000AA0FBB1F2A95E1F7A655B34EEC0180E116
:10E6900009900D928150E1F784E0EE0FFF1F8A95FB
:10E6A000E1F7E655F34E8FEF8787DF91CF9108951D
:10E6B000FFCF0F931F93DF93CF93CDB7DEB728978C
:10E6C0000FB6F894DEBF0FBECDBF8091C3159091F9
:10E6D000C415009709F435C18150954008F022C156
:10E6E0008091581690915916892B59F580915A1698
:10E6F00090915B16892B29F580915C1690915D169F
:10E70000892BF9F480915E1690915F16892BC9F4DC
:10E710008091601690916116892B99F48091621610
:10E7200090916316892B69F4809164169091651617
:10E73000892B39F48091661690916716892B09F41C
:10E74000F1C09091CA1C913029F480910C05882366
:10E7500009F4E8C0809158168F3F09F4E8C0913061
:10E7600041F488E596E10E945B4D882311F41092F4
:10E77000CA1C88E596E10E945B4D882341F088E53C
:10E7800096E10E94254E8C01E0E0F0E00EC0809101
:10E79000CA1C813011F41092CA1C0E949249FC01DB
:10E7A000009709F4BFC0008111818091CA1C81309B
:10E7B00071F5EF2B01F52091601630E08091A71CD8
:10E7C00090E08D7F28173907B1F490916116809100
:10E7D000A81C981781F480916216882361F48091B7
:10E7E00063168F3F41F4809164168E3F21F480912F
:10E7F0006516882319F019821A8206C08091661660
:10E800008983809167168A83CE01019689C001159C
:10E81000110531F0F801818D853009F049C00AC039
:10E8200088E596E160E070E040E020E00E94824EE2
:10E830008C0102C0F801118E88E496E160E840E0A6
:10E840000E94F25F892B19F088E496E102C080E013
:10E8500090E060E070E0A8010E949B558091CA1C86
:10E8600090E029E730E0829FF001839FF00D929FB6
:10E87000F00D1124E157F44E6585768587859089E2
:10E8800028EE33E040E050E00E948581CA01B901E2
:10E8900028EE33E040E050E00E944781AB01BC012C
:10E8A000C80182960E94AA6581E0F80182A73FC054
:10E8B000882309F446C0823059F483E0F801818F3F
:10E8C000C8014A9648E853E160E070E00E94AA65FA
:10E8D0008091CA1C90E029E730E0829FF001839F7D
:10E8E000F00D929FF00D1124E157F44E6585768569
:10E8F0008785908928EE33E040E050E00E948581D2
:10E90000CA01B90128EE33E040E050E00E9447819F
:10E91000AB01BC01C80182960E94AA65C80140965D
:10E920000E94DB641092C4151092C3150AC080E0E7
:10E9300090E00E94DB641092C4151092C3151092EF
:10E94000580728960FB6F894DEBF0FBECDBFCF9103
:10E95000DF911F910F9108951F93DF93CF93CDB750
:10E96000DEB760970FB6F894DEBF0FBECDBFDC01F7
:10E970006A30710518F01C9280E031C0FB01E75746
:10E98000F34E8081882311F41C9229C010914B1CF6
:10E99000AE014F5F5F4F20E030E0113019F4EBE142
:10E9A000F0E002C0E0E0F0E0C901880F991FE80F35
:10E9B000F91FE05EF34E80819181FA01819391937A
:10E9C000AF012F5F3F4F2730310539F77F87688BC5
:10E9D000CD01BE016F5F7F4F0E94597881E0609644
:10E9E0000FB6F894DEBF0FBECDBFCF91DF911F9160
:10E9F0000895CF92DF92EF92FF920F931F93DF93D0
:10EA0000CF9300D0CDB7DEB71092CA1C08E516E14F
:10EA10008FEF92E0909359168093581610925B16E0
:10EA200010925A1610925D1610925C1610925F1694
:10EA300010925E1610926116109260161092631674
:10EA400010926216109265161092641680E092E0A1
:10EA5000909367168093661698EEE92E9FEFF92E35
:10EA6000E00EF11E89E0D70197968C93C80140977C
:10EA7000B8010E94D35D1092580780E6809340163B
:10EA8000F70111821382128281E186832FEF27839F
:10EA900080E1C82ED12CC00ED11E82E099E0D601B3
:10EAA00013969C938E931297909369168093681691
:10EAB00080E094E315969C938E93149717961C927E
:10EAC0001E921697085E1F4F82E08093701681E0B9
:10EAD000F801818313821282278B158A148A168A81
:10EAE0008091CA1C90E029E730E0829FA001839FBB
:10EAF000500D929F500D1124FA01E157F44E82A956
:10EB00008823B1F0D701D496FA01E955F44E80E19B
:10EB100001900D928150E1F781E08093CA1C0E9420
:10EB2000094A1092CA1CFC01B29681A181FD05C060
:10EB30001092C4151092C3152EC028E836E1AF011B
:10EB400080E1DA010D90AD01D9010D929D01815056
:10EB5000C1F78089F80182A711A610A681E083A7DA
:10EB60008CE590E09093C4158093C31584E390E006
:10EB70009A8389838A81D70114968C93149789810B
:10EB800015968C930E94F73C80959095F60197839B
:10EB900086830E9459730F900F90CF91DF911F9140
:10EBA0000F91FF90EF90DF90CF9008950F93CF9348
:10EBB000DF930E949249892B49F58091CA1CE82F66
:10EBC000F0E034E0EE0FFF1F3A95E1F7E655F34E23
:10EBD00087858823D9F01786CF0160E420E030E0F4
:10EBE00040E050E001E00E94964B8091CA1C90E00A
:10EBF00024E0880F991F2A95E1F78655934E60E42B
:10EC000020E030E040E050E00E94C4618091CA1CE6
:10EC100090E0C9E7D0E08C9FF0018D9FF00D9C9FA4
:10EC2000F00D1124E157F44E83898823A1F00E944E
:10EC30009249892B71F08091CA1C90E08C9FF00161
:10EC40008D9FF00D9C9FF00D1124E157F44E128A18
:10EC5000118A0E947E5F89E795E00E94620B809195
:10EC6000CA1C882319F485E895E007C0813019F49F
:10EC70008EE895E002C086E995E00E94620B8CE97F
:10EC800095E00E94620B0E9401638091CA1C813052
:10EC9000C1F480914B1C8F3F69F484EB95E00E9496
:10ECA000620B0E9420498AE090E06DEA7FE50E94B5
:10ECB000250F1BC08BE39CE10E9458690E94011242
:10ECC00014C080911B1C882381F480914B1C8F3FC2
:10ECD00061F48091D21B8F3F41F08091A41B882367
:10ECE00021F082EC9BE10E945869DF91CF910F9156
:10ECF000089580910916882359F084EE95E1909348
:10ED0000E3158093E21582E00E94B73D0E9459739B
:10ED100080913516882359F080E196E19093E315B0
:10ED20008093E21582E00E94B73D0E9459730895D6
:10ED30008091DB158830E9F4E091370FF091380FBE
:10ED40003097F9F029E33FE08091C5159091C61501
:10ED5000B901AF010E941A7F8091370F9091380F4F
:10ED60009093431B8093421B1092380F1092370FE1
:10ED70000895823031F41092431B1092421B10927E
:10ED8000AA0F0895FF920F931F93DF93CF93CDB7F0
:10ED9000DEB769970FB6F894DEBF0FBECDBFF82E71
:10EDA000092FE62F6237D0F510914B1C1130B1F5C9
:10EDB0008091370F9091380F892B81F58091AA0FA0
:10EDC000882361F56093370F1092380F29E33FE0F5
:10EDD000C901BA014E2F50E00E941A7F1093CA1C3D
:10EDE00080EF93EB9A8B898B9C8B8B8B80E48D8B44
:10EDF000DE011196EBE3FCE180E101900D92815080
:10EE0000E1F70F87F88ACE0101969093DF15809382
:10EE1000DE1585E00E94B73D0E94597369960FB6D2
:10EE2000F894DEBF0FBECDBFCF91DF911F910F9140
:10EE3000FF900895FC0120E090818181808391837F
:10EE40002E5F32962031C1F70895992787FD90955E
:10EE50000E9406828833A1F1893384F4843341F11E
:10EE600085333CF4823301F1833304F58133D1F4EB
:10EE700017C0863309F187330CF51CC0833641F186
:10EE800084363CF4813601F1823604F5893351F43D
:10EE900019C0853609F18536ECF0863619F41EC0A6
:10EEA00081E0089580E0089582E0089583E0089568
:10EEB00084E0089585E0089586E0089587E0089548
:10EEC00088E0089589E008958AE008958BE0089528
:10EED0008CE008958DE008958EE008958FE0089508
:10EEE000EF92FF921F93CF93DF937C01EC0110E030
:10EEF00001C01F5F8881992787FD90950E94F2814C
:10EF0000892B19F4C0E0D0E022C02196143089F793
:10EF1000F9CFF70180810E94257790E0143029F421
:10EF2000982F88279295907F0CC0133019F4982F52
:10EF3000882707C0123029F424E0880F991F2A95EA
:10EF4000E1F7C80FD91F11500894E11CF11C1123DF
:10EF500001F7CE01DF91CF911F91FF90EF900895BF
:10EF60005F926F927F928F929F92AF92BF92CF9259
:10EF7000DF92EF92FF920F931F93DF93CF9300D016
:10EF800000D00F92CDB7DEB74C016B018C019C0114
:10EF9000A8E0EA2EFF24F8E05F2E5E010894A11C91
:10EFA000B11CE5E06E2E712C6C0E7D1E02C00F5F51
:10EFB0001F4FF80140814A3311F04423C1F7C801C3
:10EFC000821B930B059714F080E05EC0F8018291DC
:10EFD0008F010F5F1F4F8A3319F0D501F9012FC040
:10EFE000442319F0F40190E00EC0EF2DF0E0EE0F95
:10EFF000FF1FEC0DFD1D11821082F39440C08A3377
:10F0000009F49F5F319680818823C9F7252D291B3C
:10F010009F2D822F0AC0E92FF0E0EE0FFF1FEC0DAD
:10F02000FD1D1182108281509F5F8823A1F7F20E8F
:10F03000E21A0F5F1F4F98011FC08D9331969E2FCC
:10F04000921B80818A3319F0A615B705B1F7F50137
:10F05000E90FF11D1082C5010E947077EF2DF0E0DD
:10F06000EE0FFF1FEC0DFD1D9183808398012F5F34
:10F070003F4FF394EA948901EE2009F09ACF80E0A3
:10F08000F8E0FF1609F481E00F900F900F900F90B9
:10F090000F90CF91DF911F910F91FF90EF90DF9034
:10F0A000CF90BF90AF909F908F907F906F905F9028
:10F0B0000895AF92BF92CF92DF92EF92FF920F939B
:10F0C0001F93CF93DF938C01EB016115710509F458
:10F0D00069C0EE24FF2437EDC32E35E0D32E20E3A4
:10F0E000A22E9AE3B92E88819981009779F5EE20B6
:10F0F00069F540E06F2D70E001C04F5F242F30E0D4
:10F10000F901EE0FFF1FEC0FFD1F80819181892B0C
:10F1100029F4260F371F283031057CF3413039F4AC
:10F12000D801AD928D01F394229640E02EC08F2D30
:10F1300090E0840F911D089709F44150842F90E0CE
:10F14000880F991FC80FD91FF40E1FC000D000D020
:10F1500000D0EDB7FEB73196ADB7BEB712961C938F
:10F160000E931197D382C282948385830E94A87FD5
:10F17000080F191F2296F3944E2DEDB7FEB7369661
:10F180000FB6F894FEBF0FBEEDBFF8E0FF1641F0DA
:10F19000D801BD928D01B7E0BF1510F0E42EA3CFCA
:10F1A000F8011082DF91CF911F910F91FF90EF90A6
:10F1B000DF90CF90BF90AF900895AF92BF92CF9263
:10F1C000DF92EF92FF920F931F93DF93CF9300D0C4
:10F1D00000D000D0CDB7DEB77C018AED95E00E946B
:10F1E000620B00E010E06E010894C11CD11C4CEDD4
:10F1F000A42E45E0B42E00D000D000D0EDB7FEB76D
:10F200003196ADB7BEB71296DC92CE921197B3820B
:10F21000A282D701A00FB11F8C91848315820E9416
:10F22000A87F8DB79EB706960FB6F8949EBF0FBE07
:10F230008DBFC6010E94620B0F5F1F4F0031110589
:10F24000D1F626960FB6F894DEBF0FBECDBFCF9194
:10F25000DF911F910F91FF90EF90DF90CF90BF90C3
:10F26000AF900895CF92DF92EF92FF920F931F938A
:10F27000CF93DF938C017B01EA01690188818823A8
:10F2800019F020E030E002C029813A81C9010197DC
:10F29000099740F4F901E757F34E81E08083C901F3
:10F2A0000E94002380910C05882339F4C801B7011E
:10F2B000AE0196010E94A97B05C0C801B70141E0DB
:10F2C0000E94A379DF91CF911F910F91FF90EF9052
:10F2D000DF90CF9008950F931F93CF93DF93EC01AE
:10F2E0008B0180910C05882319F4CE010E940E7BBE
:10F2F0008881833319F48981833389F020E030E0F9
:10F30000FE01E20FF31FD901A553BA4E90818C91F3
:10F310009817A1F42F5F3F4F2630310589F78C8570
:10F320009D8586589D4D51F41092CA1C0E50104078
:10F33000CE010E96B80140E00E94A379DF91CF91F3
:10F340001F910F9108951F93CF93DF939C01EB01C1
:10F35000142F8091C3159091C415892B19F02FEFAC
:10F360003FEF13C080E496E1B901AE010E94237F14
:10F370001093CA1CD093C415C093C31581E00E949A
:10F38000B73D0E94597320E030E0C901DF91CF9171
:10F390001F910895FC0171A760A70895FC01768B69
:10F3A000658B0895A091E215B091E315109719F0BF
:10F3B000FD01B89605C0E091DE15F091DF15759658
:10F3C0008091DB1586FF22C050962D913C9151977C
:10F3D0008091AD0F9091AE0F8217930731F4809119
:10F3E000AF0F9091B00F009769F48091B10F909199
:10F3F000B20F8217930751F48091B30F9091B40F1D
:10F40000009721F0918380831382128220813181C1
:10F410002115310521F082819381F9010995089523
:10F42000009749F09093E3158093E21583E00E94E2
:10F43000B73D0E9459730895009749F09093DF15E6
:10F440008093DE1585E00E94B73D0E9459730895B0
:10F45000CF93DF93EC018091AF0F9091B00F8C1799
:10F460009D0771F48091AD0F9091AE0F0E94E13B2A
:10F470001092AE0F1092AD0F1092B00F1092AF0F0E
:10F480008091B30F9091B40F8C179D0771F4809108
:10F49000B10F9091B20F0E94E13B1092B20F109207
:10F4A000B10F1092B40F1092B30FE9E0F6E183812F
:10F4B00094818C179D0719F4148213821082BC96D4
:10F4C000CF0185978C53964190F3E4E4FBE1858965
:10F4D00096898C179D0711F4118A108A79968BE111
:10F4E000E637F807A0F3DF91CF910895AC011092B1
:10F4F000AC0FEDEAFFE020E014C080819181841719
:10F50000950769F4828193818617970741F42093C8
:10F51000AC0F11821082CA010E94E13B089534961B
:10F520002F5F223050F32093AC0F0895CF93DF93D9
:10F53000EA010E94FE46FC01009711F0D68BC58BB4
:10F54000CF01DF91CF9108950F931F93DF93CF9356
:10F55000CDB7DEB760970FB6F894DEBF0FBECDBF54
:10F560008C01AB018FEF92E09A8389831C821B820E
:10F570001E821D8218861F821A8619861C861B868B
:10F580001E861D8680E091E0988B8F87CE010196C4
:10F59000B8010E94967AFC01009711F0118B008B44
:10F5A000CF0160960FB6F894DEBF0FBECDBFCF91EE
:10F5B000DF911F910F910895AC011092AB0FEDEA0E
:10F5C000FFE020E012C0322F3F5F80819181892BC4
:10F5D00051F42093AB0F5183408373836283CA013C
:10F5E0000E94FE3B08953496232F223060F320932F
:10F5F000AB0F08950F931F93CF93DF938A010E945F
:10F60000373CEC01009721F019A708A70E94107A57
:10F61000CE01DF91CF911F910F910895CF92DF928C
:10F62000EF92FF920F931F93DF93CF93CDB7DEB787
:10F6300066970FB6F894DEBF0FBECDBF8C01FC01FC
:10F640002081233381F48181833369F4828188238B
:10F6500031F48091B90F89838091B80F2DC08F3F0D
:10F6600011F4F80112C08091A71C8C7082602817D9
:10F6700081F4F80191818091A81C981751F482813E
:10F68000882339F48381882321F4848189838581C7
:10F6900013C0F8018281882309F04CC0838188233C
:10F6A00009F048C08481882309F044C085818823FB
:10F6B00009F040C0298381818A83F801848595857A
:10F6C00086589D4DB9F5DE011996E0E4F6E18EE02D
:10F6D00001900D928150E1F792EFE92E9FEFF92E04
:10F6E000E60EF71EF092C415E092C3158EE0C82E08
:10F6F000D12CC00ED11E80E496E1B601A7010E9474
:10F70000237FCE0101960E94EF7126E1003412079B
:10F7100069F4C601B801A7010E94237FD801FE0148
:10F7200039968EE001900D928150E1F71092C41548
:10F730001092C31566960FB6F894DEBF0FBECDBF0C
:10F74000CF91DF911F910F91FF90EF90DF90CF90BD
:10F750000895EF92FF920F931F93CF93DF939C0135
:10F760008B017A0180E496E1B901A8010E94237F10
:10F770001092CA1C809158168F3F09F4B4C088E5D6
:10F7800096E10E945B4D882331F088E596E10E9466
:10F79000254EEC0108C00E949249FC01009709F433
:10F7A000F5C0C081D181209729F0898D853009F07D
:10F7B00047C00AC088E596E160E070E040E020E0E4
:10F7C0000E94824EEC0101C0198E88E496E160E847
:10F7D00040E00E94F25F892B19F088E496E102C0B4
:10F7E00080E090E060E070E0AE010E949B55809167
:10F7F000CA1C90E029E730E0829FF001839FF00D62
:10F80000929FF00D1124E157F44E6585768587852A
:10F81000908928EE33E040E050E00E948581CA01E3
:10F82000B90128EE33E040E050E00E944781AB018F
:10F83000BC01CE0182960E94AA6581E08AA75AC0C7
:10F84000882309F4A3C0823051F483E0898FCE016C
:10F850004A9648E853E160E070E00E94AA65809112
:10F86000CA1C90E029E730E0829FF001839FF00DF1
:10F87000929FF00D1124E157F44E658576858785BA
:10F88000908928EE33E040E050E00E948581CA0173
:10F89000B90128EE33E040E050E00E944781AB011F
:10F8A000BC01CE0182960E94AA658EE496E160E4D6
:10F8B00076E1A8010E94237F809166168F3FD1F0E8
:10F8C0008889809340168989809341168A8980931C
:10F8D00042168B89809343168C89809344168D89B8
:10F8E0008093451607C08EE496E160E476E1A801B6
:10F8F0000E94237F809166168F3FE9F483E3809313
:10F900004016809341168091721680934216809122
:10F9100073168093431680917416809344168091D9
:10F92000751680934516A7EBBFE0F70189E00190BB
:10F930000D928150E1F78091A71C8C7082608093BA
:10F9400046168091A81C8093471610924816109274
:10F950004916F701828180934A16818180934B1664
:10F9600086E880934C168DED80934D16B801625F4A
:10F970007F4F7093C4156093C31580E496E141E016
:10F980000E94EF331092C4151092C315DF91CF91EE
:10F990001F910F91FF90EF900895ABE0B0E0E3ED81
:10F9A000FCE70C94AB815C014B017A01FC011782EE
:10F9B0001682838181FD08C06FEF7FEF08C142E0AE
:10F9C00050E0E40EF51E04C03E010894611C711C59
:10F9D000F501D380F401D3FC8591D3FE81914F01D1
:10F9E000882309F4F1C0853259F4D3FC6591D3FE24
:10F9F00061914F01653219F0062F10E01BC085E2BE
:10FA000090E02BC0002309F4DFC08EE399E0602F63
:10FA100070E00E94F37E892B39F4033211F41061F7
:10FA200003C00C3661F41068F401D3FC0591D3FED9
:10FA300001914F0117FFE6CF002309F4C5C087E30A
:10FA400099E0602F70E00E94F37E892B51F044E032
:10FA500050E0E40EF51E8FE390E0B5010E947C7F3C
:10FA6000B7CF033629F0033779F00335F1F40BC033
:10FA700087010E5F1F4FF70180819181B5010E94C0
:10FA80007C7F7801A5CF1160F701C080D18004C0D0
:10FA900090E0B5010E947C7FF60110FD859110FF7A
:10FAA00081916F018823A1F78ACF043611F00936BE
:10FAB00039F517FF08C0F701208131814281538158
:10FAC00084E090E00AC0F701808191819C01442785
:10FAD00037FD4095542F82E090E0E80EF91E1F7E1E
:10FAE00057FF08C050954095309521953F4F4F4F97
:10FAF0005F4F1064CA01B901A3012AE030E034C0AD
:10FB00000037A9F0013730F40835B1F00F3609F0AD
:10FB10005BC006C0053739F0083709F055C008C08A
:10FB200028E030E00CC01F7E2AE030E008C0106101
:10FB3000146220E130E003C0146020E132E017FFDE
:10FB400008C0F701608171818281938144E050E0B7
:10FB500008C0F70180819181BC0180E090E042E023
:10FB600050E0E40EF51EA3010E94CC7FD82ED618DB
:10FB7000012F10E006FF05C08DE290E0B5010E9464
:10FB80007C7F04FF15C0FE01ED0DF11D80818033E7
:10FB900079F080E390E0B5010E947C7F02FF08C00D
:10FBA00000721070C801885A9F4FB5010E947C7F77
:10FBB000DA94F301ED0DF11D808190E0B5010E9412
:10FBC0007C7FDD20A9F704CFF50166817781CB0129
:10FBD0002B96EEE00C94C781EF92FF920F93DF9388
:10FBE000CF93CDB7DEB760970FB6F894DEBF0FBEE8
:10FBF000CDBFA82F002309F461C07E010894E11C49
:10FC0000F11C88E0F70111928A95E9F729833A837C
:10FC10004B835C836D837E83AF83988780E2801BF8
:10FC2000E82FFF27E7FDF0954D815E816F81788594
:10FC3000181684F01D861E861F86188A8827992725
:10FC40008E1B9F0B04C076956795579547958A95AF
:10FC5000D2F728C0202F332727FD3095DB01CA01BA
:10FC6000022E04C0B695A795979587950A94D2F76A
:10FC70008D879E87AF87B88B04C0440F551F661FC2
:10FC8000771FEA95D2F789819A81AB81BC8104C044
:10FC9000B695A795979587952A95D2F7482B592B16
:10FCA0006A2B7B2B49875A876B877C8729853A8506
:10FCB0004B855C856D857E85AF8598898A2F60969A
:10FCC0000FB6F894DEBF0FBECDBFCF91DF910F917D
:10FCD000FF90EF900895A0E0B0E0E1E7FEE70C941C
:10FCE000AF81EC01A880B980CA80DB80A114B10487
:10FCF000C104D10441F484E2A82E89EDB82E8BE52D
:10FD0000C82E87E0D82EC601B5012DE133EF41E0C2
:10FD100050E00E940E8227EA31E440E050E00E9469
:10FD200047817B018C01C601B5012DE133EF41E034
:10FD300050E00E940E82CA01B9012CEE34EF4FEF61
:10FD40005FEF0E9447816E0D7F1D801F911F97FFFF
:10FD500004C06150704080409048688379838A83F2
:10FD60009B839B013F77C901CDB7DEB7EAE00C94D6
:10FD7000CB810E946B7E089583EE95E00E946B7E9E
:10FD80000895A0E0B0E08093E3059093E405A0938C
:10FD9000E505B093E6050895FC0188279927E894C6
:10FDA00021912032E9F3293010F02E30C8F32B32A4
:10FDB00041F02D3239F4689404C00E94747F820FA0
:10FDC000911D219120532A30C0F31EF49095819506
:10FDD0009F4F0895FB01DC0102C005900D92415038
:10FDE0005040D8F70895FC010590061621F0002038
:10FDF000D9F7C00108953197CF010895FB01DC01C7
:10FE00004150504048F005900D920020C9F701C0C4
:10FE10001D9241505040E0F70895FB01DC0104C001
:10FE20008D910190801921F441505040C8F7881BF2
:10FE3000990B0895FB01DC0102C001900D92415025
:10FE40005040D8F708956817790768F4FB01DC0182
:10FE5000E40FF51FA40FB51F02C002900E9241508F
:10FE60005040D8F708950C941A7FDC0101C06D93BF
:10FE700041505040E0F70895A0E0B0E0E2E4FFE731
:10FE80000C94B1817C01EB018A01690109C0CE01AA
:10FE90002196F6010995F70181937F0101501040E9
:10FEA00001151105A1F7CDB7DEB7E8E00C94CD81BF
:10FEB000A0E0B0E0EEE5FFE70C94B181EC017B013E
:10FEC0008A01690109C0CE012196F70161917F0184
:10FED000F60109950150104001151105A1F7CDB7A4
:10FEE000DEB7E8E00C94CD817AE0979F902D879F54
:10FEF000802D910D112408950F931F93CF93DF93BD
:10FF00008C01EB018B8181FF1BC082FF0DC02E8114
:10FF10003F818C819D812817390764F4E881F9813C
:10FF20000193F983E88306C0E885F985802F099558
:10FF3000892B31F48E819F8101969F838E8302C02D
:10FF40000FEF1FEFC801DF91CF911F910F9108951F
:10FF5000AEE0B0E0EEEAFFE70C94B5810D891E89B2
:10FF600086E08C831A8309838FEF9FE79E838D83BE
:10FF70009E01275E3F4FCE0101966F89788DA901C2
:10FF80000E94CD7C2F813885020F131FF80110824B
:10FF90002E96E4E00C94D181FA01AA27283051F181
:10FFA000203181F1E8946F936E7F6E5F7F4F8F4FAA
:10FFB0009F4FAF4FB1E03ED0B4E03CD0670F781F09
:10FFC000891F9A1FA11D680F791F8A1F911DA11DEE
:10FFD0006A0F711D811D911DA11D20D009F4689427
:10FFE0003F912AE0269F11243019305D3193DEF6CF
:10FFF000CF010895462F4770405D4193B3E00FD085
:020000021000EC
:10000000C9F7F6CF462F4F70405D4A3318F0495D6F
:1000100031FD4052419302D0A9F7EACFB4E0A69552
:100020009795879577956795BA95C9F70097610574
:10003000710508959B01AC010A2E069457954795CA
:1000400037952795BA95C9F7620F731F841F951FBF
:10005000A01D089570D088F09F5790F0B92F992770
:10006000B751A0F0D1F0660F771F881F991F1AF0C3
:10007000BA95C9F712C0B13081F077D0B1E00895D8
:1000800074C0672F782F8827B85F39F0B93FCCF359
:10009000869577956795B395D9F73EF490958095B9
:1000A000709561957F4F8F4F9F4F0895E89409C0D9
:1000B00097FB3EF490958095709561957F4F8F4F9B
:1000C0009F4F9923A9F0F92F96E9BB279395F695B1
:1000D000879577956795B795F111F8CFFAF4BB0F2F
:1000E00011F460FF1BC06F5F7F4F8F4F9F4F16C093
:1000F000882311F096E911C0772321F09EE8872F1D
:10010000762F05C0662371F096E8862F70E060E0D8
:100110002AF09A95660F771F881FDAF7880F969551
:10012000879597F9089557FD9058440F551F59F03A
:100130005F3F71F04795880F97FB991F61F09F3FD4
:1001400079F087950895121613061406551FF2CFFD
:100150004695F1DF08C0161617061806991FF1CF4D
:1001600086957105610508940895E894BB27662774
:100170007727CB0197F908950BD078C069D028F084
:100180006ED018F0952309F05AC05FC01124EECF4D
:10019000CADFA0F3959FD1F3950F50E0551F629FE2
:1001A000F001729FBB27F00DB11D639FAA27F00DD0
:1001B000B11DAA1F649F6627B00DA11D661F829FF7
:1001C0002227B00DA11D621F739FB00DA11D621FDC
:1001D000839FA00D611D221F749F3327A00D611DF9
:1001E000231F849F600D211D822F762F6A2F1124DB
:1001F0009F5750408AF0E1F088234AF0EE0FFF1F2E
:10020000BB1F661F771F881F91505040A9F79E3F64
:10021000510570F014C0AACF5F3FECF3983EDCF3B9
:10022000869577956795B795F795E7959F5FC1F7A1
:10023000FE2B880F911D9695879597F9089597F94C
:100240009F6780E870E060E008959FEF80EC08957C
:1002500000240A94161617061806090608950024A5
:100260000A9412161306140605060895092E03941F
:10027000000C11F4882352F0BB0F40F4BF2B11F493
:1002800060FF04C06F5F7F4F8F4F9F4F0895629F45
:10029000D001739FF001829FE00DF11D649FE00D7E
:1002A000F11D929FF00D839FF00D749FF00D659FDF
:1002B000F00D9927729FB00DE11DF91F639FB00DDE
:1002C000E11DF91FBD01CF0111240895991B79E0AB
:1002D00004C0991F961708F0961B881F7A95C9F7D6
:1002E0008095089597FB092E07260AD077FD04D044
:1002F00065D006D000201AF4709561957F4F08955F
:10030000F6F7909581959F4F0895A1E21A2EAA1BAA
:10031000BB1BFD010DC0AA1FBB1FEE1FFF1FA217B5
:10032000B307E407F50720F0A21BB30BE40BF50BB2
:10033000661F771F881F991F1A9469F7609570953B
:10034000809590959B01AC01BD01CF0108952F923E
:100350003F924F925F926F927F928F929F92AF9255
:10036000BF92CF92DF92EF92FF920F931F93CF93A2
:10037000DF93CDB7DEB7CA1BDB0B0FB6F894DEBF39
:100380000FBECDBF09942A88398848885F846E845F
:100390007D848C849B84AA84B984C884DF80EE80A9
:1003A000FD800C811B81AA81B981CE0FD11D0FB6B2
:1003B000F894DEBF0FBECDBFED010895AA1BBB1B95
:1003C00051E107C0AA1FBB1FA617B70710F0A61B55
:1003D000B70B881F991F5A95A9F780959095BC0176
:1003E000CD010895911106C080538A5010F0865CAB
:1003F00006C0089599278827089585FDFBCF806260
:100400009111F8CF81568A51E0F70895911108951E
:1004100081548A5108F4805E855A089597FB092E0D
:1004200005260ED057FD04D070DF0AD0001C38F42A
:1004300050954095309521953F4F4F4F5F4F089510
:10044000F6F790958095709561957F4F8F4F9F4FF0
:0204500008950D
:1004520080E803252D313573202D20253032582098
:10046200000D0A002564000D0A73686F7274203D46
:1004720020253034580D0A706172656E74203D205B
:10048200253034580D0A726F7574653D2530345825
:100492000D0A006368616E203D2025640D0A002567
:1004A20078006C6F6E67203D2030782530386C58AC
:1004B2002530386C580D0A0066616C7365007472E1
:1004C2007565006173736F63203D2025730D0A48C3
:1004D2006F7073203D20253034580D0A0072616E12
:1004E20064203D20253032580D0A0025752C2052FB
:1004F20065763D25640D0A00536C656570203D20CC
:1005020025730D0A005965730046726571203D20FE
:1005120025644D487A0D0A00364C6F5750414E20E3
:100522003D2025730D0A0044656D6F206D6F646573
:10053200203D2025730D0A004E6F005452585F5320
:1005420054415455530000000000005452585F5368
:1005520054415445000000000000005452585F43CB
:1005620054524C5F300000000000005452585F4368
:1005720054524C5F310000000000005048595F5453
:10058200585F5057520000000000005048595F5217
:1005920053534900000000000000005048595F45D5
:1005A200445F4C4556454C000000005048595F439B
:1005B200435F4343410000000000004343415F5456
:1005C20048524553000000000000005452585F4357
:1005D20054524C5F320000000000004952515F4DFE
:1005E20041534B00000000000000004952515F538C
:1005F2005441545553000000000000565245475FD5
:100602004354524C000000000000004241544D4F40
:100612004E00000000000000000000584F53435FEE
:100622004354524C0000000000000052585F5359DE
:100632004E0000000000000000000052465F4354DC
:10064200524C5F30000000000000005841485F43F8
:1006520054524C5F3100000000000046544E5F438C
:1006620054524C000000000000000052465F435408
:10067200524C5F3100000000000000504C4C5F43C0
:100682004600000000000000000000504C4C5F4497
:100692004355000000000000000000504152545F2A
:1006A2004E554D00000000000000005645525349CF
:1006B2004F4E5F4E554D00000000004D414E5F49C8
:1006C200445F3000000000000000004D414E5F49D1
:1006D200445F31000000000000000053484F5254B4
:1006E2005F414444525F300000000053484F52546F
:1006F2005F414444525F310000000050414E5F4967
:10070200445F30000000000000000050414E5F498D
:10071200445F310000000000000000494545455F8C
:10072200414444525F300000000000494545455FA6
:10073200414444525F310000000000494545455F95
:10074200414444525F320000000000494545455F84
:10075200414444525F330000000000494545455F73
:10076200414444525F340000000000494545455F62
:10077200414444525F350000000000494545455F51
:10078200414444525F360000000000494545455F40
:10079200414444525F3700000000005841485F4323
:1007A20054524C5F3000000000000043534D415F43
:1007B200534545445F30000000000043534D415F04
:1007C200534545445F31000000000043534D415FF3
:1007D2004245000000000000000000010203040581
:1007E200060708090C0E0F10111215161718161A03
:1007F2001B1C1D1E1F202122232425262728292ACF
:100802002B2C2D2E2F2563253032582025632530A1
:10081200325820253032582030782530386C58250F
:1008220030386C580D0A00256325303258200043B9
:100832004352450025780030782530386C582530F1
:10084200386C5820202020253034582020202020A9
:1008520020200025640014000F000300000101267F
:100862000300000000000000000000000000000083
:100872000000000000000000000000000000000076
:10088200000000000030782530386C582530386C74
:100892005800AAABACADAEAF3A3B3C3D3E3F012364
:1008A20083927834200000ADBA20202025642009EC
:1008B20009202020256409090020010470B0660087
:1008C200010000000000000000525320446F6E65DA
:1008D200206F6E200045746865726E657400364C38
:1008E2006F7750414E004F74686572002C2041733F
:1008F2007369676E6564206164647265737365739E
:100902003A0D0A004E6F20676C6F62616C20616461
:1009120064726573732C2072657374617274696E8C
:10092200672052530D0A00257800200025303278C6
:080932000006020100000000B4
:10FC00002F923F924F925F926F927F928F929F922C
:10FC1000AF92BF92CF92DF92EF92FF920F931F931A
:10FC2000DF93CF9300D000D0CDB7DEB7F8948091AA
:10FC3000811390918213A0918313B09184138983CF
:10FC40009A83AB83BC83612C712C91E0892E912C1B
:10FC500071E065E052C0F999FECF93E0F101409266
:10FC60005B0090935700E89507B600FCFDCFA1E13B
:10FC7000A0935700E89507B606FCFDCF6401530139
:10FC8000EE24FF248701CBBEF501279137914791E0
:10FC90005691D801C701820D931DA41DB51D090100
:10FCA000FC01A0935B0070935700E895112482E05B
:10FCB00090E0A0E0B0E0A80EB91ECA1EDB1EE80E60
:10FCC000F91E0A1F1B1F90E0E91691E0F90690E06B
:10FCD000090790E01907B9F680E091E0A0E0B0E0F4
:10FCE000680E791E8A1E9B1EF10140925B00609394
:10FCF0005700E89507B600FCFDCF212C312C8FEF83
:10FD0000482E8FEF582E260C371C481C591C898111
:10FD10009A81AB81BC81681679068A069B0608F435
:10FD20009ACF81E180935700E8952BE088E190E03D
:10FD30000FB6F894A895809360000FBE20936000E2
:10FD4000FFCFAF92BF92CF92DF92EF92FF920F93CD
:10FD50001F93CF93DF937B018C016A01AFB6F894B8
:10FD6000F999FECF83E0F70100935B008093570081
:10FD7000E89507B600FCFDCF40E050E060E070E0A1
:10FD8000BB24B394F6018081D181C0E09E01280F8D
:10FD9000311D82E090E0C80ED91EDB01CA018E0D34
:10FDA0009F1DA01FB11F0901FC01A0935B00B09231
:10FDB0005700E89511244E5F5F4F6F4F7F4F4030E3
:10FDC00091E0590790E0690790E07907D9F685E05E
:10FDD000F70100935B0080935700E89507B600FC9D
:10FDE000FDCF81E180935700E895AFBEDF91CF91C1
:10FDF0001F910F91FF90EF90DF90CF90BF90AF9049
:02FE0000089563
:00000001FF
